:020000040800F2
:100000000080002099DF000871DF000873DF00081E
:1000100075DF000877DF000879DF000800000000C6
:100020000000000000000000000000007BDF00086E
:100030007DDF0008000000007FDF000881DF00088E
:10004000E9DF0008E9DF0008E9DF0008E9DF000870
:10005000E9DF0008E9DF0008E9DF0008E9DF000860
:10006000E9DF0008E9DF0008E9DF0008E9DF000850
:10007000E9DF0008E9DF0008E9DF0008E9DF000840
:10008000E9DF000800000000E9DF0008E9DF000800
:10009000A11C0108E9DF0008E9DF0008E9DF00082A
:1000A000E9DF0008E9DF0008E9DF0008E9DF000810
:1000B000E9DF0008E9DF0008E9DF0008E9DF000800
:1000C000E9DF0008E9DF0008E9DF0008E9DF0008F0
:1000D000E9DF0008E131000849640008E9DF0008B1
:1000E0000DC90008E9DF0008E9DF0008E9DF0008C2
:1000F000E9DF0008E9DF0008E9DF00080000000090
:1001000000000000E9DF000800000000E9DF00084F
:10011000E9DF000800000000E9DF0008E9DF00086F
:10012000E9DF0008E9DF0008E9DF0008E9DF00088F
:10013000E9DF00080000000000000000E9DF00081F
:10014000E9DF0008E9DF000800000000000000000F
:10015000000000000000000000000000000000009F
:10016000000000000000000000000000E9DF0008BF
:10017000E9DF0008000000000000000000000000AF
:1001800000000000E9DF000800000000000000009F
:10019000000000000000000000000000000000005F
:1001A0000000000000000000E9DF0008E93400085A
:1001B000E9DF0008E9DF0008E9DF000800000000CF
:1001C00000000000E9DF000800000000000000005F
:0801D000E9DF0008E9DF000887
:1001D80010B5054C237833B9044B13B10448AFF379
:1001E80000800123237010BDB00300200000000030
:1001F8005C3D010808B5034B1BB103490348AFF345
:10020800008008BD00000000B40300205C3D010828
:1002180010F8012B11F8013B012A28BF9A42F7D0A8
:10022800D01A7047034613F8012B002AFBD1181A7D
:100238000138704781F0004102E000BF83F00043BD
:1002480030B54FEA41044FEA430594EA050F08BF69
:1002580090EA020F1FBF54EA000C55EA020C7FEA2D
:10026800645C7FEA655C00F0E2804FEA5454D4EBAA
:100278005555B8BF6D420CDD2C4480EA020281EA74
:10028800030382EA000083EA010180EA020281EAAC
:100298000303362D88BF30BD11F0004F4FEA0131FE
:1002A8004FF4801C4CEA113102D0404261EB41010D
:1002B80013F0004F4FEA03334CEA133302D0524293
:1002C80063EB430394EA050F00F0A780A4F101044F
:1002D800D5F1200E0DDB02FA0EFC22FA05F2801889
:1002E80041F1000103FA0EF2801843FA05F359416F
:1002F8000EE0A5F120050EF1200E012A03FA0EFCEE
:1003080028BF4CF0020C43FA05F3C01851EBE37117
:1003180001F0004507D54FF0000EDCF1000C7EEB34
:1003280000006EEB0101B1F5801F1BD3B1F5001F72
:100338000CD349085FEA30004FEA3C0C04F1010491
:100348004FEA445212F5800F80F09A80BCF1004FBA
:1003580008BF5FEA500C50F1000041EB045141EA3C
:10036800050130BD5FEA4C0C404141EB0101013C05
:1003780028BFB1F5801FE9D291F0000F04BF0146F4
:100388000020B1FA81F308BF2033A3F10B03B3F1C6
:1003980020020CDA0C3208DD02F1140CC2F10C0256
:1003A80001FA0CF021FA02F10CE002F11402D8BFB4
:1003B800C2F1200C01FA02F120FA0CFCDCBF41EA80
:1003C8000C019040E41AA2BF01EB0451294330BD4F
:1003D8006FEA04041F3C1CDA0C340EDC04F114042C
:1003E800C4F1200220FA04F001FA02F340EA030003
:1003F80021FA04F345EA030130BDC4F10C04C4F149
:10040800200220FA02F001FA04F340EA0300294628
:1004180030BD21FA04F0294630BD94F0000F83F472
:10042800801306BF81F480110134013D4EE77FEA55
:10043800645C18BF7FEA655C29D094EA050F08BFA1
:1004480090EA020F05D054EA000C04BF1946104682
:1004580030BD91EA030F1EBF0021002030BD5FEAC6
:10046800545C05D14000494128BF41F0004130BDEE
:1004780014F580043CBF01F5801130BD01F0004542
:1004880045F0FE4141F470014FF0000030BD7FEAB5
:10049800645C1ABF194610467FEA655C1CBF0B46B0
:1004A800024650EA013406BF52EA033591EA030FC7
:1004B80041F4002130BD00BF90F0000F04BF0021BF
:1004C800704730B54FF4806404F132044FF00005F2
:1004D8004FF0000150E700BF90F0000F04BF00216B
:1004E800704730B54FF4806404F1320410F00045D1
:1004F80048BF40424FF000013EE700BF42004FEACC
:10050800E2014FEA31014FEA02701FBF12F07F4348
:1005180093F07F4F81F06051704732F07F4208BFFF
:10052800704793F07F4F04BF41F40021704730B506
:100538004FF4607401F0004521F000411CE700BF52
:1005480050EA010208BF704730B54FF000050AE0D5
:1005580050EA010208BF704730B511F0004502D5D6
:10056800404261EB41014FF4806404F132045FEAD8
:10057800915C3FF4D8AE4FF003025FEADC0C18BF81
:1005880003325FEADC0C18BF033202EBDC02C2F173
:10059800200300FA03FC20FA02F001FA03FE40EA05
:1005A8000E0021FA02F11444BDE600BF70B54FF009
:1005B800FF0C4CF4E06C1CEA11541DBF1CEA1355E7
:1005C80094EA0C0F95EA0C0F00F0DEF82C4481EA4F
:1005D800030621EA4C5123EA4C5350EA013518BF6F
:1005E80052EA033541F4801143F4801338D0A0FB5C
:1005F80002CE4FF00005E1FB02E506F00042E0FB09
:1006080003E54FF00006E1FB03569CF0000F18BF0E
:100618004EF0010EA4F1FF04B6F5007F64F54074B6
:1006280004D25FEA4E0E6D4146EB060642EAC62149
:1006380041EA55514FEAC52040EA5E504FEACE2EB6
:10064800B4F1FD0C88BFBCF5E06F1ED8BEF1004FB9
:1006580008BF5FEA500E50F1000041EB045170BD35
:1006680006F0004646EA010140EA020081EA030179
:10067800B4EB5C04C2BFD4EB0C0541EA045170BD75
:1006880041F480114FF0000E013C00F3AB8014F1EF
:10069800360FDEBF002001F0004170BDC4F1000438
:1006A800203C35DA0C341BDC04F11404C4F12005B9
:1006B80000FA05F320FA04F001FA05F240EA020014
:1006C80001F0004221F0004110EBD37021FA04F64A
:1006D80042EB06015EEA430E08BF20EAD37070BD04
:1006E800C4F10C04C4F1200500FA04F320FA05F063
:1006F80001FA04F240EA020001F0004110EBD37065
:1007080041F100015EEA430E08BF20EAD37070BDD4
:10071800C4F1200500FA05F24EEA020E20FA04F3AD
:1007280001FA05F243EA020321FA04F001F000415C
:1007380021FA04F220EA020000EBD3705EEA430ECD
:1007480008BF20EAD37070BD94F0000F0FD101F0FC
:100758000046400041EB010111F4801F08BF013C35
:10076800F7D041EA060195F0000F18BF704703F073
:100778000046520043EB030313F4801F08BF013DFA
:10078800F7D043EA0603704794EA0C0F0CEA1355B6
:1007980018BF95EA0C0F0CD050EA410618BF52EA70
:1007A8004306D1D181EA030101F000414FF0000076
:1007B80070BD50EA410606BF1046194652EA430684
:1007C80019D094EA0C0F02D150EA013613D195EAF8
:1007D8000C0F05D152EA03361CBF104619460AD140
:1007E80081EA030101F0004141F0FE4141F470014A
:1007F8004FF0000070BD41F0FE4141F4780170BD3A
:1008080070B54FF0FF0C4CF4E06C1CEA11541DBF9E
:100818001CEA135594EA0C0F95EA0C0F00F0A7F8A0
:10082800A4EB050481EA030E52EA03354FEA0131CD
:1008380000F088804FEA03334FF0805545EA1313E0
:1008480043EA12634FEA022245EA111545EA1065A8
:100858004FEA00260EF000419D4208BF964244F13F
:10086800FD0404F5407402D25B084FEA3202B61A5E
:1008780065EB03055B084FEA32024FF480104FF432
:10088800002CB6EB020E75EB030E22BFB61A7546A6
:1008980040EA0C005B084FEA3202B6EB020E75EB39
:1008A800030E22BFB61A754640EA5C005B084FEAA1
:1008B8003202B6EB020E75EB030E22BFB61A75466E
:1008C80040EA9C005B084FEA3202B6EB020E75EB79
:1008D800030E22BFB61A754640EADC0055EA060E3A
:1008E80018D04FEA051545EA16754FEA06164FEA7D
:1008F800C30343EA52734FEAC2025FEA1C1CC0D129
:1009080011F4801F0BD141EA00014FF000004FF0B5
:10091800004CB6E711F4801F04BF01430020B4F176
:10092800FD0C88BFBCF5E06F3FF6AFAEB5EB030C2E
:1009380004BFB6EB020C5FEA500C50F1000041EB2B
:10094800045170BD0EF0004E4EEA113114EB5C04F8
:10095800C2BFD4EB0C0541EA045170BD41F48011CB
:100968004FF0000E013C90E645EA060E8DE60CEAD3
:10097800135594EA0C0F08BF95EA0C0F3FF43BAFF0
:1009880094EA0C0F0AD150EA01347FF434AF95EAA7
:100998000C0F7FF425AF104619462CE795EA0C0F8B
:1009A80006D152EA03353FF4FDAE1046194622E758
:1009B80050EA410618BF52EA43067FF4C5AE50EA32
:1009C80041047FF40DAF52EA43057FF4EBAE12E722
:1009D8004A0011D212F5001211D20DD56FF47873B6
:1009E800B3EB62520ED44FEAC12343F0004343EA0B
:1009F800505323FA02F070474FF00000704750EA56
:100A0800013002D14FF0FF3070474FF000007047BF
:100A180053B94AB9002908BF00281CBF4FF0FF315D
:100A28004FF0FF3000F070B9ADF1080C6DE904CE5D
:100A380000F006F8DDF804E0DDE9022304B07047B1
:100A48002DE9F047089E0D4604460F46002B4AD173
:100A58008A42944665D9B2FA82F343B102FA03FC9A
:100A6800C3F120029F4020FA02F217439C404FEA4C
:100A78001C4E1FFA8CF5B7FBFEF1220C0EFB11770A
:100A880042EA074201FB05F090420AD91CEB020238
:100A980001F1FF3780F01C81904240F21981023940
:100AA8006244121AA4B2B2FBFEF00EFB102244EA12
:100AB800024400FB05F5A5420AD91CEB040400F129
:100AC800FF3280F00781A54240F204816444023875
:100AD80040EA0140641B00211EB1DC400023C6E946
:100AE8000043BDE8F0878B4208D9002E00F0ED8066
:100AF8000021C6E900050846BDE8F087B3FA83F18E
:100B0800002949D1AB4202D3824200F2F880841A0C
:100B180065EB030201201746002EE2D0C6E9004724
:100B2800DFE702B9FFDEB2FA82F3002B40F09080D3
:100B38008A1A4FEA1C471FFA8CFE0121B2FBF7F50F
:100B480007FB1520220C42EA00420EFB05F09042FA
:100B580008D91CEB020205F1FF3802D2904200F2DC
:100B6800CB804546121AA4B2B2FBF7F007FB10225D
:100B780044EA02440EFB00FEA64508D91CEB040417
:100B880000F1FF3202D2A64500F2BB801046A4EB6A
:100B98000E0440EA05409FE7C1F120078B4022FA86
:100BA80007FC4CEA030C05FA01F420FA07F3FD40B0
:100BB8004FEA1C492343B5FBF9F81FFA8CFE09FBE1
:100BC80018551C0C44EA054408FB0EF5A54202FA28
:100BD80001F200FA01F00BD91CEB040408F1FF3A0A
:100BE80080F08880A54240F28580A8F1020864441C
:100BF800641B9DB2B4FBF9F309FB134445EA0444B2
:100C080003FB0EFEA64508D91CEB040403F1FF35CF
:100C18006CD2A6456AD9023B644443EA0843A3FB65
:100C28000295A4EB0E04AC42C846AE4656D353D048
:100C380056B1B0EB080264EB0E0404FA07F7CA4099
:100C4800CC401743C6E9007418460021BDE8F08778
:100C5800C3F1200102FA03FC20FA01F225FA01F19E
:100C68009D402A434FEA1C471FFA8CFEB1FBF7F060
:100C780007FB1015110C41EA054100FB0EF58D42EA
:100C880004FA03F408D91CEB010100F1FF382FD254
:100C98008D422DD902386144491B92B2B1FBF7F558
:100CA80007FB151142EA014205FB0EF1914208D9F2
:100CB8001CEB020205F1FF3816D2914214D9023D0D
:100CC8006244521A45EA004138E73146304608E79F
:100CD8003946E6E61046FBE64845A9D2B9EB0208D4
:100CE80065EB0C0E013BA3E74546EAE72B4694E784
:100CF8004046D1E7D0467BE7023D624432E70846EA
:100D08000AE76444023842E7704700BF0022427095
:100D180082700122C270B1FA81F10222490902717E
:100D2800032201704271704743788B421FD001291A
:100D380041700AD0022910D0C1B90123C370817053
:100D480002230371032343717047037843B10123DE
:100D580083700223C3700023F3E70378002BF6D0D7
:100D6800022383700023C3700123EAE7FEE770477C
:100D780082B00B88ADF800304B88ADF802308B8814
:100D8800ADF80430CB88ADF806300239431C053085
:100D980013F8012F0DF1080C0CEB4202834232F8D4
:100DA800082C21F8022FF3D102B0704710B50C4679
:100DB8001146FFF7B9FF2146BDE81040FFF7D8BF3D
:100DC8000A4B10B54FF07F32C0E923234FF47F431D
:100DD800A0F89430FF2380F896300446983000F04D
:100DE800DDFC002384F8A43010BD00BFFFFF7F00A6
:100DF80013B504461146CDE9002300F049FC0099DB
:100E080004F1140000F044FC009904F1280000F0FB
:100E18003FFC009904F13C0000F03AFC009904F111
:100E2800500000F035FC009904F1640000F030FC3B
:100E3800009904F1780000F02BFC019A4FF4FA7342
:100E48004FF4FA6104F1980000F093FC2046FFF794
:100E5800B7FF002384F8A5304FF47F43A4F8A630E9
:100E680002B010BD704700F01ABC143000F017BC77
:100E780008B5503000F01DFC292200F11403B3FB23
:100E8800F2F313F0FF0302D1031E18BF0123184623
:100E980008BD08B5643000F00CFC292200F11403E9
:100EA800B3FBF2F313F0FF0302D1031E18BF0123B3
:100EB800184608BD90F8903013B990F98C00704727
:100EC80090F98D00704790F8903013B990F98E0022
:100ED800704790F98F00704710B504460BF038FE44
:100EE80038B104F13C0000F0DEFB012838BF0120D6
:100EF800C0B210BD783000F0DEBB783000F0E3BB44
:100F080010B5044600F0A5FB04F1140000F0A1FBA5
:100F180004F1280000F09DFB04F13C0000F099FB6F
:100F280004F1500000F0A1FB04F1640000F09DFB07
:100F380004F17800BDE8104000F09DBB7F2807D081
:100F4800002807DA10F1800F06D04042C0B270477F
:100F580000207047012070477F20704710B1404241
:100F680040B270477F2070477F280FD010F1310FB3
:100F78000EDA10F1780F0DDB7830FE2340B25843BB
:100F880023304623B0FBF3F0C0B27047FF20704710
:100F9800FE20704700207047012805DD40F2FE73EF
:100FA800984203DC80B270470120704740F2FF701E
:100FB8007047A0F57870C0EBC02040F2AE7390FB8C
:100FC800F3F000F58060FFF7E7BFFFF7F2BF0328F3
:100FD80012DD0C2812DD0F2812DD122812DD16286A
:100FE80012DD192812DD1C2812DD1F2812DD212828
:100FF800CCBFFF20062070470020704701207047B3
:101008000220704708207047032070470720704768
:10101800042070470520704705289ABF014B185CCB
:10102800FF207047AC3D010805289ABF014B185CAA
:10103800FF207047B23D01087F2803D0002803DA5B
:10104800C0B2704700207047FF2070477F2811D03A
:1010580010F1320F10DA884210DD401A6423C1F112
:10106800FF21584301F57F01CE31313090FBF1F07B
:10107800C0B27047FF207047642070470020704757
:10108800014B4140585C7047B83D01085AB110B453
:10109800054C0A4411F8013B58408A42205CF9D1BA
:1010A8005DF8044B70477047B83D0108392808D8E7
:1010B80022280ED9094B2338C0B2C34003F00100DF
:1010C80070475F2807D0613819288CBF002001209D
:1010D8007047002070470120704700BF01EC7F0077
:1010E800F8B50246451E461D00245F2715F8010F76
:1010F800FF2804BF0134E4B2FFF7D8FF00B92F700E
:10110800AE42F3D1062C04D119B10B6813608B8859
:10111800938000239371F8BD2DE9F843DFF83490EC
:10112800471E441D012500264FF0280817F8011F07
:10113800084812F0B0FD034610B1A0EB0903DBB27A
:10114800A3FB05329E19A742A5FB0853EED13046F2
:10115800BDE8F883B83E010810B54179A1F1300027
:10116800C3B2092B07D80523B0FBF3F303EB8303C2
:10117800C01AC0B210BD044C204612F08CFD0028E5
:10118800F1D0001BC0B2EEE7B83E0108F0B5094B3C
:10119800094F821D2826B1FBF3F4272C94BF3D5D2F
:1011A800302502F8015D824203FB1411B3FBF6F30C
:1011B800F1D1F0BD00801A06B83E010870B50446AA
:1011C800FFF730F882B20023551E98B2A84214FAED
:1011D80083F104DA265C302E03F10103F5D0121AEC
:1011E80001322046BDE8704012F024BD2DE9F04FD1
:1011F8000D4699B0164600211A461F46804612F041
:1012080033FD00212A2201A8009112F02DFDDFF8FC
:10121800CC90DFF8CCA0DFF8CCB005EB4606AE42A8
:1012280011D16846FEF7FEFF30B100F160030DEB07
:101238000300002300F8613C6946404612F074FD43
:1012480019B0BDE8F08F35F9020B47F6FF739842E5
:10125800E7D0002812DC59460CA812F065FD684654
:10126800FEF7E0FF04460CA8FEF7DCFF20448742A7
:10127800D5D30CA9684612F0FFFCD0E7B0F57A7F09
:101288000BDA0CA980B210F0E8FF0CA8FFF796FF64
:1012980051460CA812F0F0FCE1E764230CA93230A7
:1012A800B0FBF3F080B210F0D8FF0CA8FFF786FF70
:1012B8000CA8FEF7B7FF00F15F036B4400F1600173
:1012C8000DEB010013F8302C00F8302C2E2203F817
:1012D800302C002300F82F3C4946DAE7A63D0108E8
:1012E800A13D01089C3D0108F0B589B06D46002478
:1012F8002F468E1CE1B28A4204D83946FFF776FFA2
:1013080009B0F0BD36F8241025F8021B0134F1E7C6
:1013180042F210736421B0FBF3F203FB1200B0FB3E
:10132800F1F301FB130000EB023000EB831080B2F5
:101338007047020B00F03F0342F2107101FB0233C9
:10134800C0F38510642202FB003070472DE9F0419C
:1013580042F2107388B0B1FBF3F603FB16141F4971
:10136800DFF87C80054612F0DFFC6946F0B210F029
:1013780051FF6846FFF722FF6946284612F07CFCB9
:101388004146284612F078FC64276946B4FBF7F614
:10139800F0B210F03FFF6846FFF710FF6946284695
:1013A80012F06AFC07FB16444146284612F064FC1A
:1013B8006946E0B210F02EFF9DF801308DF800303C
:1013C8009DF802308DF801306946002328468DF8D3
:1013D800023012F051FC08B0BDE8F081015001085C
:1013E800AA3D010870B50E4600210546144612F0C4
:1013F8003BFC00239AB2944200D870BDF25C002AEC
:10140800FBD0EA540133F5E770B50E4614460021C7
:101418000132054612F028FC00239AB2944200D803
:1014280070BDF25C002AFBD0EA540133F5E730B511
:101438000024A3B2934201D3012005E0055D0B5DB2
:101448001DB9B3FA83F0400930BD1BB19D4204F1C8
:101458000104EED00020F7E77D23438043F23903EF
:1014680009B2C360002301808180C3800372704782
:1014780002680449044B01FB023323F00043036074
:10148800180C7047FD430300C39E2600F0B50025E5
:1014980097B001608580044656222946684612F0B6
:1014A800E3FB0126E27DAA4209D80023802104F14A
:1014B800B800A37517B0BDE8F04012F0D5BB2046C0
:1014C800FFF7D6FFE7797B1B002190FBF3F202FBC5
:1014D8001300C0B2EC460A46CBB29F4223D8002381
:1014E8000022277B1146D0B2874227D80029D9D1BC
:1014F800A279033A012A04EB050105D925B191F92E
:10150800172012BB012BCDD90B76A26852F82310F5
:10151800583305F10E026B44013544F8221003F8E4
:10152800586CEDB2BEE71CF801EBBEF1000F03D119
:101538008242D5D00132D2B20131CDE72069805C38
:101548000132984208BF0121CDE7501E8342DBDB00
:1015580001329342D8DCA5E72DE9F047154696B04D
:10156800013D0160027104464371EDB2562200212B
:10157800684612F079FB0027022D84BF4FF001095D
:1015880000253E464FF0010A94F807809CBF4FF0B3
:101598000309B8FBF9F8E27DB24209D8002380219B
:1015A80004F1B800A37516B0BDE8F04712F05CBBB3
:1015B8002046FFF75DFFA8EB0603002190FBF3F23E
:1015C80002FB1300C0B2EC460A46CBB2434506D232
:1015D8001CF801EBBEF1000F2AD1824226D1434507
:1015E80028BF434603FB0951002094F80CE001F0A2
:1015F800FF018446C2B296451CD8BCF1000FCAD17F
:1016080016B1FFB9012BC6D9A2191F461176A268D7
:1016180052F8211006F10E02013644F8221003F1A7
:1016280058026A44F6B202F858ACB4E70132D2B2B2
:101638000131CAE72269125C01308A4208BF4FF0C3
:10164800010CD7E77A1E9342DEDB7A1C9342DBDC7F
:10165800A1E7D0E901236421D31AC36082604B4318
:10166800418AB3FBF1F303747047D0E90123D31A1D
:10167800C0E90223704743682BB1C26864214A431A
:10168800B2FBF3F2D3B203740023C3604360704724
:101698000023C0E902334182436003747047436802
:1016A800013343607047007C7047436819444160C8
:1016B8007047C068704711B1C3680133C36043689D
:1016C800013343607047007C7047002303808370B8
:1016D8000372704703781BB10022027018467047E6
:1016E800437813B100224270F8E7837813B10022DF
:1016F8008270F3E7037A002BF0D000220272EDE744
:101708000170704701707047817070478170426046
:1017180070474068704700234360038170470A237D
:1017280010B50446838002F08DF82368E0809B683A
:1017380020469847208110BD038970B504469BB1A7
:10174800858845B1013DADB285806DB903681B68D8
:10175800BDE87040184702F075F8E388C01A23897D
:1017680080B2834201D2258170BD236820465B6820
:10177800EEE707EE902A0A44F8EE676A07EE902A29
:10178800F8EE677A436086EEA77A07EE903AF8EEAD
:10179800E77A80ED007AC0ED027A7047D0ED017AE1
:1017A800F8EEE77AC0ED027A7047000080EAE0734D
:1017B800022910B5A3EBE07304467DD162B9002875
:1017C800ACBF7F223F229342A8BF1346002C184685
:1017D80001DA43F0400010BD012A1FD1632B05DC5C
:1017E8005800002CF7DA40F48070F4E740F2F54234
:1017F800934211DC07EE903A9FED6A0AF8EEE77A19
:1018080027EE800A11F00AFAFCEEC07A17EE900A69
:10181800400040F00100E4E7FF20E2E7022A40F040
:10182800BF80632B05DC9800002CD4DA40F40070EC
:10183800D1E7B3F57A7F11DA07EE903A9FED590AAE
:10184800F8EEE77A27EE800A11F0E8F9FCEEC07AA4
:1018580017EE900A800040F00100E5E742F20F72AF
:10186800934211D807EE903A9FED4F0AF8EEE77AC7
:1018780027EE800A11F0D2F9FCEEC07A17EE900A32
:10188800800040F00200CFE7484A934211D807EEA3
:10189800903A9FED470AF8EEE77A27EE800A11F0B2
:1018A800BDF9FCEEC07A17EE900A830043F00300FE
:1018B800BAE740F2FF10B7E7032971D1012A20D116
:1018C800B3F57A7F05DA5800002C84DA40F400601A
:1018D80081E7B3F5205F11DA07EE903A9FED310A00
:1018E800F8EEE77A27EE800A11F098F9FCEEC07A54
:1018F80017EE900A430043F00100E5E740F2FF705D
:10190800E2E7022A4CD1B3F57A7F06DA9800002C78
:10191800BFF661AF40F480505DE742F20F72934228
:1019280011DC07EE903A9FED1F0AF8EEE77A27EEF2
:10193800800A11F073F9FCEEC07A17EE900A830062
:1019480043F00100E3E71B4A934211D807EE903AAF
:101958009FED150AF8EEE77A27EE800A11F05EF996
:10196800FCEEC07A17EE900A830043F00200CEE73F
:10197800B3F57A2F11D207EE903A9FED0D0AF8EEE3
:10198800E77A27EE800A11F049F9FCEEC07A17EEE3
:10199800900A830043F00300B9E740F6FF70B6E70A
:1019A800002018E7CDCCCC3D0AD7233C17F0010026
:1019B8006F12833A9F86010000230360704700007E
:1019C80038B5084B09291B7828BF09218B420446E2
:1019D8000D4602D10023036038BD01F027FF2571B1
:1019E8002060F9E7CC030020036810B504460BB962
:1019F800002010BD01F01AFF2368C01A40F2EE2340
:101A08009842F5D90023054A2360127823799A422F
:101A1800EED0034A0120D377EBE700BFCC030020C8
:101A280028040020FF23437100230171837103817F
:101A38008372704738B5037904460D465BB1417926
:101A4800A94208D041B101290AD00023A3716571C8
:101A580055B1012D0FD038BD03689B689847F4E74E
:101A680003680021DB68F9E723689B6801212046A9
:101A78009847A071EFE723682946DB68F7E72DE967
:101A8800F04F2DED068B85B0837B077C0093C37BDD
:101A9800009A857CC67C90F815C090F820E090F8F4
:101AA8002280BF000C4647EA931703F03F01437CAE
:101AB800490141EAD20103F0010247EA822705F011
:101AC8000F02D20142EA530206F07F031B0143EAE8
:101AD8001513057D01936D0045EAD6150CF0030634
:101AE80045EA4623867D029206F01F05AD0108EE01
:101AF800103A45EA9C03C57D90F819C00391ED00A2
:101B080008EE903A45EA5613057E0CF0070609EEF2
:101B1800103A45EA0623857E05F03F06760109EE70
:101B2800903A46EADC03C67E90F81CC0B60046EA46
:101B380095160CF0010546EA8526457F05F00F0B42
:101B48004FEACB1B4BEA5C0B90F81EC00CF07F0AE7
:101B58004FEA0A1A4AEA151AC57F6D0045EADC15EC
:101B68000EF0030C45EA4C2590F821C00AEE103A15
:101B78004FEAC808009B48EA5C180CF01F0990F867
:101B88000DC003F007004CEA00204FEA891949EA22
:101B98009E09FFF70EFA039920800846FFF709FA15
:101BA80060803846FFF705FA029AA0801046FFF7D2
:101BB80000FA019BE0801846FFF7FBF9208118EE38
:101BC800100AFFF7F6F9608118EE900AFFF7F1F9AD
:101BD800A08119EE100AFFF7ECF9E08119EE900ADE
:101BE800FFF7E7F920821AEE100AFFF7E2F96082A0
:101BF8003046FFF7DEF9A0825846FFF7DAF9E082AF
:101C08005046FFF7D6F920832846FFF7D2F96083BC
:101C18004846FFF7CEF9A0834046FFF7CAF94FF4CC
:101C28008063E0832384638405B0BDEC068BBDE844
:101C3800F08F2DE9F04104460F4601F003FE4FF006
:101C480001080546236820461B689847064650B990
:101C5800A37A012B1FD12389ED1A40F6C4139D42A4
:101C6800C8BFA07217E0236820465B689847A37A2C
:101C7800A3B90F2814D1A4F80A80E37AE218013333
:101C8800DBB2182B1073E3720AD939462046FFF7E6
:101C9800F6FE0023A3723046BDE8F081012BECD09C
:101CA8002581CFE7827922B14379012B01D8FFF74B
:101CB800C0BF0020704770477047704700207047CA
:101CC8007047002070470020704770470020704719
:101CD80000207047054BDA6C0243DA64DB6C82B093
:101CE80003400193019B02B0704700BF00100240FF
:101CF800054B9A6D02439A659B6D82B00340019330
:101D0800019B02B0704700BF00100240054B1A6EDD
:101D180002431A661B6E82B003400193019B02B016
:101D2800704700BF0010024050E8003F43F0200316
:101D380040E80032002AF7D1704750E8003F43F0EE
:101D4800800340E80032002AF7D1704750E8003F8E
:101D580023F0200340E80032002AF7D1704750E80A
:101D6800003F23F0400340E80032002AF7D17047D3
:101D780050E8003F23F0800340E80032002AF7D102
:101D8800704770470288044B5140C9B233F811308C
:101D980083EA122303807047006D0108A2B110B4D2
:101DA800B0F800C0094C0A4411F8013B83EA0C035F
:101DB800DBB2914234F8133083EA1C2CA0F800C03F
:101DC800F2D15DF8044B7047704700BF006D010801
:101DD80037B54FF6FF730446ADF806304518AC42E8
:101DE80003D1BDF8060003B030BD14F8011B0DF196
:101DF8000600FFF7C7FFF2E7044B1888044B1B885F
:101E080080B29BB2C01A18BF012070477C3E0020E8
:101E18007A3E0020044A00231380044A1380044AAF
:101E28001380044A138070477A3E00207C3E0020CD
:101E38007E4000208040002001207047704700004D
:101E4800044B1888044B1B8880B29BB2C01A18BF79
:101E5800012070478448002082480020044A00235B
:101E68001380044A1380044A1380044A138070477D
:101E78008248002084480020864A0020884A0020A2
:101E880000207047704700000649074A0B881288EF
:101E98000133C3F3080392B29A421EBF034AD054D7
:101EA8000B80704774340020723400207232002096
:101EB8000023A0F87032A0F86E3270470023A0F813
:101EC8005C32A0F85A3270473A4B5A6A037A92B297
:101ED80063B18389D31A9BB2B3F5FA7F84BF002319
:101EE8000372837A4F2B84BF00230372037A8281A3
:101EF800082B0FD8DFE803F0050E0E0E0E0E0F1795
:101F08002200EE2901D0C82904D10123837241752A
:101F1800062303727047837A5A1C034482725975E8
:101F280041720723F5E7827A531C0244DBB28372BD
:101F38005175427A9A42EDD20823EAE7837A5A1C0D
:101F4800034482725975C37D162B04D1012380F88E
:101F580065300923DDE74369174A03F0FF239342FD
:101F680003D1012380F86730F3E7144A93421CD168
:101F7800837E102B19D1C37E022B08D0052B0DD0E0
:101F8800012BE6D1027EEE2A08BF80F86A30037E74
:101F9800EE2BDED1012380F86B30DAE7012380F8DD
:101FA8006830037F80F86930D3E7012380F8663012
:101FB800CFE700BF0004004000C8002800C8003276
:101FC800044B1888044B1B8880B29BB2C01A18BFF8
:101FD8000120704774340020723400200278024BCC
:101FE80051405B5C0370704780590108FF23037000
:101FF800704700BF7047B0F86E32B0F870229B1A75
:1020080098B21B0444BF00F5006080B2003818BFC6
:1020180001207047A0F11400EDE7B0F87032B0F875
:102028006E229A421FBFC218B0F8721292F8742238
:10203800013316BF0B400022A0F8703210467047DB
:10204800A0F11400E9E770B50B7803704B78437082
:102058000B78FD2B05460C4638D18B788370CB78EE
:10206800C3700B7903714B7943718B7983718B68DA
:10207800C3718B68C3F30F2303728B7A43720A26EA
:10208800627804F10C01A81911F056FE6378B4F8CF
:102098000C213344981CEA545A1CB4F80C1192B21F
:1020A800090AA954A278D20780B20ED504F588721D
:1020B800054404F58E7452F8041B45F8041BA2422B
:1020C800F9D112782A700F3398B270BD00238B7043
:1020D8000B7983704B79C3708B7903718B6843716B
:1020E8000626CDE738B54A78352A0D46044601F16B
:1020F8000C010AD811F020FE68780021C0F13602E0
:102108002044BDE8384011F0AFBD403551F8043BDC
:1021180040F8043BA942F9D10B88038038BD38B593
:102128004A781B2A0C46054601F10C010AD811F021
:1021380003FE60780021C0F11C022844BDE8384045
:1021480011F092BD283451F8043B45F8043BA142F4
:10215800F9D138BD38B54A78082A0D46044601F148
:102168000C010AD811F0E8FD68780021C0F10902D5
:102178002044BDE8384011F077BDEB6803604B6838
:1021880043600B7A037238BD38B54A78072A0C4683
:10219800054601F10C010AD811F0CEFD6078002146
:1021A800C0F108022844BDE8384011F05DBDE3687D
:1021B80003604B68436038BD08B5242203480021FA
:1021C80011F052FD024B00221A7008BDAC0D002020
:1021D8007C0600202DE9F0411378037092F8018005
:1021E80080F80180FD2B04460F46154654D193789C
:1021F8008370D378C37013790371537943719379DA
:1022080083716B7A127A1B0403EB0223EA79134475
:1022180023F07F430A26A26863F31702A260A91974
:10222800424604F10C0011F087FD7A7B904507D2F5
:1022380008F10C00A2EB08020021204411F014FD63
:1022480063781E44AB195A78AB5D03EB0223A4F8FC
:102258000C31A378DB070ED5023615FA86F304F5A0
:10226800887203F10C0153F8040B42F8040B8B42FB
:10227800F9D11B781370BB7A84F82131FB7A84F882
:1022880022313B7B84F823317B7B84F824313B78F3
:1022980084F82031BDE8F0810023438093780371EE
:1022A800D37843711379837153790626B3E738B528
:1022B8004A78132A0C46054601F10C010AD811F098
:1022C8003BFD60780021C0F114022844BDE8384085
:1022D80011F0CABC203451F8043B45F8043BA14234
:1022E800F9D138BD084611460FF017BD0FF074BC80
:1022F80008B50FF063FC003818BF012008BD08B509
:102308000FF092FC003818BF012008BD0FF0E4BBA5
:102318002DE9F04F0C465188B1F58C7F054685B004
:102328004FF000000ED31070D91CC9B2012995BF17
:1023380001210023518053809CBF2370117000231A
:102348002B7049E016780E2E00F2938001A757F8FB
:1023580026F000BF3123000899230008C123000894
:10236800E92300087B2400087B2400087B2400085C
:102378007B2400087B2400087B2400087B240008B9
:102388007B2400087B2400087B240008FB2300082A
:10239800481C508063542178FD299BB206D10C3328
:1023A8000A21D380918002231370C8E708330621DD
:1023B800D38091800E23F7E7481C50806354D807D8
:1023C80042BFD1880D31D180012B4FF000018CBF65
:1023D8000B46032313702970002005B0BDE8F08F69
:1023E800481C5080635400218B4214BF0B460E23B7
:1023F800F0E7481C508063545388D1888B4232D30D
:1024080000235380137002232B7069802378FD2BDF
:1024180035D163792B72A3796B72637A227A1B04A4
:1024280003EB0223E27913446B60637803F10C0237
:102438006A80A278D10701D519336B8000266968B4
:10244800DFF8FC806E814FF4BC720C20B3180133A6
:102458005B0800FB03F758F80770B94218D25A1EF8
:10246800B242F3D816E092889A423FF668AF012349
:1024780066E7107050809080D0802870ACE7E378D1
:102488002B7223796B7263796B6063780833D4E7B6
:102498001E46E5D80C27774358F80730994227D1CC
:1024A80023782046FD2B10F801BF0CBF4FF00A0916
:1024B8004FF0060909EB0B03591E89B247440193F3
:1024C800FFF786FC97F804A0ADF80E0051460DF111
:1024D8000E00FFF757FC019BE218E35C527803EB10
:1024E8000223BDF80E209BB29A420AD0052300E0D1
:1024F80003232B701846023801288CBF00200120C6
:102508006BE7BB79DA0706D5FA79934582BF04EB06
:1025180009018A5CAA729B0709D50C2303FB068371
:1025280062781B7A9A4282BF4C44E35CEB720C23BC
:1025380003FB068385F80CA05B796B730220DAE74E
:10254800805A01080148436AFFF7EEBB0044004087
:102558000A4A0B4B12680B49A3FB02323220920C39
:1025680000FB02F2084B486802F5FA72A3FB02323C
:1025780092094B681B1A9A42FBD870474402002004
:1025880083DE1B43001000E0D34D621008B5FFF74F
:10259800DFFF4FF0904310229A6108BD4FF090433F
:1025A80010229A62FFF7D4BF30B587B0034601AC5A
:1025B80000F1100518685968224603C20833AB4277
:1025C8001446F7D10024094D8DF81440A96801A8D4
:1025D800FDF71EFE10B920B207B030BD01342E2C15
:1025E80005F10C05F2D14FF0FF30F5E708000020A7
:1025F80002780A4B90F801C08178D243D2B29A5C33
:1026080082EA0C0290F803C09A5C4A40995C02790D
:1026180081EA0C01595C4A40985C7047805901086E
:10262800028810B58488531C234044889C421EBFEE
:1026380012189171038010BD411A88B20B0444BF6F
:1026480000F5007080B2704770B5104C0025234625
:1026580026782EB166788E4202D1A67896420BD0A3
:1026680001350C2D04F10404F2D1002413F8245090
:102678001DB101340C2CF9D170BD012503F824508B
:1026880003EB8403D87059709A70F5E7810600202F
:102698002DE9F8430B460D795A7A9E7ADF7A204B5A
:1026A800097A1B5CDB07044600D50DB9FFF7CCFFA0
:1026B80000231C491A4898464FF0010E9C4201F825
:1026C800018B25D02DB90278920702D501F801ECCB
:1026D8001EE0154A4FF0000C92F80090B9F1000F77
:1026E8000FD092F8039099450BD1002EEED092F8B6
:1026F8000190B14505D1002FE8D092F80290B94574
:10270800E4D00CF1010CBCF10C0F02F10402E3D18E
:102718000133DBB2042B00F10100CFD1BDE8F8830F
:10272800B10600207D06002081060020F0B5054690
:10273800FD2305F80C3B85B004468DF8043090F86D
:10274800243103F10C020244012B42D800266370A5
:1027580066808DF805308B7A23718DF808308B7A76
:10276800ADF8066001338B7263798DF80930A3796F
:102778008DF80A30A368C3F317031A128DF80B30CB
:1027880009211B140DF105008DF80D308DF80C2072
:10279800FFF71EFB6778ADF802003A4629460DF1AF
:1027A8000200FFF7FBFA94F82311FFF7EBFA94F80D
:1027B8002421BDF80230A4F80C31974210D207F159
:1027C8000C00D21B3146204405B0BDE8F04011F0A2
:1027D8004BBA12F8010D0028B8D1013BDBB2B3E7C0
:1027E80005B0F0BD704707B503688DF807101B6981
:1027F80001220DF10701984703B05DF804FB13B5FA
:10280800044608460191FDF70DFD236801991B69EF
:1028180082B2204602B0BDE81040184708B5FFF75D
:10282800EEFF08BDB0F1904F08B5014607D1012071
:10283800FFF750FA114B99420BD1202014E0104BAE
:1028480098420BD003F58063984209D10420FFF722
:1028580041FA0C4B994210D1402005E00220E7E7ED
:10286800094B984204D10820BDE80840FFF732BA66
:10287800064B9842DED11020F6E708BD0014004848
:102888000004004800180048000C004800100048E8
:1028980008B5224B984201460BD14FF40060FFF770
:1028A80035FA1F4B99420DD1BDE808402020FFF7AB
:1028B8001FBAB0F1804F0ED01A4B98420FD10220A8
:1028C800FFF716FA184B99420FD14FF40050BDE8A4
:1028D8000840FFF71BBA0120FFF70AFAE1E7134B9C
:1028E800984208D10420FFF703FA114B99420CD102
:1028F8004FF48030EBE70F4B9842D2D11020FFF70E
:10290800F7F90D4B994206D008BD0C4B9942F8D106
:102918004FF40030DBE74FF48020D8E7002C01406B
:10292800001400400004004000340140000800404A
:1029380000400140001000400048014000440140B0
:102948002DE9F04387B00E460546144600211422AF
:1029580001A89DF838809DF83C901F4611F084F935
:1029680000960B2C07D8DFE804F007070A121414A6
:10297800141616161A1CFEE70323019301E002231E
:102988000493032F11D8DFE807F011132111012355
:10299800F6E70123F1E7012301930393F1E702230B
:1029A800EBE7022301930123F7E7FEE702230293F3
:1029B800B8F1100F0CD8DFE808F02D2D0C11131505
:1029C80017191B1D1F21232527292B000123EEE79B
:1029D800FEE701230593022301931EE00223F9E792
:1029E8000323F7E70423F5E70523F3E70623F1E7D5
:1029F8000723EFE70823EDE70923EBE70A23E9E7D5
:102A08000B23E7E70C23E5E70D23E3E70E23E1E7D4
:102A18000F23DFE7B8F1000FDDD1B9F1000F02D0C5
:102A28002846FFF7FFFE053C042C05D8DFE804F034
:102A3800030B04030B00AE62694628460DF014F937
:102A480007B0BDE8F083AE61F6E713B54FF0010CAF
:102A58000024CDE9004CFFF773FF02B010BD13B599
:102A68000124CDE900340323FFF76AFF02B010BD4B
:102A780007B50D48FFF76AF9036823F001030360FF
:102A8800436823F400434360036843F00103036091
:102A980008210023CDE90013044803230A22FFF785
:102AA8004FFF03B05DF804FB0044004000040048F9
:102AB80070B586B00023164604460D46ADF80630BC
:102AC800FFF7E6FE042E04D8DFE806F030340438B9
:102AD8004100FEE71F4B204A1B68B3FBF2F39BB291
:102AE8000022013B01A92046ADF80430CDE90225BA
:102AF800049205920DF032FB236823F080032360D3
:102B0800A36823F4A03323F00703A360636823F0CA
:102B1800007323F070036360636823F470036360D9
:102B2800A36823F08003A36006B070BD094B0B4A6D
:102B38001B68D2E7074B0A4A1B68CEE7054B074AD2
:102B48001B68B3FBF2F303EB83035B00C7E70123C6
:102B5800C6E700BF4402002080A8120140420F00CF
:102B68008096980010B50446FFF7A2FF236843F04B
:102B78000103236010BD00224FF0FF31FFF7F2BFC1
:102B8800034A034603CA1860596010689860704782
:102B98009075FF1F1B4B10B51B4C5B6823600EF034
:102BA800F3FF0BF01FFA4FF090400CF0FDFF1748B1
:102BB8000CF0FAFF16480CF0F7FF16480DF02AFB48
:102BC80015480DF027FB0DF095F94FF0E022002392
:102BD80013615361936172B64FF0FF319A0002F1AD
:102BE800604202F561420133082BC2F88010C2F836
:102BF8008011F3D162B6034B1B6883F308882368FE
:102C08009847FEE70000FF1F7806002000040048F0
:102C18000008004800380140004400400749084ABD
:102C2800881AEFF30883521A1A44013A013B984272
:102C380088BF0022AA2111F017B800BF0080002029
:102C48000004000010B5114C032320460622402141
:102C5800FFF7FBFE032302224FF400414FF09040A0
:102C6800FFF7F3FE03231A4620462021FFF7EDFE67
:102C78002046032305228021FFF7E7FE2046032391
:102C8800BDE8104005220121FFF7DFBE000400481F
:102C9800024B1869C0F34010704700BF0004004899
:102CA80008B5FFF7F5FF00B908BD00BFF9E7000058
:102CB800024B01229A6280229A6170470004004800
:102CC800024B80229A6201229A61704700040048F0
:102CD800104A53694FF4704123F4704391FAA1F1FB
:102CE80053610D4B5A6822F400425A601A6822F464
:102CF80000421A60DA6822F40042DA609A6842F404
:102D080000429A60054BD02283F828234FF4807242
:102D18005A607047000001400004014000E100E0F3
:102D2800044B4FF400425A611A6842F400421A6098
:102D3800704700BF000401400348002303224FF4FA
:102D48008071FFF782BE00BF00040048024B18697B
:102D5800C0F30020704700BF0004004808B50522F2
:102D6800002302214FF09040FFF76FFE0023052259
:102D780001214FF09040FFF768FE4FF09043022288
:102D88009A6201229A6208BD4FF090414B691A0479
:102D9800DB4302F4003203F0020313438B617047F4
:102DA8004FF090414B691A04DB4302F4803203F080
:102DB800010313438B61704708B5052200234FF4C4
:102DC80080714FF09040FFF740FE4FF090434FF472
:102DD80080729A6208BD4FF090431A284FF48072AF
:102DE800CCBF9A619A6270471D2826DC1A2806DD36
:102DF800022B18BF04231B200B7010707047172874
:102E080005DD022B0CBFFE2300231820F4E713284E
:102E180005DD022B0CBFFA23FC231420ECE7102855
:102E280005DD022B0CBFF823F9231120E4E7022B60
:102E38000CBF10200E20F723DEE70A231E20DBE755
:102E480010B40446084611461A46A3685DF8044BB8
:102E58005B7AFFF7C9BF00000C4BD3F8FC2022F0C7
:102E68008072C3F8FC20D3F8FC2042F08072C3F8CB
:102E7800FC20A3F55D431A6822F001021A601A6863
:102E880042F001021A6000225A60704700ED00E02B
:102E9800064A074B51681B6810B5064CB3FBF4F3A0
:102EA800584353685B1A8342FBD310BD001000E0FF
:102EB8004402002040420F007FB50123CDE90413EE
:102EC800002201A902A8CDE902230BF047FA002845
:102ED8000CBF0420052007B05DF804FB014608B5C7
:102EE80000200BF0A5F900280CBF0420052008BD20
:102EF80008B5FFF7E1FF031F5842584108BD08B560
:102F0800FFF7ECFF031F5842584108BD2DE9F3476E
:102F18002A4B2B4D012814462A482B4A0E4617BF28
:102F2800AA463D213C211D46019106BF9A4680468E
:102F380090460BF037F901992846FFF7D9FF30B9C9
:102F480000240BF041F9204602B0BDE8F087002EBE
:102F580008BF4FF4FC64073424F0070405F1100798
:102F6800B1463444AAEB050AA1450BD14FF0113202
:102F78004FF0FF332846FFF7C2FF003818BF012083
:102F88008400DEE76EB90AEB0703D3E90023B3F147
:102F9800FF3F08BFB2F1FF3F06D1083709F1080922
:102FA800E2E7D9E90023F2E7B84505D93846FFF743
:102FB800A6FF0028F1D1C3E70324C2E700E0010817
:102FC80000E80108FFEF0108FFE7010810B50BF062
:102FD800E9F809483C21FFF78BFF58B107483D2124
:102FE800FFF786FF003818BF012084000BF0ECF8CB
:102FF800204610BD0446F9E700E0010800E8010892
:1030080030B5084D002340F2EF749AB2914201D8CE
:10301800042030BDA34203D05A5DC2540133F4E703
:103028000320F6E710E0010813B50A46044672B615
:10303800019101460020FFF769FF62B60428019A52
:1030480005D172B601202146FFF760FF62B602B0D3
:1030580010BD000038B5124B1C68D3F80058B4F105
:10306800113F09D1B5F1113F17D0002211460120B7
:10307800BDE83840FFF74ABFB5F1113F03D1002240
:1030880011461046F4E7FFF7A1FF042804D12C40AD
:1030980001340CBF0220012038BD0420FCE700BF2A
:1030A80000E00108034B18739A68D207FCD5187B17
:1030B800704700BF0030014038B5441E8D18A94242
:1030C80000D138BD14F8010FFFF7ECFF01F8010B30
:1030D800F5E7084611461A46FFF7EEBF38B5064D24
:1030E80004460144A14200D138BD2878FFF7DAFF31
:1030F80004F8010BF6E700BF380200200846114625
:10310800FFF7ECBF10B5014404468C4200D110BD56
:1031180014F8010BFFF7C6FFF7E708461146FFF75B
:10312800F1BF000010B58AB028220021684610F0CF
:103138009BFD4FF48050FEF7E9FD10210323062282
:103148004FF09040FFF781FC4FF0904010238361CF
:103158000A2206232021FFF782FC06230A22802167
:103168004FF09040FFF77BFC0623032240214FF0ED
:103178009040FFF774FC1822154C06924FF48272A7
:10318800002301924FF40072CDE90333CDE90733F0
:103198000093059207234FF4E0626946204609939D
:1031A80002920CF0A1FF636823F010036360636868
:1031B80023F008036360236843F040032360A36897
:1031C8009B07FCD5237B034BFF221A700AB010BD66
:1031D80000300140380200201C4B10B4DC69A00606
:1031E80011D51A6891060ED519481A495A6A0388E2
:1031F80009880133C3F30A0389B299421FBF1649EC
:10320800D2B2CA54038011481F232206036215D57F
:1032180003681B0612D5114B114A1988138889B205
:103228009BB299420DD013880133C3F3080313806E
:1032380013880C4A9BB2D35CDBB283625DF8044B03
:1032480070475DF8044BFEF793BD00BF003801409E
:103258007C3E00207A3E00207A3600208040002004
:103268007E4000207E3E00200A490B4A08B50B88A4
:1032780012880133C3F3080392B29A4207D0074A6F
:10328800D05407480B80FEF758FD012008BD0020E8
:10329800FCE700BF804000207E4000207E3E0020EA
:1032A8000038014038B504464518AC4200D138BD55
:1032B80014F8010BFFF7D8FFF7E708461146FFF7A8
:1032C800F1BF0000054B064A1B8810880133C3F381
:1032D800080380B2181A18BF0120704780400020E8
:1032E8007E40002008B5FFF7EDFFB0FA80F04009F6
:1032F80008BD0000054B064A1B8812889B1A98B225
:103308001B0444BF00F5006080B270477C3E00207B
:103318007A3E0020FFF7EEBF0848094A0188138863
:1033280089B29BB29942F9D013880133C3F30A03D7
:1033380013801388034A9BB2D05C70477C3E002000
:103348007A3E00207A360020FFF7E6BF70B588B0D5
:103358000C460646154600212022684610F084FCDB
:10336800231E18BF01231B03CDE9023569460C2330
:1033780003480196049405930CF08EFF08B070BDC5
:103388000038014010B5064C236823F00103236080
:10339800FFF7DCFF236843F00103236010BD00BF83
:1033A80000380140002208461146FFF7EBBF000035
:1033B80010B53D4C236823F0010323604FF480408F
:1033C800FEF7A4FC4FF4007108230A224FF0904046
:1033D800FFF745FB082303224FF480614FF090402C
:1033E800FFF73DFB002211464FF4E130FFF7AEFF37
:1033F80063682E4A23F490436360A36823F02A038A
:10340800A360236823F00053236002F6080353E8FF
:10341800003F23F0604302F6080040E8003100292D
:10342800F3D102F6080353E8003F23F0606302F685
:10343800080040E800310029F3D11D4BB02283F881
:10344800252320225A601848FEF792FCFEF787FCD5
:1034580040230362174B1980174B1980FEF776FC3F
:10346800164B1980164B1980436823F40063436098
:10347800836823F008038360436823F48043436030
:10348800836823F022038360836843F48053836056
:10349800036843F001030360C3699A02FCD5C3695A
:1034A8005B02F9D510BD00BF003801400030014073
:1034B80000E100E07E400020804000207A3E0020AD
:1034C8007C3E002008B5FFF773FF0348436ABDE858
:1034D8000840FEF729BC00BF00380140FFF7F2BFE3
:1034E8001C4B10B4DC69A00611D51A6891060ED5DC
:1034F80019481A495A6A038809880133C3F30A0329
:1035080089B299421FBF1649D2B2CA5403801148E2
:103518001F232206036215D503681B0612D5114B1B
:10352800114A1988138889B29BB299420DD0138821
:103538000133C3F30803138013880C4A9BB2D35C8E
:10354800DBB283625DF8044B70475DF8044BFEF70D
:103558000FBC00BF00800040844800208248002043
:1035680082400020884A0020864A002086480020A1
:103578000A490B4A08B50B8812880133C3F30803BC
:1035880092B29A4207D0074AD05407480B80FEF7F8
:10359800D4FB012008BD0020FCE700BF884A0020BA
:1035A800864A0020864800200080004038B504463E
:1035B8004518AC4200D138BD14F8010BFFF7D8FF0D
:1035C800F7E708461146FFF7F1BF0000054B064A2A
:1035D8001B8810880133C3F3080380B2181A18BF78
:1035E80001207047884A0020864A002008B5FFF766
:1035F800EDFFB0FA80F0400908BD0000054B064A0F
:103608001B8812889B1A98B21B0444BF00F50060FF
:1036180080B270478448002082480020FFF7EEBF40
:103628000848094A0188138889B29BB29942F9D09F
:1036380013880133C3F30A0313801388034A9BB228
:10364800D05C7047844800208248002082400020D7
:10365800FFF7E6BF70B588B00C4606461546002150
:103668001C2201A810F000FB231E18BF01231B0316
:10367800CDE9033501A90C23034802960594069366
:103688000CF08CFB08B070BD0080004010B5064CF3
:10369800236823F001032360FFF7DCFF236843F06E
:1036A8000103236010BD00BF0080004000220846CF
:1036B8001146FFF7EBBF000013B53B4C236823F01E
:1036C80001032360394BDA6D42F00102DA65DB6DE4
:1036D80003F001030193019B0A220D2304214FF0FB
:1036E8009040FFF7BCF90D23032208214FF09040CA
:1036F800FFF7B5F9002211464FF4E130FFF7AAFFB2
:10370800236823F00053236004F1080353E8003FC3
:1037180023F0604304F1080141E80032002AF3D1A4
:1037280004F1080353E8003F23F0606304F1080242
:1037380042E800310029F3D11D4BF02283F85B23C6
:103748004FF000629A601848FEF712FBFEF707FB7D
:1037580040232362174B1980174B1980FEF7F6FA9E
:10376800164B1980164B1980636823F40063636055
:10377800A36823F00803A360636823F480436360AD
:10378800A36823F02203A360A36843F48053A360D3
:10379800236843F001032360C3699A02FCD5C36917
:1037A8005B02F9D502B010BD008000400010024055
:1037B80000E100E0864A0020884A00208248002074
:1037C8008448002008B5FFF777FF0348436ABDE83F
:1037D8000840FEF7A9BA00BF00800040FFF7F2BF1B
:1037E800024B1A68024B1A60704700BF984A0020C3
:1037F800980B0020054A064B1968136899421DBFAB
:103808000133012013600020704700BF980B00208F
:10381800984A0020034A0449136809680B44136056
:10382800704700BF984A002048020020014B1868E2
:10383800704700BF984A00200148FFF79CB900BFB5
:1038480000040040014B586A80B2704700040040F1
:1038580008B5FFF7F1FFBDE80840FFF7C1BF00005A
:1038680038B51A4C90220021201D10F0FDF90623CE
:103878002380162363800F231549A38005222C2358
:10388800A01DFDF731FD134A134B1149C4E90D235F
:1038980000252C23052204F13E00A587FDF724FD11
:1038A8000223E3660D4984F87250012304F17C0079
:1038B800A4F87030C4E91D5510F036FA7F2384F857
:1038C8009130052384F8923038BD00BFE40500200C
:1038D8006052010802000F0003000700483F01087A
:1038E80070B5094E05460C46415C304610F0D3F9D8
:1038F800034628B1831B0133DBB2282B28BF0023E2
:10390800F35C2B5570BD00BF5459010870B50C46C7
:103918001146064610F008FA44B100250521304644
:103928000135FFF7DDFFEBB29C42F7D870BD000010
:1039380073B5054605F11106214C224A01463601A8
:103948006846FFF7E3FFB01C69462044264410F0A0
:10395800EBF90223737204EB05130022A3F81A2172
:10396800142303FB05400421012380F850104FF471
:10397800807540F20111A0F84A30C364A0F85230B3
:1039880080F85530A0F85650A0F8581040F203209F
:1039980084F83420E384A562A08584F82E3084F866
:1039A800303084F83320C4F83A20C4F83E20C4F8F4
:1039B8004220A4F84610A4F8481002B070BD00BF19
:1039C80028040020083F0108F7B50546AF4CB04A67
:1039D80005F11106014637016846FFF797FFB81C45
:1039E800274469462044FDF77BFB7B7AA94A052BCF
:1039F80088BF022304EB061088BF7B721188437AC4
:103A080041FA03F3DF070FD40223437261B1480779
:103A1800C1F3800308D441FA03F7FF07D8B240F195
:103A2800D08104EB0613587204EB05112B0191F8B1
:103A38001A01052802D9002081F81A01E7185088D0
:103A480097F81A1140FA01F1C90711D4012187F832
:103A58001A1168B18707C0F3400109D440FA01FC84
:103A68001CF0010FCFB200F0B181E11881F81A7192
:103A7800E11891F81B01032802D9002081F81B01E5
:103A880004EB0616717A012903D9042901D0002113
:103A98009180E618908896F81B1140FA01F111F010
:103AA80001010ED186F81B1158B110F0010108D19F
:103AB80040FA01F7FF07CEB240F18D81234483F825
:103AC8001B61142303FB054191F84A00042802D91D
:103AD800012081F84A0003FB054393F84B100429A1
:103AE80002D9002183F84B10142303FB0543918E60
:103AF80093F84B0041FA00F0C00712D4012083F874
:103B08004B0071B18807C1F340030AD441FA03F6A8
:103B1800F707D8B240F16481142303FB054383F807
:103B28004B00142303FB054393F84C10032902D9D7
:103B3800012183F84C10142000FB0540D18E90F829
:103B48004C3041FA03F313F0010310D180F84C30E4
:103B580069B111F001030AD141FA03F6F607D8B2A8
:103B680040F14381142303FB054383F84C001423DD
:103B780003FB054393F84E10012902D9002183F86D
:103B88004E10142000FB0540118F90F84E3041FA7A
:103B980003F313F0010310D180F84E3069B111F02E
:103BA80001030AD141FA03F6F707D8B240F122819E
:103BB800142303FB054383F84E00142303FB05433A
:103BC80093F84F10022902D9002183F84F101420CE
:103BD80000FB0540518F90F84F3041FA03F313F082
:103BE800010310D180F84F3069B111F001030AD1F7
:103BF80041FA03F6F607D8B240F10181142303FB1A
:103C0800054383F84F00142303FB054191F84D0049
:103C1800022802D9002081F84D0003FB054393F8E0
:103C28005010052902D9042183F85010142303FBEE
:103C3800054191F85200012802D9012081F852006B
:103C480003FB054393F85510012902D9012183F894
:103C58005510142303FB054393F85310022902D986
:103C6800002183F85310142000FB0540918F90F831
:103C7800533041FA03F313F0010318D180F853309D
:103C8800A9B111F0010312D106E000BF28040020F9
:103C9800083F0108E405002041FA03F6F707D8B207
:103CA80040F1B280142303FB054383F85300142327
:103CB80003FB054191F856000C2802D9002081F831
:103CC800560003FB054393F84C10012906D193F8DD
:103CD8004F10022904BF002183F84F10142303FB5F
:103CE8000543012140F2011083F85710A3F858004A
:103CF80094F82630042B01D984F8261094F827303C
:103D0800042B02D9002384F82730B2F86C0094F809
:103D1800273040FA03F313F0010F814B0ED1012134
:103D280084F8271050B18607C0F3400106D440FA42
:103D380001F7FF07CEB26CD583F8276094F82810F6
:103D4800022902D9002184F8281094F829100229A0
:103D580002D9012184F82910B2F86E1094F82920AC
:103D680041FA02F212F001020CD184F8292049B17B
:103D780011F0010206D141FA02F6F607D0B24CD58D
:103D880083F8290094F82A200C2A02D9002284F802
:103D98002A2093F832200C2A02D9002283F83220F4
:103DA80093F82B20042A02D9002283F82B20002222
:103DB8005C49104611F9014F14F1780F31DA087097
:103DC80031E00133102B7FF426AE2DE601311029A6
:103DD8007FF444AE4CE6013110297FF469AE70E6F9
:103DE8000133102B7FF492AE9BE60133102B7FF446
:103DF800B3AEBCE60133102B7FF4D4AEDDE601335D
:103E0800102B7FF4F5AEFEE60133102B7FF444AFA0
:103E18004DE7013110298AD190E70132102AAAD141
:103E2800B0E7782CCBDC0132D2B20C2AC2D13E49A1
:103E38000022012011F8014F0132022CD2B288BFB2
:103E48000870042AF6D193F83420012A02D90022F6
:103E580083F83420354AB2F8701093F8342041FAC8
:103E680002F212F001020CD183F8342049B111F0AA
:103E7800010206D141FA02F4E407D0B211D583F861
:103E8800340093F82C20052A02D9032283F82C2029
:103E980093F82D20032A08D80AD1002283F8342069
:103EA80006E00132102AE5D1EBE7022283F82D2043
:103EB80093F82E20022A02D9012283F82E2093F8A3
:103EC8003020022A02D9012283F8302093F83320C7
:103ED8000C2A02D9002283F83320142101FB053172
:103EE800FF2203EB05154FF6FF7081F8512081F88A
:103EF800542083F82F2083F831204FF0FF32C5F883
:103F08001C21A5F820011A629A84A1F85A20A1F868
:103F18005C2083F83500DA861A8703B0F0BD00BF4D
:103F280028040020610400206D040020E40500201E
:103F380030B5052804D8DFE800F01E0423191E2335
:103F4800FEE720251F2400220F21104B987003380C
:103F5800012894BF002001201A7119771A74A3F858
:103F68004850A3F84A409873987630BD09256F24C5
:103F780000220721E9E71425322400220A21E4E778
:103F88003525132401221921DFE700BFCC030020C7
:103F98002DE9F04300F11105964F974C2D0105F1DD
:103FA8000209B94485B006464846FDF7B5F83D44D0
:103FB80080460390042103A8FDF70AFF6B7A63701B
:103FC80007EB0613E083C4F8088093F81A01C4F8D5
:103FD80014804FF0010884F85180A4F85280A4F8A6
:103FE8005480FFF7A5FF142303FB0673350193F8EC
:103FF8004A20824B13F92230237323766378052BEA
:1040080009D8DFE803F0030656585A5C00236373A7
:1040180001E084F80D807A4B617B1B88617603F0A0
:104028000102980748BF42F00202A2855A0748BF1A
:10403800A28D84F8281044BF42F00402A285180714
:1040480042BFA28D42F01002A285DA0642BFA28DBD
:1040580042F02002A285980642BFA38D43F00803D0
:10406800A385002384F82A3021B94846FDF774F85F
:1040780084F82A003D4495F81B2184F829206AB168
:10408800E18B02EB021303EB03230B44E383A368E6
:104098004FF0113101FB0233A360636194F828509B
:1040A800E38B6362052D0CD8DFE805F00C55571536
:1040B8004B4D0223ABE70423A9E70523A7E7032316
:1040C800A5E7FEE7A378032B03D8DFE803F0034A4C
:1040D8004803FEE7182507EE905ADFF828C184F850
:1040E8002050F8EEE77A1CE90F00B7EE087A67EE81
:1040F800877A8CE80F00FCEEE77A40F2E243CDEDD8
:10410800017AA4F84C309DF80430B4F84820A4F89B
:104118004E304FF47A73B3FBF2F3A4F84030142313
:1041280003FB06736D08052D93F8503038BF05253D
:1041380084F85050052B3DD8DFE803F01542363996
:104148003C3F0225C7E7A378022B08D0052B06D0F1
:10415800012B06D0FEE71925BDE70625BBE70C2590
:10416800B9E71225B7E74FF416536364002384F8C0
:10417800563084F85830142303FB067696F84C2002
:10418800032A03D096F84F30022B02D1012384F87A
:104198005630511E4B424B4194F8561084F8573014
:1041A80089B1012A0FD1FEE74FF41643DDE74FF43A
:1041B8006143DAE74FF4E133D7E74FF46133D4E7EB
:1041C8004FF49643D1E72378142000FB037393F848
:1041D8004C30022B07D1012384F8583021B194F8D0
:1041E80058301BB1FEE709B9012AF8D005B0BDE87F
:1041F800F08300BF28040020CC030020605201088F
:10420800E4050020FC03002002484FF4DE72FF2181
:104218000FF02ABD2804002002484FF4DE71FEF793
:1042280003BF00BF2804002002484FF4DE71FEF7E8
:10423800E7BE00BF2804002008B5FFF7F5FF034BD1
:104248001878BDE80840FFF7BFBB00BFCC030020CB
:1042580038B5FFF7D9FFFEF7FDFE04280CD0FFF7AD
:10426800D3FFFEF7F7FE042803D1FFF7DDFF04288C
:1042780006D0FFF7C9FF03E0FFF7D6FF0428EED109
:104288002F4930482F4C10220FF012FD38B12E491B
:10429800102220460FF00CFD08B1FFF7B5FFA38AE6
:1042A800B3F5215F28D008D30025E8B20135FFF720
:1042B8003FFB0A2DF9D10023E3774FF42153A38262
:1042C800012522691E491F4842F642039A424FF0CF
:1042D80010021CBF236101250FF0EAFC70B11849D8
:1042E80018481022FDF77EF8184919480822FDF7EA
:1042F80079F8FFF791FF03E00025E2E7002DF8D1F8
:10430800E37F104A092B84BF0023E377E17F142061
:10431800002300FB0144013394F84C0082F84C0060
:104328000A2B02F11402F6D10A4C2170FFF798FA11
:104338002078FFF749FB2078BDE83840FFF728BE12
:104348000F3F010828040020203F0108313F0108E1
:10435800DA050020CC0300200129F7B5054600D96D
:10436800FEE70B4E06EB01131C460F016278F15D68
:1043780003619B780EF048F9E3790193A3790093E0
:1043880022796379E17828460EF065F903B0F0BD2B
:10439800206F010838B5836804466BB1024652F8AD
:1043A800183BDD6900F11903A847217E2046022247
:1043B800BDE838400EF0B1B938BD000070B5816075
:1043C800897A86B0044601B101210EF0F6F820463C
:1043D8000EF086FA20460EF05EFA217BFF2903D004
:1043E800FA2220460EF063FAA3685B7A013B042B9D
:1043F80004D8DFE803F0043E3E414100FEE7E9222D
:10440800E12120460EF090FA012120460EF020FA14
:10441800962120460EF05DFA382120460EF06FFAFC
:1044280020460EF073FAA368204693F90810FFF7A8
:10443800B1FFA3689D7A15B319782046FFF78CFF62
:104448000022114620460EF0D2F80023009340F2D5
:10445800032220464FF6FF710EF02CF920464FF646
:10446800FF710EF04EF9204606B0BDE870400EF020
:10447800FFB9DB22D721C4E76F226B21C1E70F4BBD
:104488000F49DE8B0F4B63614CF25033009320468B
:1044980019230B220EF058FA0123CDE903335B23CD
:1044A800CDE90153102319462046009504220EF049
:1044B80089FA314620460EF0A9FAC1E7CC0300205C
:1044C800A0860100006F010810B504460EF0D0F96F
:1044D80020464FF6FF71BDE810400EF012B90000FB
:1044E80038B58168036891F90810DD69044600F160
:1044F800190300F11802A847A3689A7A42B11A78FA
:10450800012A00D9FEE7044B03EB0213236138BDEF
:10451800024B6361FBE700BF206F0108006F0108D1
:1045280010B50A4CA06858B1236923B9636913B957
:104538002046FFF7D5FFA3689B7A23B123699868C3
:10454800A0F57A7010BD63699869F9E774310020A5
:10455800836810B5044683B103691BB943690BB975
:10456800FFF7BEFFA3689B7A1BB12369B3F90C0060
:1045780010BD6369B3F91C00FAE71846F8E78368C9
:1045880010B5044643B103691BB943690BB9FFF77A
:10459800A7FF94F9190010BD1846FCE790F8D83029
:1045A8005BB190F8D930074A180102EB03139B68F6
:1045B8001978135853F821007047837D0E3350F84B
:1045C80023007047005201082DE9F3419DF824703B
:1045D8001646402F88464FF05B024FF00001044614
:1045E8001D4628BF40270FF03FFB904BDB8B2380F5
:1045F8003278A37862F30203A3707378DB0003F0C8
:10460800080343EA0811A37803F007031943A170CC
:104618007279E37862F30003E370B279637962F345
:104628008613637196F90200FCF788FCE37860F35F
:104638004703E370F279237962F300032371327A36
:1046480062F3460323713279DBB202F0010203F010
:104658007F0343EAC213237132796379C2F34502B7
:1046680023F03F0313436371A37967F34703A371EF
:104678002B78AA78E3716B7802F01F0203F0070326
:1046880043EAC20323726A88637AC2F3451223F0AD
:104698003F03134363722A79DBB202F0030203F08B
:1046A8003F0343EA82136372AB88C3F38703A372A1
:1046B8006A79E37AC2F3800223F001031343E372B9
:1046C800AA79DBB202F07F0203F0010343EA420356
:1046D800E372EA88237BC2F3C31223F00F03134368
:1046E80023732B7AAA7AE3736B7A02F01F0203F022
:1046F800070343EAC20323746A89637CC2F3451241
:1047080023F03F03134363742A7BDBB202F00302F6
:1047180003F03F0343EA82136374AB89C3F387034F
:10472800A3746A7BE37CC2F3800223F00103134382
:10473800E374AA7BDBB202F07F0203F0010343EAD1
:104748004203E374EA89237DC2F3C31223F00F0303
:10475800134323752B8ADB0863756B8ADB08A37503
:10476800AB8ADB08E375EB8ADB0823762B8BB3F582
:10477800C06F4ED2B3F5007F94BF00230123227B84
:1047880063F3051222736B8BB3F5C06F43D2B3F595
:10479800007F94BF00230123227B63F387122273D7
:1047A800AB8BB3F5C06F38D2B3F5007F94BF00234D
:1047B8000123227D63F305122275EB8BB3F5C06FDD
:1047C8002DD2B3F5007F94BF00230123227D63F32C
:1047D8008712089B22751F4404F11802BB4220D19E
:1047E8004FF6FF7321460DF106000D22ADF8063095
:1047F800FDF7D4FA2146BDF8063021F80D3F4C22CA
:10480800FDF7CCFABDF80630A4F8593002B0BDE87F
:10481800F0810223B3E70223BEE70223C9E702239C
:10482800D4E713F8011B02F8011FD7E7CC030020D7
:1048380013B59DF81040CDE9003413460A4600210F
:10484800FFF7C2FE02B010BD13B5144B0288DB8B14
:104858009A4204461DD1837803F0F003102B01D04F
:10486800202B18D1A379A52B15D84FF6FF730DF17E
:10487800060059222146ADF80630FDF78FFAB4F844
:104888005900BDF80630C01A18BF0120800002B0D8
:1048980010BD0120FBE70220F9E700BFCC03002090
:1048A80030B5374B027893F8261061F30302027093
:1048B80093F8271061F30712027093F828104278D2
:1048C80061F30302427093F8291061F307124270F2
:1048D80093F82A10827861F30302827093F83210F9
:1048E800827961F30302827193F82B10827861F365
:1048F8000712827093F83410C27961F30302C2710F
:1049080093F82C10C27861F30302C27093F82D104B
:1049180061F30712C27093F82E10027961F3030253
:104928000271427993F8301061F30302427193F8EF
:104938003310827961F30712827103F1390100F1B2
:104948000A0200F1160411F9015F02F8015FA242A0
:10495800F9D193F84610C27D61F30102C27593F84C
:10496800471061F38302C27593F8481061F305128A
:10497800C27593F8493063F38712C27530BD00BF22
:10498800280400200278314BC2F3030230B583F8C3
:1049980026200278C2F3031283F827204278C2F354
:1049A800030283F828204278C2F3031283F82920EF
:1049B8008278C2F3030283F82A208279C2F30302C1
:1049C80083F832208278C2F3031283F82B20C2794D
:1049D800C2F3030283F83420C278C2F3030283F8D7
:1049E8002C20C278C2F3031283F82D200279C2F377
:1049F800030283F82E204279C2F3030283F83020A1
:104A08008279C2F3031283F8332003F1390100F1EC
:104A18000A0200F1160412F9015F01F8015FA242CF
:104A2800F9D1C27DC2F3010283F84620C27DC2F3E8
:104A3800810283F84720C27DC2F3011283F848201F
:104A4800C27DC2F3811283F8492030BD28040020BA
:104A58001FB58DF80C300123019303AB0093134667
:104A68000A460221FFF7B0FD05B05DF804FB00001F
:104A7800F0B5224D012385F87230044685B0B0F8B0
:104A88000900FCF756FC6867B4F80B00FCF751FC0A
:104A98001422A86704F10D0105F17C00FCF7B4FCB1
:104AA80094F9213085F8913094F8223085F89230C5
:104AB80004F12300FFF766FF6E4604F1410304F199
:104AC800510718685968324603C20833BB42164674
:104AD800F7D10B482C2308226946FCF787FB94F88A
:104AE8005130A5F86C3094F85230A5F86E3094F82F
:104AF8005330A5F8703005B0F0BD00BFE4050020C4
:104B0800220600202DE9F04395B0DFF8909003923B
:104B180004AF4FF0400805460E464246002138468D
:104B28000FF0A2F81C4C99F80010222204EB011196
:104B38008DF810200DF11200062201F58971FCF79D
:104B480051FC99F8000004EB001107A891F81A210C
:104B580091F8194102F00F0204F00F0444EA02141C
:104B680091F81B2102F00F0244EA0224BDF8182034
:104B780022F47F6222F00F021443ADF81840FFF7C9
:104B88008FFECDE90078039B324602212846FFF7C5
:104B98001BFD15B0BDE8F08328040020CC030020DD
:104BA800034B04491A68044801FB02001860704767
:104BB800B80600200D6619005FF36E3C38B50A4A46
:104BC8000A4D13782C78A34203D101332B7028782F
:104BD80038BD1470FFF7E4FF6FF0004398423CBF04
:104BE80001342C70F3E700BFB5060020B60600209C
:104BF8000A4A126882600A4A00238380837183818B
:104C08000384136803615368064A43611368836128
:104C18005368C3614EF6602303607047984A0020CA
:104C2800373F0108403F010810B5114C0220FFF73B
:104C38007FF92046FFF748FC11212046FFF7AAFB21
:104C4800A36803B9FEE7002120460DF09FFC4FF44E
:104C58007A70FEF71DF9204601210DF0AEFCA3681D
:104C680020461978FFF778FB2046FFF72DFC10BD8A
:104C78007431002008B590F8203002468BB9FEF751
:104C880065F810B982F8210008BD92F82130013387
:104C98005BB2312B82F82130F6DD012382F8203017
:104CA800F2E7FEF753F818B1322382F82130EBE728
:104CB80092F82130013B5BB2002B82F82130D8BF3B
:104CC80082F82000E0E70000134B90F820201B68D2
:104CD800CAB182689B1AB3F57A6F01D9012343716F
:104CE8000379ABB10D4B427B1B781AB1022B1CBF69
:104CF800032202739A1E534253414373837953B17B
:104D08000323037370478360EAE701230371F8E71D
:104D18004379002BF9D17047984A00208D0700206D
:104D2800037B9A1E012A4FF0000202D890F8201047
:104D380011B90273184670471346FBE770B51B4C50
:104D48001B4E05465B22002120460EF08DFF2B6985
:104D580023606B696360174B174D1B7831789A1E77
:104D680053425341627A05EB011163F30002627208
:104D780001F58971062204F10A00FCF733FB337848
:104D880005EB0315237C95F81A2162F307132374A6
:104D980095F81B21637C592162F303032046637451
:104DA800FDF716F8A4F8590070BD00BFB93100200E
:104DB800CC0300208D070020280400200A4A38B5BB
:104DC800138801339BB2502B04460D4601D813803B
:104DD80038BD002305491380FDF711FD29462046FB
:104DE800FDF70DFDF4E700BF9C0B002068400108AB
:104DF8002DE9F84F154604460F467749FDF7FFFCA5
:104E080029462046FDF7FBFC744B0022012F1A802F
:104E18004FF0904610D10223B362B76146F2A81052
:104E2800FEF736F8B76246F2A810FEF731F82946C1
:104E38002046FFF7C3FFF0E7BB1E01220C2B00F250
:104E4800BE80DFE803F0374A5E1F07BCBCBC717147
:104E5800717171004FF090464FF001080227C6F8B3
:104E6800188046F2A810B762FEF712F8C6F8288034
:104E780046F2A810B761FEF70BF829462046FFF75F
:104E88009DFFEBE74FF090464FF001080227C6F868
:104E9800188046F2A810B761FDF7FAFFC6F8288017
:104EA80046F2A810B762FDF7F3FF29462046FFF740
:104EB80085FFEBE7B26202274FF09046B76146F2F2
:104EC800A810FDF7E5FFB76246F2A810FDF7E0FF6E
:104ED80029462046FFF772FFF0E70223B361012756
:104EE8004FF09046B76146F2A810FDF7D1FFB762C0
:104EF80046F2A810FDF7CCFF29462046FFF75EFFD3
:104F0800F0E7B26102274FF09046B76146F2A81069
:104F1800FDF7BEFFB76246F2A810FDF7B9FF2946B4
:104F28002046FFF74BFFF0E7A7F1090A5FFA8AFA74
:104F380000264FF0010956453EBF4FF0904302222C
:104F48009A614FF004084FF0904B46F2A810CBF846
:104F58001890FDF79DFF46F2A810CBF82890FDF7B2
:104F680097FF08F1FF3829462046FFF727FF18F07A
:104F7800FF08EAD10223CBF828304FF004084FF09D
:104F8800904B46F2A810CBF81890FDF781FF46F237
:104F9800A810CBF82890FDF77BFF08F1FF382946C9
:104FA8002046FFF70BFF18F0FF08EAD10136A7F1FA
:104FB8000803F6B2DBB2B34238BF0026BBE70223D0
:104FC800B261B3614CF25030FDF762FF29462046CA
:104FD800FFF7F4FEF6E700BF684001089C0B0020CD
:104FE80010B50446084694F901308B4201D1237864
:104FF80023B901232370FDF7EEFE607010BD000099
:105008001FB50C4670B9084801930DF10E020DF159
:105018000F010DF0DBFB019B9DF80E1002482246A4
:105028000DF085FA04B010BD7431002038B515466E
:105038001C46A8B9FDF73CFE2B460A4601460A481D
:105048000DF04EFA08484FF6FF710DF05AFB06486E
:10505800A1010DF06FFBBDE838407D20FDF718BFBA
:105068000148FFF731FA38BD7431002037B50C46D6
:1050780038B91A48836833B9812281F88C2081F8BD
:105088008E3003B030BD9D7ADDB101F18E020DF195
:1050980006010DF085FB94F98E30002B04DABDF87B
:1050A80006201344ADF80630BDF90630002B0FDB9F
:1050B8004FF6FF73ADF80630BDF8063084F88C3033
:1050C800DFE70DF106010DF0B2FC84F88E50EBE736
:1050D8007F33F1DA4FF68173ECE700BF74310020BB
:1050E80070B5114C0D4606465B23224621462846DC
:1050F800FFF786FFD6E90613206862689A4208BF60
:1051080088420ED120465921FCF762FEB4F8594076
:10511800231A5C425C4128460449FFF7A7FF601C3C
:1051280070BD0024F7E700BFBA2F0020CC30002064
:105138000A4608B501460148FFF75AFE0400002058
:10514800002303708370437003714371C370704709
:1051580003780022022B427104D0032B09D0012BC3
:1051680016D0FEE701230371437183784370C3703F
:10517800704783784278991AA3EB020218BF01217D
:1051880012F0060F14BF0122002201714271EDE7EF
:105198000271704702788170002A0CBF0222032234
:1051A8000270FFF7D5BF000008B5437802789A422D
:1051B80013D0042B8ABF042303700370027888BFBE
:1051C8004370064B064813F92210064B19731976DB
:1051D800836813B11972FFF7DDF808BD6052010842
:1051E80074310020CC03002010B50AB9437010BDFB
:1051F800541E0B2CFBD80332D2B231F8122040F2E5
:105208007E618A4207D95AB222EAE2729A42C8BF3C
:105218005AB24270EBE7B2F5C17F02D29A1E52B27F
:10522800F2E740F2D4418A4204D95AB2032A06DC92
:10523800DA1EF4E7B2F54B7F03D35A1EEFE70122DB
:10524800E4E70022E2E70000074B282202FB0030D7
:1052580083681A78542A05D15878A0F178035842FF
:10526800584170470020704774520108074B2822A4
:1052780002FB003083681A78522A05D15878A0F1C9
:10528800780358425841704700207047745201080B
:10529800074B282202FB003083681A78542A04D16D
:1052A8005878783818BF012070470120704700BF30
:1052B8007452010828230B4A434310B5D1580446B9
:1052C800FFF7D4FF48B92046FFF7BEFF064B1B780F
:1052D80028B103EB830301EB8301084610BD01EB02
:1052E8000311FAE774520108CC0300202B2838B5C3
:1052F80005461AD80E4B282202FB00334CB21B7904
:10530800022B0DD0FE2B10D1FFF7D4FF0378E4B2A7
:10531800A3420AD004702846BDE83840FFF7B8BF5A
:10532800FFF7C8FF90F90030F2E7002038BD00BF52
:10533800745201082B2838B504460D4619D80E4B6F
:10534800282202FB00331B79FF2B12D1FFF7B2FF93
:1053580006222946FCF76BF858B92046FFF7AAFF42
:1053680029460622FCF750F82046BDE83840FFF7EA
:105378008FBF002038BD00BF745201082DE9F043EB
:10538800074615462820394A41435018012B046A1C
:1053980087B025D15258364B9A4235D0A3F1CE0169
:1053A8008A4233D03349F23B9A4208BF0C46FF2366
:1053B8008DF800304FF0000801262046FAF732FF3A
:1053C8005FFA88F9484529D806F118036B44AE42BC
:1053D80003F8188C30D80020387007B0BDE8F08387
:1053E800022BE4D15258224B9A4211D0591C8A42BE
:1053F80010D0A3F1CE018A420ED0A3F1F2018A4265
:105408000AD01D49EC3BCFE71C4CD0E7194CCEE73E
:105418001B4CCCE71B4CCAE71B4CC8E714F80930F7
:105428002C2B06D106F118036B44013603F8188CAF
:10543800F6B208F10108C0E705F118030DEB030502
:10544800002315F8182C15F9175C0132D2B29918F7
:10545800C9B2A94207EB030003DB00230370012054
:10546800BBE7615C01700133DBB2F0E774520108FD
:1054780041050020493F01087D3F01089A3F010886
:105488001F400108FD3F0108D33F0108054B2822B2
:1054980002FB0030436A0BB1188870474FF6FF7063
:1054A800704700BF7452010838B50B4B282202FB25
:1054B8000030056A2846FAF7B5FE00221146D4B234
:1054C8004B1CA042DBB201D8184638BD2C5D013216
:1054D8002C2C08BF1946F2E7745201080F4B2822FA
:1054E80002FB003310B51B79FE2B014614D1FFF7E0
:1054F800CDFF04460846FFF7D7FF00221346D1B276
:10550800884201D8184610BD44FA02F1C90744BFC1
:105518000133DBB20132F2E7FF23F3E774520108EB
:105528002DE9F04F4FF0000A1D4E93B004460F4688
:10553800D146D6F808805FFA8AF54FF0000B0DE0E7
:1055480018F8030001920EF06BFBC3B2019A202BEE
:1055580008BF5F2302F8403C0BF1010B5FFA8BF3A5
:1055680040460193FAF75EFE019B03F14802984218
:105578006A44E5D802F8409C394602A8FAF748FE82
:1055880048B10AF1010ABAF12C0F06F12806D0D168
:105598000025284600E00120257013B0BDE8F08FF3
:1055A8007452010837B51E4D1346282202FB0155D7
:1055B80004462A79FE2A18D0FF2A24D0022A2BD1A1
:1055C8000846FFF777FE214690F900000CF089FEA7
:1055D8002D692B783BB1134920460EF04DFB294627
:1055E80020460EF049FB012018E00846019300917F
:1055F800FFF760FE019B02780099204603B0BDE8E2
:105608003040FFF7BBBE0846FFF754FE06220146AE
:105618002046FBF7F9FEE6E70020207003B030BD16
:10562800745201085D410108F8B5194B1646282245
:1056380002FB063300241A790470022A07460D4635
:1056480003D0FE2A13D02046F8BD93F918209142C2
:10565800F9DB93F91C309942F5DC4FF0000165F352
:1056680007013046FFF742FE01243870EBE70029B6
:10567800E9DB3046FFF718FFA842E4DD3046FFF7C4
:1056880005FF40FA05F313F00103E6D11C46DAE7FB
:10569800745201082DE9F84300230370124B174692
:1056A800282202FB073306461B79FF2B0C4603D042
:1056B80000252846BDE8F8830846FAF7B3FD062812
:1056C800F6D104F1FF3804F1050918F8010FFBF7CA
:1056D800EDFC05460028EBD0C845F6D121463846F2
:1056E800FFF728FE3070E4E774520108F8B5104E51
:1056F8004FF0280C0CFB0266002736790770FE2E47
:1057080004460B46154603D0FF2E0BD0022E0DD1B2
:1057180018460EF0EDF92A4601462046BDE8F84045
:10572800FFF782BFBDE8F840FFF7B4BF3846F8BDC1
:105738007452010810B504460846B2B9FBF70CFDCF
:10574800042812D8DFE800F003090B0D0F00084900
:1057580020460EF0E9FA012010BD0649F8E706498F
:10576800F6E70649F4E70649F2E70020F4E700BF48
:105778004C40010851400108564001085B400108AF
:105788006140010810B504460068FDF738F8024981
:105798002068FDF734F810BD674001080B1E18BFDC
:1057A8000123122A14D91D2A14D9312A8CBF0822A0
:1057B800052203710023016080F885304371C0F829
:1057C800883080F88C3080F88D20A0F88E307047B3
:1057D8000122EEE70322ECE790F88530642B08D825
:1057E800C2180133DBB2517180F8853018440023A8
:1057F8004371704708B50530FAF70AFDB0FA80F032
:10580800400908BD2DE9F04192B0064608460191CD
:105818001546FAF707FD06F1050804464046FAF76B
:1058280001FDE4B2631CC7B2BB42019903DB00204F
:1058380012B0BDE8F081224640460EF039FA002841
:10584800F5D1221D23461644BB4202461BD300F164
:1058580048036B44002403F8404C0028E7D09DF827
:1058680008303D2BE3D1302302A88DF80830FAF731
:10587800D9FC2346DAB2904212D802A80EF038F9C1
:1058880028600120D4E716F8011F202905D04832E6
:105898006A440130C0B202F8401C0133DBB2D3E7DE
:1058A80048326A44013312F8402C303A092AE1D9C7
:1058B800BDE7000010B50D4B1B78022B04460ED136
:1058C8000B4B93F8722052B19B6FB3F5215F07D24F
:1058D8000849FFF757FF08492046FFF753FF10BD57
:1058E800FDD00649FFF74EFF0549F5E78D07002073
:1058F800E40500206A400108A0400108D6400108DC
:105908000C41010810B50446FFF7D4FF2068074989
:10591800FCF784FF064B206819783031C9B2FCF7D0
:1059280062FF04492046FFF72DFF10BD42410108E0
:10593800CC030020483F01082DE9F0474379702B3C
:1059480090B080460F46164671D18379202B6ED1D0
:10595800C0790EF05DF900285CD000254FF0020AEE
:105968002C4608F105094846FAF75CFC824522D323
:1059780005F140030DEB0305002305F8403CC4B3D3
:10598800E8461D4618F8010B0EF04AF9785501351E
:10599800EBB2A342F6D300253D550134E4B2684684
:1059A800FAF740FC6719FFB2874206EB050334D3C8
:1059B80000221A702DE008EB0A035B793D2B0ED00C
:1059C800202B07D005F140016A1C0DEB010505F8F5
:1059D800403CD5B20AF101035FFA83FAC3E72C46CB
:1059E800F0E705F140036B4413F8400C0EF018F98A
:1059F80078556846FAF716FCE5B2A84207EB0503A6
:105A080004F10104EDD800220A491A7030460EF05C
:105A18008BF9012010B0BDE8F08707F140020DEBCB
:105A28000207013517F8402C1A70EDB2B7E70020CD
:105A3800F0E700BF504801082DE9FF472C4E282306
:105A480003FB016604463379FE2B0D4620D0FF2B5D
:105A58004BD0022B2DD196F9185026490068FCF737
:105A6800DDFE284669460CF03CFC69462046FFF7F7
:105A780089FE96F91C5020492068FCF7CFFE69463C
:105A880028460CF02EFC69462046FFF77BFE10E006
:105A98000846FFF7FBFCDFF86890DFF868A080464F
:105AA8000027FEB20123324629466846FFF766FC06
:105AB80010B904B0BDE8F087BBB248FA03F3DB07BE
:105AC80011D520684946FCF7A9FE06F13001206887
:105AD800C9B2FCF788FE20685146FCF79FFE69466C
:105AE8002046FFF74FFE0137DBE70449CDE700BF4B
:105AF800745201084C4101085441010863410108EE
:105B08005C4101085F410108F0B504468BB00846C6
:105B18000D46FFF7E3FC254F254906462068FCF7AC
:105B28007DFE282303FB05772068B968FCF776FE1D
:105B380020492068FCF772FE2EB91F492046FFF75E
:105B480021FE0BB0F0BD0122294602A8FFF72AFD6D
:105B5800206802A9FCF762FE3B79FE2B03D0FF2BDD
:105B68001AD01649EAE72846FFF7A4FB0578144936
:105B78002068FCF753FE05F130012068C9B2FCF734
:105B880032FE10492068FCF749FE012EE9D10E4982
:105B98002068FCF743FEE4E70C4B02A95A786846F4
:105BA800FFF7C8FD0028DCD06946F1E77452010808
:105BB8005C4101085F41010872410108483F010842
:105BC800824101087041010885410108CC03002089
:105BD80070B590F88E3004466BB990F88F30012B71
:105BE80001D9032B07D1214B1B78022B03D0204965
:105BF8002046FFF7C7FD1D4E002594F88E102B296F
:105C080003D9002384F88C3020E04B1C84F88E30B4
:105C180094F88F30012B09D10846FFF715FB0028AF
:105C2800EBD10846FFF722FB38B1E6E7022B0ED18D
:105C38000846FFF709FB0028DFD02046FFF764FF7E
:105C4800013594F88D30EDB2AB42D6D270BD032B3E
:105C580008D10846FFF70AFB0028CED03378022B7C
:105C6800DFD1EAE7002BF9D0E7E700BF8D07002076
:105C78009441010838B53D4B1A6890F88C30012BD7
:105C8800044671D1D0F88830D31AB3F5FA7F6BD3B4
:105C9800374DC0F888202846FBF71EF90CF030FB7A
:105CA80001462068FCF7BAFD32492068FCF7B6FDCA
:105CB80005F11400FBF7F7FC0CF022FB0146206805
:105CC800FCF7ACFD2C492068FCF7A8FD95F894007A
:105CD8000CF016FB01462068FCF7A0FD2749206858
:105CE800FCF79CFD95F98C000CF014FB014620682C
:105CF800FCF794FD22492068FCF790FD95F9920085
:105D08000CF008FB01462068FCF788FD1B49206859
:105D1800FCF784FD95F98E000CF0FCFA014620682A
:105D2800FCF77CFD17492068FCF778FD05F1500069
:105D3800FBF7BFFC80B20CF0F7FA01462068FCF7CD
:105D48006DFD0E492068FCF769FD05F16400FBF75D
:105D5800B0FC80B20CF0E8FA01462068FCF75EFD62
:105D680009492046FFF70EFD38BD00BF984A0020BC
:105D7800CC300020B1410108B3410108B641010807
:105D8800B4410108B9410108BC41010830B50446D5
:105D980089B0FFF78FFD13492046FFF7F3FC12493E
:105DA8002068FCF73BFD114B1B78022B18D1104DD6
:105DB80095F8723093B1206805F17C01FCF72EFD4F
:105DC8000C492068FCF72AFD696F6846FBF7BEFAA4
:105DD80069462046FFF7D6FC09B030BD0649F8E70A
:105DE8000649F6E7BE410108DC4101088D0700209D
:105DF800E4050020B6410108E34101089A41010881
:105E08002DE9F043324EDFF8D880DFF8D89091B012
:105E18000446002794F88D20FBB29A4209D994F8D9
:105E28008E50F37DAB4207F1010705D8002384F8B3
:105E38008C3011B0BDE8F08328460CF061FA0146B9
:105E48002068FCF7EBFC41462068FCF7E7FC731977
:105E58000E35187E0CF054FA01462068FCF7DEFC7B
:105E680049462068FCF7DAFC56F825000CF066FA7B
:105E780001462068FCF7D2FC16492068FCF7CEFCE6
:105E8800154908A80DF050FF06EB850393ED000AAD
:105E9800DFED127AB8EE400A20EE270A0CF0BEFEBB
:105EA800FCEEC07A694617EE900A0CF0E4F96846F1
:105EB800FBF784F920686946FCF7B0FC08A920467E
:105EC800FFF760FC94F88E30013384F88E30A1E738
:105ED800A00B0020094201080F42010800007A3A8D
:105EE800F8410108FF4101082DE9F041284E294FEA
:105EF800DFF8E0800446002594F88D20EBB29A4242
:105F080044D994F88E30142B3DD8DFE803F00B15F4
:105F18001A1C1E20222426282A2C2E303234363CE5
:105F28003C383A002046FFF7C5FC94F88E30013320
:105F380084F88E300135DFE717492046FFF722FC49
:105F4800F3E71649F9E71649F7E71649F5E7164959
:105F5800F3E71649F1E71649EFE71649EDE7164961
:105F6800EBE71649E9E71649E7E71649E5E7164971
:105F7800E3E71649E1E71649DFE74146DDE7394639
:105F8800DBE73146D9E7002384F88C30BDE8F0819F
:105F9800D3440108A7440108144201083442010807
:105FA8005E42010883420108AB420108CF42010862
:105FB800F34201081C4301084543010889430108CD
:105FC800AB430108CD430108EC4301081B44010819
:105FD800484401087F4401082DE9F04303799DB046
:105FE8000446C3B190F88C30013B032B19D8DFE885
:105FF80003F00252575C006803685B69984768B110
:10600800206803689B6998470023AB4984F88C3063
:106018002046FFF7B7FB1DB0BDE8F0832046FFF729
:1060280029FEA64B1E6894F885308BB1D4F88830C9
:10603800F31AB3F5FA6F0BD9A1492046FFF7A2FB73
:10604800A0492046FFF79EFB002384F88530637142
:106058009B4FDFF8D482DFF8D492206803685B692D
:1060680098470028D7D0206803689B6998470A2872
:106078000546C4F888601DD00D281BD02C2819D0DF
:106088003B2817D001462068FCF7ADFB294620467F
:10609800FFF7A2FBE1E71DB0BDE8F043FFF724BF1F
:1060A8001DB0BDE8F043FFF793BD1DB0BDE8F04358
:1060B800FFF7A6BE39462046FFF764FB4146204657
:1060C800FFF798FB50B1022384F88C30002384F842
:1060D8008E30002384F885306371BEE74946204638
:1060E800FFF788FB0028EED177492046FFF782FBAF
:1060F8000028E8D175492046FFF77CFB054618B112
:106108002046FFF743FEE4E771492046FFF772FB9C
:1061180040B12046FFF7F6FB032384F88C30A4F83F
:106128008E50D6E76B492046FFF764FB50B12046F6
:10613800FFF7E8FB032384F88C304FF48073A4F84E
:106148008E30C6E764492046FFF754FB40B120462D
:10615800FFF7D8FB032384F88C304FF40073EEE785
:106168005E492046FFF746FB40B12046FFF7CAFBD1
:10617800032384F88C304FF44073E0E70CAA04A999
:106188002046FFF7D9FB002846D004A90DF10A00E4
:10619800FFF7C6F920B952492046FFF7F3FA98E706
:1061A800504B1B78022B06D09DF80A00FFF75EF8CB
:1061B80008B14D49F0E79DF830303F2B0DD120460E
:1061C800FFF7A0FB9DF80A1001912046FFF79CFC01
:1061D80001992046FFF730FC7BE70BB94349DBE721
:1061E8009DF80A500CA92A460DF10B00FFF77EFA1C
:1061F80008B93F49D0E72046FFF784FB29462046E7
:10620800FFF782FC9DF80B30002B3FF462AF0521AD
:106218003848FBF779FA5CE737492046FFF7EAFA8E
:1062280090B134480621FBF76FFA2046FFF76AFB66
:106238002C4B1B78022B05D02B492046FFF7A2FADE
:106248002E49A9E72E49A7E72E492046FFF7D2FA9B
:1062580028B101212748FBF757FA2B499CE72B491E
:106268002046FFF7C7FA90B122480721FBF74CFAFE
:106278002046FFF747FB1B4B1B78022B05D01A491A
:106288002046FFF77FFA224986E7224984E7224918
:1062980003AA2046FFF7B6FA00285AD0039D092D15
:1062A80001D91E4978E72046FFF72CFB1C4B1B78C9
:1062B8009D423DD11B496FE710450108984A0020CF
:1062C8002A4501082C4501085048010801500108D9
:1062D8003B4501083E450108434501084945010879
:1062E8004F4501088D070020944101086B450108BE
:1062F8008345010898310020964501089D4501080D
:10630800B4450108C8450108CD450108E445010820
:10631800EB450108044601081A460108264601080B
:10632800CC0300204A4601080151010836450108FE
:106338002A4632480A21FBF7E9F931492068FCF777
:106348006DFA05F13001C9B22068FCF74CFA2D4905
:1063580022E72D492046FFF74DFA054640B10123B3
:106368002A4984F88C302046FFF70CFA284913E7AD
:1063780028492046FFF73EFA28B1042384F88C30D8
:1063880084F88E50A5E624492046FFF733FA08B171
:1063980003213DE721492046FFF72CFA08B10B21DC
:1063A80036E71F4903AA2046FFF72CFAE8B1039DF8
:1063B80042F22733A5F57A729A4201D91949EBE6D8
:1063C80014A9A8B20BF049FF14A8FAF7F7FE206841
:1063D8001549FCF723FA14A92046FFF7D3F9074813
:1063E8002A460C21FBF792F973E694F885100F4AB8
:1063F8000F4B00290CBF11461946CDE698310020F5
:106408005F460108483F01088846010875460108AB
:106418008E460108AB460108B5460108C04601088A
:10642800C8460108D4460108EC460108F6440108AC
:10643800024501080148FFF7CFBD00BFF406002060
:1064480070B5254CE569AB0607D523689E0604D5CB
:10645800606A224BC0B21B6898471F232806236234
:1064680015D52368190612D51D4B1E4A198813889D
:1064780089B29BB2994219D013880133C3F3080338
:1064880013801388184A9BB2D35CDBB2A3626A06F6
:1064980020D5114803685B061CD5FBF760FC402338
:1064A8000362124BBDE870401B6818470A48FBF7A7
:1064B8005FFC402323624FF0402202F5806353E8DB
:1064C800003F43F0400302F5806040E800310029B6
:1064D800F3D1DCE770BD00BF004400403C0200205F
:1064E80078360020763600207634002040020020DE
:1064F8000848094A0188138889B29BB29942F9D0A1
:1065080013880133C3F3080313801388034A9BB22B
:10651800D05C70477434002072340020723200203E
:10652800FFF7E6BF70B588B00C4606461546002151
:10653800202268460DF098FB231E18BF01231B0379
:10654800CDE9023569460C23034801960494059366
:1065580009F0A2FE08B070BD0044004010B5064C1A
:10656800236823F001032360FFF7DCFF236843F06F
:106578000103236010BD00BF0044004010B5134C58
:106588002046FBF7E3FBF1B111484FF400524FF4FA
:106598008061FFF7E3FF23680E4823F001032360BF
:1065A800636843F400436360636823F48033636083
:1065B800236843F001032360082303221946FCF7EC
:1065C8004EFAFBF7BFFF012010BD00BF004400409A
:1065D800A08601000004004810B5134C2046FBF7C4
:1065E800B5FBF1B111484FF400524FF48061FFF749
:1065F800B5FF23680E4823F001032360636843F462
:1066080000436360636843F480336360236843F046
:1066180001032360082302221946FCF720FAFBF73E
:1066280091FF012010BD00BF00440040A08601007A
:106638000004004810B53B4C236823F00103236095
:106648004FF40030FBF754FB0823194636480A225A
:10665800FCF705FA0823344803221021FCF7FFF958
:10666800002211463148FFF75DFF636823F4904329
:106678006360A36823F02A03A360236823F0005310
:1066880023604FF0402202F5816353E8003F23F076
:10669800604302F5816040E800310029F3D14FF0F2
:1066A800402202F5816353E8003F23F0606302F55E
:1066B800816040E800310029F3D11D4BA02283F806
:1066C800262340245C601748FBF752FBFBF747FB87
:1066D800184B04621980184B1980FBF737FB174BCE
:1066E8001980174B1980436823F40063436083685B
:1066F80023F008038360436823F48043436083687E
:1067080023F022038360836843F480538360036823
:1067180043F001030360C3699A02FCD5C3695B02B5
:10672800F9D510BD0044004000040048801A060056
:1067380000E100E076360020783600207234002030
:10674800743400200649074A0B8812880133C3F3C2
:10675800080392B29A421EBF034AD0540B80704776
:10676800783600207636002076340020F8B50123EC
:1067780080F86C3090F8BD30044603F0FF005BB140
:1067880094F8BD5004F16C070026B3B29D4204D8BA
:10679800002384F8BD300120F8BD17F8010FFFF77A
:1067A800D1FF0136F1E700000148FBF7C6BA00BF88
:1067B8000044004007B521B103B05DF804EBFCF7D5
:1067C80057B90D4B0D481A6822F001021A605A6831
:1067D80042F400425A601A6842F001021A600191BC
:1067E8000821009103230222FCF7AAF803B05DF800
:1067F80004EBFBF7A7BE00BF0044004000040048BC
:1068080010B50446FFF716FF134B14481A6822F018
:1068180001021A605A6842F400325A605A6842F417
:1068280080325A605A6842F400425A601A6842F04C
:1068380001021A60082319460222FCF710F90748DA
:10684800102103230222FCF700F920460021BDE8AD
:106858001040FFF7AFBF00BF0044004000040048ED
:10686800002282810271C280028182720261FFF776
:10687800C7BF036810B504461B689847237A082BDE
:1068880003D9092B02D00023237210BD23682046A8
:106898005B6898470028F6D0FCF7EAF80A232372C9
:1068A800BDE81040FFF780BF01460148FFF7E1BF90
:1068B800E016002001460148FFF7DBBF94070020DF
:1068C80010B500210446FFF775FF0023237210BDA1
:1068D8000148FFF7F5BF00BFE01600200148FFF7A9
:1068E800EFBF00BF9407002008B5017A094A0929BB
:1068F800126801D8026108BD0169521A142AFAD92E
:1069080000210172FFF756FF0348FBF728FA4023DE
:106918000362F0E7984A0020004400400238C0B201
:1069280010289ABF014B185C00207047CA51010813
:106938003B4B0246586A137A10B580B233B193893B
:10694800C31A9BB2FA2B84BF00231372137A908167
:10695800052B19D8DFE803F003080E334A564F29F0
:1069680012D1012313720FE0572901D10223F9E74D
:106978000023F7E70023FF29937206D141F204733D
:106988001381537E002BF3D110BD9F290FD901F03D
:106998001F000124947282F83200FFF7BFFF507283
:1069A80018B982F84B400923DCE70523DAE71829F0
:1069B800DED80029F7D0032351721372E1E7B2F849
:1069C8006E02B2F87242431C2340B2F870429C42F5
:1069D8001EBF801880F87412A2F86E32937A517A2A
:1069E8000133DBB299429372DDD9CDE7907A431C2B
:1069F8001044DBB29372C176517A9942C4D801230C
:106A08009376D0E7907A431C1044DBB2937280F8F7
:106A18003210517A9942B7D2012382F84B30C2E73B
:106A2800000400402DE9F04389B0002301AFB0F81D
:106A380068908DF804300446B8460125B4F86A20F9
:106A480048461146EEB2FBF7F7FDA0B1192D11D05B
:106A580091451FBFA318B4F86C1093F86E3001323B
:106A680014BF0A40002308F8013F18BFA4F86A20A1
:106A78000135E3E72E46B6B20024013417F8010BBE
:106A8800A4B2FFF75FFEA642F7D8012009B0BDE81F
:106A9800F08370B590F8665000F14C040026B3B24C
:106AA8009D4200D870BD14F8010FFFF74BFE013668
:106AB800F5E770B5457E044605B1FEE7012680F886
:106AC8004C6090F8663033B1FFF7E3FF84F8665006
:106AD8003546284670BDB0F86A10B0F86800FBF774
:106AE800ABFD0028F5D02046FFF79CFFF0E7027FBA
:106AF800C37E02F0070243EA02230B80838BC3F3B1
:106B0800CA034B80C369C3F38A338B8090F8203063
:106B1800C27F03F00F03DB0143EA5203CB80038CEF
:106B2800C3F30A130B81036AC3F3CA334B8190F88A
:106B3800243090F8232003F01F039B0143EA9203BB
:106B48008B81838CC3F34A13CB81C38CC3F30A03B1
:106B58000B8290F8283090F8272003F03F035B0160
:106B680043EAD2034B82836AC3F38A138B82438D31
:106B7800C3F34A03CB8290F82C3090F82B2003F013
:106B88007F031B0143EA12130B83C36AC3F3CA13BF
:106B98004B83C38DC3F38A038B8390F8303090F80E
:106BA8002F20DB0043EA5213CB8390F8312040F2C8
:106BB800547312F0010F14BF1A46AC220A8490F8DD
:106BC800312012F0020F08BFAC234B847047437E7C
:106BD80070B5044643B1002303720D468E18B542C2
:106BE80003D100232372A37670BD236815F8011B17
:106BF8001B6820469847F2E7437E30B56BB190F8A2
:106C0800664004F0FF0554B100F14D040C6090F8A3
:106C180066101170002280F86620184630BD2B4699
:106C2800FBE7000042765AB30123037640F2FF11D6
:106C3800A0F86C1040F2FF710023A0F872127F21B7
:106C480080F84C30A0F86A308376A0F8683080F875
:106C58004B30A0F8703280F86630A0F86E32A0F899
:106C6800763AA0F8743AA0F8781A80F8FA3A52B945
:106C7800054B064A1A60064B064A1A60FFF7F0BD34
:106C880001760029D2D170473C020020B168000883
:106C980040020020D968000873B5467E04461EB13C
:106CA8000025284602B070BD037E0191002BF7D065
:106CB800FFF71AFEA37E03F0FF05002BF0D0019921
:106CC800A6762046FFF713FFEBE7427E10B5EAB938
:106CD800037EBBB190F84C4004F0FF0394B10479F3
:106CE80080F84C200CB10271C280C48882790134CA
:106CF800052AC48008D0092A06D0012A4FF00002CC
:106D080006D10A70184610BD0122FAE70023F9E7F8
:106D18001346F7E7037E63B190F84B2002F0FF03B8
:106D28003AB1002280F84B2090F8322002F01F027E
:106D38000A7018467047F8B506460D4617460021F2
:106D480019224D300CF090FF2846FFF7E7FD05F0BB
:106D58001F050446603D0134024686F84D50394609
:106D680006F14E00E4B20CF0E7FF86F86640F8BD85
:106D780070B590F8FA4AC4B9B0F8745AB0F8762ADF
:106D8800AE1AB3B2360444BF80339BB27BB195428E
:106D980008D08318013293F87A4AB0F8783A1A4042
:106DA800A0F8762A0C70012070BD0020FCE7184678
:106DB800FAE7000010B53A4C86B018220021684660
:106DC8000CF052FF237837488DF80630FDF7C0FBEA
:106DD800ADF800003348FDF7D2FB9DF8073094F872
:106DE80051208DF8030062F303038DF807302E4B12
:106DF80093F87220002A47D09DF8052042F001023E
:106E08008DF8052093F8912093F892308DF804209E
:106E180003F00F039DF80720244863F30712244B5F
:106E28008DF807201A78931E5A425A41214B1B7934
:106E38005B0043F0010343EA820390F89320402A61
:106E48008CBF0022012243EAC2039DF8022003F00E
:106E58000F0322F00F0213438DF80230FAF73CF8C3
:106E68009DF8023040288CBF0020012060F30413F5
:106E78008DF8023010482C236A460B218DF8083013
:106E8800FFF759FF06B010BDBDF8043023F4FF73B7
:106E980023F0010343F07F03ADF804300523B9E77D
:106EA800CC03002074310020E4050020CC30002001
:106EB8008D070020C0060020E01600207FB51822AC
:106EC800002168460CF0D0FE42F64200FAF720FA9C
:106ED800ADF800004FF42150FAF71AFA0749ADF857
:106EE8000200142201A8FAF77DFA05486A4604212F
:106EF800FFF721FF07B05DF804FB00BFF746010864
:106F0800E016002010B5124C86B018220021684601
:106F18000CF0AAFE94F87230B3B1606FFAF7F8F982
:106F2800ADF80000A06FFAF7F3F91422ADF80200EB
:106F380004F17C0101A8FAF755FA06486A460521CA
:106F4800FFF7F9FE06B010BD03491422F2E700BFAF
:106F5800E4050020E0160020483F01082DE9F04F25
:106F6800344C282303FB014489B007460846FEF742
:106F78008DFA2379D4F82080FE2B814603D14FF671
:106F8800FF73984206D14146384609B0BDE8F04F34
:106F98000CF0CABE0846FEF78DF9002590F800B03F
:106FA8002E46AA462C46EAB240460192F9F73AF92B
:106FB800019A013090424FF02D0102D809B0BDE886
:106FC800F08F18F802000AF1200CEC440AF10103D2
:106FD8002C28DBB20CF8180C00D040BB5E4503D05F
:106FE80049FA06F0C00718D50DF1080E0022D0B2F4
:106FF80054FA82FC83425FFA8CFC08D8544401346A
:1070080004F0FF040136502CF6B20FD9FEE71EF843
:10701800010B07F80C000132E9E73955631CDBB2B4
:1070280018F80220FA540234E4B2EBE700230135E1
:107038009A46B8E774520108054B1870054B064884
:1070480000221A70054B012207211A70FBF7E8BAD3
:10705800252F0020262F002054210020242F002037
:10706800054A064800231370054A1370054A07218C
:107078001370FBF7D5BA00BF252F0020542100203C
:10708800262F0020242F002010B50B78033B0C4638
:10709800082B0BD8DFE803F010050C1A1D0A0A0AA2
:1070A8000E00042100F67420FBF7BAFA207810BD10
:1070B8000521F7E70B21F5E7042100F67420FBF71B
:1070C800AFFA0521FBF7ACFA0B21EDE7FFF7C8FF94
:1070D800ECE74878FFF7B0FFE8E707B58DF8071049
:1070E8000DF10701FFF7D0FF03B05DF804FB0000C6
:1070F800F0B5704D2C782B2C87B00ED918220021B2
:1071080068460CF0B1FDFF236B488DF800306A46E5
:107118000721FFF710FE07B0F0BD684E317818223E
:1071280000294AD1664F68460CF09EFD282303FBD0
:1071380004738DF800401B79FE2B29D0FF2B2FD02C
:10714800022B09D1012320468DF80130FEF7B2F851
:1071580090F900308DF812302B78282202FB037743
:107168000DF10200B9681022FAF73CF952480721DC
:107178006A46FFF7E0FD0123297852483370FFF78C
:10718800EDFE5148072107B0BDE8F040FBF748BACB
:10719800042320468DF80130FEF78CF80378D9E7F0
:1071A800052320468DF80130FEF784F806220146B3
:1071B8000DF11200FAF716F9CEE7012947D100219F
:1071C80068460CF051FD3E4B8DF80040282202FB2A
:1071D80004331A79022A0BD0FE2A19D00024364823
:1071E8006A460821FFF7A7FD44B302233370C8E7B6
:1071F8001A7D8DF805201A7E8DF801201A7F8DF8EA
:107208000320196906220DF10700FAF7EBF8E5E704
:107218005B6A83B11B882B49ADF8013015220DF14B
:107228000300FAF7DFF82748F8F7FCFF142894BFA3
:1072380000240124D3E74FF6FF73ECE734702B7872
:1072480001332B70214B1B78002B9AD063E702295E
:1072580068464FF0000116D10CF006FD1C498DF868
:10726800004017220DF10100FAF7BCF81548F8F7AD
:10727800D9FF6A46044609210F48FFF75CFD2B2C0D
:1072880015D90323B2E70CF0EFFC12498DF8004042
:1072980017220DF10100FAF7A5F89DF8003006480D
:1072A800803B6A4609218DF80030FFF744FD002332
:1072B8003370C4E7252F0020E0160020262F002079
:1072C80074520108272F002054210020242F002069
:1072D8003C2F0020532F002010B500230B700246CE
:1072E80000782B280C4611D8094B282101FB0033C4
:1072F8001B79FF2B06D0B2F90110FDF7F7FF2070BC
:10730800012010BD511CFEF715F8F8E71846F8E7FC
:1073180074520108043807280DD8DFE800F0040685
:107328000C080C0C0C0AFFF7C9BDFFF7EBBDFFF703
:10733800DFBEFFF73FBD7047D20638B505460C469D
:1073480004D5BDE8384020490CF0EEBCCB044CBF56
:107358001E491F490CF0E8FCA1070BD51D4928461A
:107368000CF0E2FCE3072ED428461B49BDE8384060
:107378000CF082BCA20501D51849F0E7230601D517
:107388001749ECE7E00501D51649E8E7164BA34392
:1073980001D11649E3E7E10301D51549DFE72205E5
:1073A80001D51449DBE7E30601D51349D7E76007A0
:1073B80001D51249D3E7210701D51149CFE7E202E8
:1073C800D0D51049CBE738BD064701080B4701085F
:1073D8000F470108144701083947010819470108F0
:1073E800DA4B0108CD4D0108100001001E470108C5
:1073F800234701083A4C0108284701082B47010890
:10740800304701083447010810B51422044600210A
:107418002A300CF029FC0023C4F8D032A4F8D43266
:10742800012384F8D63210BD0B68C0F890304B6841
:10743800C0F894300B7A80F89830012380F82D300A
:1074480080F8333090F89630DB0980F8D5327047F1
:10745800993001F1280351F8042B40F8042B994284
:10746800F9D10B8803808B788370704710B500F1D1
:10747800C40301F1340251F8044B43F8044B914220
:10748800F9D1012380F82E3010BDF83001F11C032A
:1074980051F8042B40F8042B9942F9D10B7803706A
:1074A800704710B500F2151301F11C0251F8044B96
:1074B80043F8044B9142F9D1012380F8323010BDD2
:1074C80010B500F2311301F11C0251F8044B43F8D6
:1074D800044B9142F9D140F201134385012380F80E
:1074E800303080F8D23290F8D53253B990F8D4328F
:1074F8003BB9D0F83931C0F82C32D0F83531C0F862
:10750800283210BD00F2671001F1100351F8042B66
:1075180040F8042B9942F9D10B880380704700F298
:107528004D1001F1180351F8042B40F8042B99422F
:10753800F9D10B880380704710B500F2791301F177
:10754800140251F8044B43F8044B9142F9D101233A
:1075580080F83130D0F8993013F0100308D0D0F803
:107568009D3013F010031CBFD0F8A130C3F30013F3
:1075780080F83D3010BD00F28D1001F1140351F870
:10758800042B40F8042B9942F9D10B8803807047EB
:1075980091F8203030B57BB90B4600F2A31201F107
:1075A800340453F8045B42F8045BA342F9D11B8806
:1075B8001380012380F82F3091F82030012B0ED151
:1075C80000F2D91301F1340251F8044B43F8044B8B
:1075D8009142F9D10A881A80012380F8343030BDED
:1075E8000B68C0F80F324B68C0F813320B7A80F87A
:1075F8001732012380F8D33270470B68C0F818326D
:107608004B68C0F81C32012380F8323070470B6891
:10761800C0F820324B68C0F82432012380F8363095
:10762800704710B500F50A7301F13C0251F8044B9C
:1076380043F8044B9142F9D1012380F8303080F8A7
:10764800D43210BD10B500F5197301F1340251F8A8
:10765800044B43F8044B9142F9D10A881A8001235C
:1076680080F82C3010BDF0B500252C460126AB4221
:1076780006D80368214001FA02F213430360F0BD03
:1076880006FA05F73C430135F1E770B504460846AC
:1076980094F82A6016B90026304670BD94F8E03098
:1076A8000022022B84F82A20F5D90A60D4F8355133
:1076B800002DC8BF6D423223B5FBF3F11E2301EB49
:1076C8004101FFF7D0FFD4F8351102231E22C90F5C
:1076D800FFF7C9FFE0E770B50446084694F82B6049
:1076E80016B90026304670BD94F8E0300022022B0F
:1076F80084F82B20F5D9D4F839510260002DC8BF81
:107708006D423223B5FBF3F11E2301EB4101FFF774
:10771800AAFFD4F83931002B4FF002034FF01E02B4
:10772800B4BF03211946FFF79EFFDBE738B50446CF
:10773800084694F8D022AAB994F82C30DBB384F820
:107748002C2004F5197304F29A2204F5267153F8D3
:10775800045B42F8045B8B42F9D11B881380012338
:10776800A4F8D03200230360182594F8D132312BC5
:1077780006D85A1C234484F8D12293F89B12E1B905
:1077880094F89A12012319400722FFF76CFF94F826
:107798009A1201230F22C1F34001FFF764FF94F806
:1077A8009A1201231722C1F38001FFF75CFF00231F
:1077B80084F8D0320123184638BD2A46083D0723ED
:1077C800EDB2FFF750FFF82DCFD194F8D132312B1D
:1077D800D6D8EFE703462DE9F04793F82D60084621
:1077E800002E65D093F81552D3F89010B3F88B415A
:1077F80093F8D57293F8D3820022AD1A83F82D201E
:1078080001F1010118BF01254CB1632CD7BFC4EBAE
:1078180084143F2431346422D8BFB4FBF2F4B3F9A2
:107828001331002B47D0642293FBF2F3522BA8BFED
:107838005223132BB8BF1323A3F113094FF0000AE7
:1078480005235246C0F800A0FFF70DFF02230522CA
:107858005146FFF708FF012307223946FFF703FFC8
:10786800012308223946FFF7FEFE0123092251466B
:10787800FFF7F9FE02230A225146FFF7F4FE01231F
:107888000C225146FFF7EFFE01230D224146FFF778
:10789800EAFE01230E222946FFF7E5FE07231322FD
:1078A8002146FFF7E0FE06231A224946FFF7DBFED2
:1078B8003046BDE8F0879946C0E700002DE9F84357
:1078C80090F82E800D46B8F1000F3AD090F8E130CC
:1078D8000021FF2B80F82E1003D00F2B28BF0F2379
:1078E800194690F8E090B9F1030F2DD84FF0000633
:1078F8002FD07F273446002228462A600423FFF72A
:10790800B2FE022304224946FFF7ADFE01220221FE
:107918003846F9F74BFF0823014606222846FFF7A9
:10792800A2FE02230E223146FFF79DFE02221146D7
:107938002046F9F73BFF0A23014616222846FFF79F
:1079480092FE4046BDE8F883A9F10306062E28BF3B
:1079580006260A23B0F8D870D0F8D440B7FBF3F75E
:107968000B4B7F2FA8BF7F279C4208DC094B9C420A
:1079780009DB64234FF0030994FBF3F4BBE7064CDF
:107988004FF00309B7E7054C4FF00309B3E700BF11
:10799800C3C9C1003D363EFF18F00100E80FFEFFE5
:1079A8002DE9F04190F830302DED088B05460E4654
:1079B8002BB90027BDEC088B3846BDE8F08190F85C
:1079C800D272002380F83030002FF2D0D0ED8A7ABE
:1079D800D0F835319FED60BA9FED60AAF8EEE78ADE
:1079E80009EE103A68EE8B8AB8EEC99A68EE8A8A70
:1079F80029EE0B9AB0EE680A0BF074F829EE0A9A91
:107A0800F0EE40AAB0EE490A0BF06CF8D5F839311F
:107A1800D5ED8B7A08EE103AB8EEC88AF8EEE77A18
:107A280028EE0B8A6BEE677A28EE0A8AF0EE409A07
:107A3800A7EE8A8A4FF00008B0EE480A0BF09EF8CD
:107A480029EE80BAB0EE490A0BF098F8F0EE40BA89
:107A5800B0EE680A0BF092F8B0EE40AAB0EE480A11
:107A68000BF040F829EE8AAA60EE4A0AB0EE4B0AFB
:107A7800EAEEAB0A0BF016F8DFED397A60EE277AFA
:107A880039EE689AF5EEC07AF1EE10FA44BF9FED30
:107A9800357A77EE877AB6EE00AAFDEEE77A29EE18
:107AA8000A0A17EE903A9BB2A3F1B40424B2002C50
:107AB800BCBFB4331CB2B4F5B47FA4BFA4F5B4748E
:107AC80024B20BF05BF8F0EE408A28EE0A0A0BF0BD
:107AD80055F860EE007A67EEAA7A27EEA90AA8EEB2
:107AE800A80A0AF0E1FF0AF0B1FFDFED1F7AD5F826
:107AF8004131C6F8008020EE270A6422BDEEC00A94
:107B080093FBF2F5B8EEC00A0222FDEEC07A03211B
:107B180017EE900AF9F74AFE07EE905A01460C2331
:107B280042463046FFF79FFDF8EEE77A0222FDEE67
:107B3800E77A032117EE900AF9F738FE0D2301467C
:107B48000C223046FFF78FFD07231922032194FBEF
:107B5800F1F1FFF788FD2DE795BFD63335FA8E3C56
:107B6800E12E65420000B443706D424BF8B590F8C1
:107B780031702DED028B04460D46002F43D0D0F80E
:107B8800853100EE103A0026B2EE048A80F83160A2
:107B980028EE000A0BF042F8D4F87D31F0EE408A66
:107BA80000EE103A28EE000A0BF038F8B4F9891103
:107BB8002E60FDEEE87A01EB810417EE900A0122AF
:107BC8000221B0EE408AF9F7F1FD09230146324659
:107BD8002846FFF748FDFDEEC87A0122022117EE7C
:107BE800900AF9F7E3FD0823014609222846FFF722
:107BF8003AFD0B2311222146FFF735FD01231C22F4
:107C08003146FFF730FDBDEC028B3846F8BDF8B5BC
:107C180090F83D702DED028B04460D46002F43D0A1
:107C2800D0F8853100EE103A0026B2EE048A80F8CA
:107C38003D6028EE000A0AF0F1FFD4F87931F0EE41
:107C4800408A00EE103A28EE000A0AF0E7FFB4F97D
:107C580089112E60FDEEE87A01EB810417EE900A97
:107C680001220221B0EE408AF9F7A0FD092301465E
:107C780032462846FFF7F7FCFDEEC87A01220221BA
:107C880017EE900AF9F792FD0823014609222846C3
:107C9800FFF7E9FC0B2311222146FFF7E4FC01233F
:107CA8001C221946FFF7DFFCBDEC028B3846F8BDF5
:107CB800F8B590F832702DED048B04460D46002F70
:107CC8004AD0D0F819319FED269A9FED260A07EE83
:107CD800903A67EE897A0026B1EE048A80F832601D
:107CE800A7EE880A0AF09AFFD4F81D3107EE903AF9
:107CF800F0EE408A67EE897A9FED1B0AA7EE880AA4
:107D08000AF08CFFDFED197AB0EE408A94ED860A0E
:107D180020EE270A0AF082FFFDEEE87A284617EEE1
:107D2800901A0B2332462E60FFF79DFCFDEEC87AB1
:107D38000A2317EE901A0B22FFF795FCFDEEC07A86
:107D48000122032117EE900AF9F730FD0B230146B3
:107D580015222846FFF787FCBDEC048B3846F8BD92
:107D6800E12E6542000061440000E1430000C84282
:107D780038B50346084693F8334014B90024204622
:107D880038BD93F8D652691CC9B20022042983F879
:107D9800332083F8D61203D9012183F8D612EDE7F0
:107DA800012DEBD193F8941002601823FFF75BFCC8
:107DB800042318222946FFF756FCE0E71C2945D87A
:107DC800DFE801F00F121416181A1C1E4420442272
:107DD800442426282A2C2E30323436383A3C3E4069
:107DE80042001B490BF0A0BF1A49FBE71A49F9E703
:107DF8001A49F7E71A49F5E71A49F3E71A49F1E783
:107E08001A49EFE71A49EDE71A49EBE71A49E9E792
:107E18001A49E7E71A49E5E71A49E3E71A49E1E7A2
:107E28001A49DFE71A49DDE71A49DBE71A49D9E7B2
:107E38001A49D7E71A49D5E71A49D3E71A49D1E7C2
:107E48001A49CFE71A49CDE71A49CBE71A49C9E7D2
:107E5800D14B01080F4701083B470108404701087B
:107E6800454701084A4701084F4701085447010898
:107E7800594701085E470108634701086847010838
:107E88006D47010872470108774701087C470108D8
:107E980081470108864701088B4701089047010878
:107EA800954701089A4701089F470108A447010818
:107EB800A9470108AE470108483F0108192941D8D8
:107EC800DFE801F00D10121416181A1C1E402022AB
:107ED8002426282A2C2E30323436383A3C3E1A4989
:107EE8000BF022BF1949FBE71949F9E71949F7E7E8
:107EF8001949F5E71949F3E71949F1E71949EFE78E
:107F08001949EDE71949EBE71949E9E71949E7E79D
:107F18001949E5E71949E3E71949E1E71949DFE7AD
:107F28001949DDE71949DBE71949D9E71949D7E7BD
:107F38001949D5E71949D3E71949D1E71949CFE7CD
:107F48001949CDE71949CBE71947010854470108F2
:107F5800D14B0108B34701080F470108B84701088A
:107F6800BD470108C24701086D470108404701089D
:107F78004F4701084A470108C747010881470108D8
:107F880045470108CC470108D1470108D6470108F1
:107F9800DB470108E0470108E5470108EA4701080F
:107FA800EF470108F4470108F9470108483F01086D
:107FB800102925D8DFE801F0090C240E1012141638
:107FC80018241A1C1E24242022000E490BF0ACBED3
:107FD8000D49FBE70D49F9E70D49F7E70D49F5E7C5
:107FE8000D49F3E70D49F1E70D49EFE70D49EDE7D5
:107FF8000D49EBE70D49E9E70D49E7E70D49E5E7E5
:108008000D49E3E7194701080F470108FE47010832
:10801800CD4D01084A470108954701080348010862
:1080280008480108404701084F4701088B470108E5
:1080380045470108CC470108483F0108142921D8C1
:10804800DFE801F00B0E1012142020162018202053
:10805800202020201A20201C1E000B490BF064BE93
:108068000A49FBE70A49F9E70A49F7E70A49F5E740
:108078000A49F3E70A49F1E70A49EFE70A49EDE750
:108088000A49EBE70A49E9E7D14B01080F4701081C
:108098000D480108404701084547010854470108B1
:1080A80012480108724701081947010817480108D2
:1080B800483F010823289ABF014B185C02207047EB
:1080C800DB5101080B46013B1146032B0BD8DFE8B7
:1080D80003F002040608FFF771BEFFF7EFBEFFF7D3
:1080E80067BFFFF7ABBF01490BF01EBE483F010851
:1080F80038B5384B0446821C03F1280153F8040BA9
:1081080042F8040B8B42F9D100252946C4E92455CD
:1081180084F898502B2204F199000BF0A5FD29460C
:10812800342204F1C4000BF09FFD29461D2204F1FE
:10813800F8000BF099FD29461C2204F215100BF0EB
:1081480093FD29461C2204F231100BF08DFD2946BF
:108158001A2204F24D100BF087FD2946122204F270
:1081680067100BF081FD2946142204F279100BF0F8
:108178007BFD2946162204F28D100BF075FD294669
:10818800362204F2A3100BF06FFD2946362204F2C2
:10819800D9100BF069FD2946C4E98655C4E988550C
:1081A800C4F80F52C4F8135284F817523C2204F54D
:1081B8000A700BF059FD2946362204F519700BF0A8
:1081C80053FD3622294604F29A200BF04DFD204635
:1081D80038BD00BF743D01082DE9F04F2DED068B29
:1081E80085B0437EC77E0093837E009A457F867F55
:1081F80090F820C090F82BE090F82D80BF000C4636
:1082080047EA931703F03F01037F490141EAD2018E
:1082180003F0010247EA822705F00F02D20142EA81
:10822800530206F07F031B0143EA1513C57F019330
:108238006D0045EAD6150CF0030645EA462390F88A
:108248002160029206F01F05AD0108EE103A45EADA
:108258009C0390F8225090F824C00391ED0008EE9A
:10826800903A45EA561390F823500CF0070609EEA9
:10827800103A45EA062390F8255005F03F067601A6
:1082880009EE903A46EADC0390F8266090F827C099
:10829800B60046EA95160CF0010546EA852690F8E0
:1082A800285005F00F0B4FEACB1B4BEA5C0B90F8FC
:1082B80029C00CF07F0A4FEA0A1A4AEA151A90F800
:1082C8002A506D0045EADC150EF0030C45EA4C25F2
:1082D80090F82CC00AEE103A4FEAC808009B48EA0A
:1082E8005C180CF01F0990F818C003F007004CEA5E
:1082F80000204FEA891949EA9E09F8F766FE0399B2
:1083080020800846F8F761FE60803846F8F75DFE81
:10831800029AA0801046F8F758FE019BE0801846A4
:10832800F8F753FE208118EE100AF8F74EFE608128
:1083380018EE900AF8F749FEA08119EE100AF8F72E
:1083480044FEE08119EE900AF8F73FFE20821AEE0B
:10835800100AF8F73AFE60823046F8F736FEA08237
:108368005846F8F732FEE0825046F8F72EFE208392
:108378002846F8F72AFE60834846F8F726FEA083C9
:108388004046F8F722FEE08305B0BDEC068BBDE859
:10839800F08F4A78013A92B202310020F8F776BE9F
:1083A80038B504460175002944D04FF6FF730025FF
:1083B800A0F8F030204B80F8BD5080F8CE5080F8FF
:1083C8006C50C0F8D05080F8655080F8DC5080F8C8
:1083D8006650C0F8E05080F8675080F8EA5080F89E
:1083E8006850C0F8EC5080F86A50C0F8F43080F853
:1083F8006B5080F80751C0F8085180F80E51C0F84A
:10840800105180F81651C0F8185100F58E70FEF71B
:10841800FBFF0A4B0A4A1A600A4B0B4AC4F8F4538A
:10842800A4F8F853C4F8FC531A602046BDE8384055
:10843800FEF716BA38BD00BF0000C07F3C0200201E
:10844800BD68000840020020E5680008037D70B59B
:1084580004460D4613B90026304670BDFEF744FAAF
:1084680094F8653003F0FF06002BF4D0002384F85D
:10847800653004F115012046FFF78BFFA37D2344E7
:108488009B7D8342E7D129462046FFF7A5FEE3E717
:108498000346007D30B500B393F86C4004F0FF004C
:1084A800DCB11D79002483F86C4065B1132A1C7176
:1084B80014D8134C227802B9DA800132D2B2022AD7
:1084C80088BF00222270DC889A790134012ADC8076
:1084D80002D0022A00D01AB90A7030BDDC80F2E757
:1084E80093F8672002F0FF0432B1002283F8672076
:1084F80004230B702046F0E703230B70EDE700BF61
:10850800BD060020027D03460AB90020704790F896
:10851800682002F0FF0022B1002283F868200A7068
:10852800704793F86A2002F0FF002AB1002283F80E
:108538006A2001230B70704793F86B2002F0FF004C
:1085480022B1002283F86B200223F3E793F8662018
:1085580002F0FF00002AD8D0002283F866205A7D56
:10856800EE2AD2D1DB7D812BCFD10323E2E738B5C8
:1085780004461D46EA23084684F86D30AB1C1146B4
:1085880084F86E302A4684F86F0004F170000BF00E
:10859800D3FB04F16D012046FFF7FBFE6319043598
:1085A80083F87000EDB284F8BD5038BD13460A4612
:1085B8008221FFF7DCBF000070B50C4600F1BE0653
:1085C80005461022002130460BF04EFB6379032B41
:1085D80010D12079FFF76EFD22680146D2B23046ED
:1085E800FFF770FD94F90630002B03DB0349304692
:1085F8000BF042FB012385F8CE3070BD39470108E6
:10860800002310B51A464FF6FF74191D00EB4101FF
:1086180001334988A14218BF52180A2BF5D1B0F886
:1086280029301344B0F82B201A44B0F82D30B0F894
:108638002F001344184410BD2DE9F04190F82F7015
:1086480004460D4697B3002680F82F6000F2A31069
:10865800FFF7D6FFB4F9C131D4F8A3812E60B34235
:10866800B8BF34464FF0640290FBF2F1A8BF0A226B
:108678002846A8BF93FBF2F409230022FEF7F3FF74
:10868800012202212046F9F791F808230146092220
:108698002846FEF7E8FF47F6FF7141454FF00F0304
:1086A8004FF01102A8BF4146FEF7DDFF3846BDE88E
:1086B800F0812DE9F04190F8347004460D4697B3E7
:1086C800002680F8346000F2D910FFF799FFB4F95A
:1086D800F731D4F8D9812E60B342B8BF34464FF091
:1086E800640290FBF2F1A8BF0A222846A8BF93FBB8
:1086F800F2F409230022FEF7B6FF012202212046E8
:10870800F9F754F80823014609222846FEF7ABFF7B
:1087180047F6FF7141454FF00F034FF01102A8BF14
:108728004146FEF7A0FF3846BDE8F081F0B591B0AC
:108738000D46F22301A904461646ADF80830FFF7A6
:1087480049F838B12389ADF80A30019B0393012316
:108758008DF8093001A92046FFF708FA70B19DF895
:10876800093010A9062202FB0312218A22F8361CBE
:108778000133019942F8341C8DF8093001A92046CB
:10878800FFF745FA70B19DF8093010A9062202FBDF
:108798000312218D22F8361C0133019942F8341C4A
:1087A8008DF8093001A92046FFF782FA70B19DF8CB
:1087B800093010A9062202FB0312618A22F8361C2E
:1087C8000133019942F8341C8DF8093001A920467B
:1087D800FFF774F870B19DF8093010A9062202FB62
:1087E8000312618922F8361C0133019942F8341CBE
:1087F8008DF8093001A92046FEF747FF70B19DF8B2
:10880800093010A9062202FB0312618822F8361CDF
:108818000133019942F8341C8DF8093001A920462A
:10882800FEF759FF70B19DF8093010A9062202FB26
:108838000312A18822F8361C0133019942F8341C2E
:108848008DF809309DF80970082F11D801A9204624
:10885800FFF7F2FE60B110AA062303FB0723A289E3
:1088680023F8362C0137019A43F8342C8DF8097017
:108878009DF80970082F11D801A92046FFF719FFA4
:1088880060B110AA062303FB0723E28A23F8362CDB
:108898000137019A43F8342C8DF809709DF8097056
:1088A800082F11D801A92046FFF77AF860B110AA5D
:1088B800062303FB0723E28923F8362C0137019AA4
:1088C80043F8342C8DF809709DF80970082F11D8D9
:1088D80001A92046FFF74CFA60B110AA062303FB52
:1088E8000723A28A23F8362C0137019A43F8342C3F
:1088F8008DF809709DF80970082F11D801A9204634
:10890800FEF714FF60B110AA062303FB0723E288D1
:1089180023F8362C0137019A43F8342C8DF8097066
:108928009DF8090050B100EB40035B000233DAB256
:10893800327002A928460BF0FFF9012011B0F0BDF2
:1089480010B5524BD0F8D0201B6894B004463AB109
:108958009A1A40F6C4118A4284BF012280F8CE20B8
:10896800D4F8E0203AB19A1A40F6C4118A4284BF7A
:10897800012284F8DC20D4F808213AB19A1A40F68A
:10898800C4118A4284BF012284F80721D4F8102137
:108998003AB19A1A40F6C4118A4284BF012284F877
:1089A8000E21D4F8EC203AB19A1A40F6C4118A4242
:1089B80084BF012284F8EA20D4F818213AB19A1A1F
:1089C80040F6C4118A4284BF012284F8162194F823
:1089D800CE2072B1002284F8CE20C4F8D03004F141
:1089E800BE0210232121204614B0BDE81040FFF735
:1089F800BEBD94F8DC1041B1C4F8E030082384F817
:108A0800DC20194604F1D402EDE794F8072142B1BD
:108A180084F80711C4F8083104F1F8020F23022181
:108A2800E1E794F80E1141B184F80E21C4F8103131
:108A380004F5867202230721D5E794F8EA2042B1AB
:108A480084F8EA10C4F8EC3004F1E40206231E218D
:108A5800C9E794F8161141B184F81621C4F8183101
:108A680004F58A7202230921BDE70DF1030201A969
:108A780004F58E70FFF75AFE30B19DF8033001AA55
:108A880080212046FFF773FD14B010BD984A0020DE
:108A980070B591F8205004460E465DBB0846FFF7B6
:108AA800AFFD642390FBF3F040BAA4F8D400B6F904
:108AB8001E30581C1CBF0A2593FBF5F56DBAA4F8A7
:108AC800D6503368591C16D00C4A934228BF134617
:108AD8001A0C84F8D8201A0A84F8D92084F8DA30D5
:108AE80096F923305A1C08BF002384F8DB30012391
:108AF80084F8DC3070BD0023EAE700BFFFFF7F0089
:108B08008B689FED147A07EE903A67EE877AFDEE50
:108B1800E77A17EE903A5BBAA0F8E4304B6807EEB4
:108B2800903A67EE877AFDEEE77A17EE903A5BBAED
:108B3800A0F8E630CB6807EE903A67EE877AFDEE4C
:108B4800E77A17EE903A5BBAA0F8E830012380F88C
:108B5800EA30704700401C464B681BBAC0F8F83032
:108B68008B681BBA4FF47A72C0F8FC30CB6893FB61
:108B7800F2F3134483F310035BBAA0F804314B8B70
:108B88005BBADFED137A90ED3D7ADFED126AA0F85B
:108B9800023127EE277AC7EE267AFCEEE77A17EE3F
:108BA800903A5BBAA0F8003190F8F030FF2B0CD067
:108BB80090F8F120FF2A02D0934238BF134680F87C
:108BC8000631012380F8073170470023F7E700BF1B
:108BD8000000C842666666404B68C0F8F430CB684F
:108BE8009FED087A07EE903A67EE877AFDEEE77A0E
:108BF80017EE903A5BBAA0F80C31012380F80E31D9
:108C0800704700BF0000C84270B58A68C2F31702F7
:108C18004A2A90B004460B4600F0F38040D8212A37
:108C280022D8172A06D8002A79D0012A00F0028112
:108C380010B070BD183A092AFAD801A151F822F0EB
:108C4800758D0008398C0008398C0008898E000859
:108C5800398C0008398C00085B8D0008398C0008B5
:108C6800398C0008238E00082A2A00F02F813E2A1A
:108C7800DED14D78192D01F10C0100F24B812A4605
:108C880001A80BF059F801ABC5F11A0200215819D7
:108C98000AF0EAFF01A904F58E70FEF740FCC7E769
:108CA800AD2A00F0558129D8932A45D01BD87C2AB3
:108CB80000F08480882ABBD14D78152D01F10C0174
:108CC80000F236812A4601A80BF036F801ABC5F14F
:108CD8001602002158190AF0C7FF01A904F58E7081
:108CE800FEF749FCA4E7A22AA2D101A8F9F732FAB3
:108CF80001A904F58E70FEF773FC99E7F22A00F0DB
:108D08003081FD2A00F05181E22A91D101A8F9F7BA
:108D18003BFA01A904F58E70FEF779FC88E701A8F3
:108D2800F9F718FA01A92046FFF746FC01A904F54E
:108D38008E70FEF779FB7BE701A8F9F7D3F901A953
:108D48002046FFF7A5FE01A904F58E70FEF720FC6A
:108D58006EE7194601A8F9F7E2F9204601A9FFF7DD
:108D6800CFFE04F58E70FEF79CFB61E75D78332D2E
:108D780003F10C0114D82A4601A80AF0DDFF01AB63
:108D8800C5F13402002158190AF06EFF9DF8213010
:108D980084F8F03001A904F58E70FEF767FB47E709
:108DA8000A4601AD3C33106851682E4603C60832A6
:108DB8009A423546F7D110683060E7E74D78382D8C
:108DC80001F10C010FD82A4601A80AF0B5FF01AB42
:108DD800C5F13902002158190AF046FF9DF82530DF
:108DE80084F8F13024E70A4601AD4433106851682D
:108DF8002E4603C608329A423546F7D113783370A7
:108E0800ECE701A8F9F753FA204601A9FFF7E4FEB9
:108E180004F58E70FEF790FB0AE7194601A8F9F7EA
:108E28007EF9204601A9FFF797FE04F58E70FEF73C
:108E380047FBFDE64D782A2D01F10C0110D82A4692
:108E480001A80AF079FF01ABC5F12B0200215819DE
:108E58000AF00AFF01A904F58E70FEF7F9FAE7E6B1
:108E68000A4601AD3433106851682E4603C60832ED
:108E78009A423546F7D111889378B3703180E9E783
:108E88005D781C2D03F10C0110D82A4601A80AF0C0
:108E980053FF01ABC5F11D02002158190AF0E4FE89
:108EA80001A904F58E70FEF7F0FAC1E60A4601AD95
:108EB8002433106851682E4603C608329A42354654
:108EC800F7D11068306013793371E9E74D78112DC7
:108ED80001F10C0110D82A4601A80AF02DFF01ABB8
:108EE800C5F11202002158190AF0BEFE01A904F5C5
:108EF8008E70FEF707FB9BE60A4601AD1C3310682F
:108F080051682E4603C608329A423546F7D113886F
:108F18003380EBE70A4601AD2433106851682E46CA
:108F280003C608329A423546F7D113883380B1E632
:108F38000A4601AD1C33106851682E4603C6083234
:108F48009A423546F7D1106830609388B380C4E6FA
:108F580001A8F9F719F901A904F58E70FEF74DFB80
:108F680066E64D783B2D01F10C0110D82A4601A880
:108F78000AF0E2FE01ABC5F13C02002158190AF0E3
:108F880073FE01A904F58E70FEF74BFB50E60A4606
:108F980001AD4433106851682E4603C608329A4220
:108FA8003546F7D110683060EBE701A8F9F79AF871
:108FB80001A904F58E70FEF745FB39E64A7922B11E
:108FC8008B79012B01D1FFF71FBE7047B0F5E16F18
:108FD80003DC10F5E16F04DB7047A0F5616000B2B7
:108FE800F4E700F5616000B2F3E70000B0F8F83389
:108FF8008A8810B5044613F0080008BFC4F80801B1
:1090080013F0020308BFC4F81831B2F5005F00F08E
:10901800C08007D86C2A18D06D2A00F09D806A2A73
:109028006ED010BD42F202039A4249D042F6FF7355
:109038009A42F6D1D4F8FC23896804F1BE00FEF701
:109048007BF9012384F8CE30EBE7B1F90A009FEDF4
:10905800557AFFF7BBFF07EE900AF8EEE77A67EE5E
:10906800877AFDEEE77A17EE903A5BBAA4F8E43017
:10907800B1F90800FFF7AAFF07EE900AF8EEE77AC1
:1090880067EE877A9FED487AFDEEE77A17EE903A19
:109098005BBAA4F8E630B1F90C00FFF797FF07EECA
:1090A800900AF8EEE77A67EE877AFDEEE77A17EE30
:1090B800903A5BBAA4F8E830012384F8EA30B0E7C4
:1090C800B1F809300A22B3FBF2F35BBAA4F8D43042
:1090D800B1F80B30B3FBF2F35BBAA4F8D630D1F891
:1090E800113084F8DA301A0C84F8D8201A0A84F877
:1090F800D9204B7F84F8DB30012384F8DC3090E7FB
:1091080000288ED0D1F80A301BBAC4F8F830D1F84C
:109118000E301BBAC4F8FC308B8A242253433233F6
:109128006422B3FBF2F35BBAA4F80031CB8A0A20BD
:1091380043435BBAA4F80231D4F8F43393FBF2F357
:1091480003F57A735BBAA4F804314B7A84F80631D4
:10915800012384F8073164E7B1F90C2052BAA4F866
:109168000C21012284F80E21002B3FF45AAFD1F8CC
:109178000E100A2391FBF3F303F51C53103383F30A
:109188000F035BBAA4F81431C4F8F41384F8072168
:1091980047E78B89A4F8F833D1F81130C4F8FC33C9
:1091A8003FE700BF58A08B416E882E4330B5204C56
:1091B80085B0054694F99200F7F73EFF00238DF835
:1091C80005308DF8073094F895308DF80830194B34
:1091D80094F893208DF8040098788DF80620F7F716
:1091E8001BFF8DF809001448FBF7C9F9F7F7EFFEE4
:1091F8008DF80A002046F7F75DFEF7F71DFF8DF89A
:109208000B002046F7F768FE8DF80C002046F7F7AC
:109218005AFE8DF80D002046F7F76FFE0A238DF8E9
:10922800050001AA14212846FFF7A1F905B030BDB1
:10923800CC300020CC0300207431002073B5184CCA
:1092480005462046F7F736FEF7F7F6FE8DF80000DC
:109258002046F7F72FFE06461248FBF779F9014634
:109268003046F7F7F3FE8DF801002046F7F734FE95
:109278008DF802002046F7F726FEFF238DF804300C
:10928800094B8DF803009878F7F7CEFE06238DF882
:1092980005006A461D212846FFF769F902B070BD2E
:1092A800CC30002074310020CC030020F7B5144DD9
:1092B800144E044695F99200F7F7BEFE8DF80000AB
:1092C800304695F99270FBF743F901463846F7F7AF
:1092D800BDFE95F893308DF801008DF802303046C8
:1092E80000238DF80330FBF74AF905238DF80400B5
:1092F8006A461C212046FFF73AF903B0F0BD00BFCB
:10930800CC3000207431002030B591B04EF6EA63BD
:109318001A49ADF80030044614220DF10200F8F79E
:1093280073F80DF10200F6F77DFFC3B2DA1CD0B274
:10933800694651FA82F26D250DF800504C205070A4
:10934800522090705320D070312010716FF02B0094
:1093580050710120507203200021907211330620B1
:109368009171D1711172D07211735173DBB26A4667
:1093780029212046FFF7FBF811B030BDF746010858
:109388000038024B18BF0120187070477C06002077
:109398002DE9F041002A4AD1042B00F2A1809EB2A7
:1093A800002B42D04D4C4FF0800EFF250F8894F8CB
:1093B8001EC0C35D23EA0C03C355A37F01325B08BB
:1093C8001FFA82FCA3773BB90B8801330B8084F822
:1093D8001EE00B88C554A37FB1F8008010F8087010
:1093E80027EA030300F80830A37F5B08A3773BB99B
:1093F8000B8801330B8084F81EE00B88C554A37FCB
:10940800B1F8008010F8087027EA030300F8083064
:10941800A37F5B08A37733B90B8801330B8084F8EB
:109428001EE00B88C5546645C0D8BDE8F081FF2A08
:10943800FBD1032B00F249819FB2002BF5D0274CBA
:1094480000258026B1F800C094F81EE010F80C3012
:1094580023EA0E0300F80C30A37F01355B081FFADE
:1094680085FCA37733B90B8801330B80A6770B886B
:10947800C254A37FB1F8008010F808E02EEA030375
:1094880000F80830A37F5B08A37733B90B88013352
:109498000B80A6770B88C254A37F5B08A37733B9E8
:1094A8000B8801330B80A6770B88C254A37FB1F8D1
:1094B800008010F808E02EEA030300F80830A37FC4
:1094C8005B08A3772BB90B8801330B80A6770B8831
:1094D800C2546745B6D8BDE8F08100BFAC0D002086
:1094E8000D889A4C425DA67F22EA06024255A27F69
:1094F800520803F5C063A2773AB90A8801320A8094
:109508008022A2770A88FF2585540D88A67F425DB0
:1095180022EA06024255A27F5208A2773AB90A887F
:1095280001320A808022A2770A88FF258554A27F0B
:109538005208A2773AB90A8801320A808022A277B3
:109548000A88FF258554A27F5208A2773AB90A886B
:1095580001320A808022A2770A88FF2585540D8867
:10956800A67F425D22EA06024255A27F5208A277F0
:109578003AB90A8801320A808022A2770A88FF2530
:1095880085541E0605D40D88A67F425D22EA060290
:109598004255A27F5208A2773AB90A8801320A8056
:1095A8008022A2770A88FF2585545D0605D40D8898
:1095B800A67F425D22EA06024255A27F5208A277A0
:1095C8003AB90A8801320A808022A2770A88FF25E0
:1095D80085549A0605D40D88A67F425D22EA0602C4
:1095E8004255A27F5208A2773AB90A8801320A8006
:1095F8008022A2770A88FF258554DF0605D40D88C6
:10960800A67F425D22EA06024255A27F5208A2774F
:109618003AB90A8801320A808022A2770A88FF258F
:1096280085541E0705D40D88A67F425D22EA0602EE
:109638004255A27F5208A2773AB90A8801320A80B5
:109648008022A2770A88FF2585545D0705D40D88F6
:10965800A67F425D22EA06024255A27F5208A277FF
:109668003AB90A8801320A808022A2770A88FF253F
:1096780085549A0705D40D88A67F425D22EA060222
:109688004255A27F5208A2773AB90A8801320A8065
:109698008022A2770A88FF258554DB0705D40A882B
:1096A800A57F835C23EA05038354A37F5B08A37724
:1096B800002B7FF4BAAE0B88802201330B80A2778F
:1096C8000B88FF22C254BDE8F0810E881F4C855DCF
:1096D800A77F25EA07058555A57F6D0803F5E06393
:1096E800A57735B90D8801350D808025A5770D88BA
:1096F80042550D88A67F425D22EA06024255A27FA6
:109708005208A2773AB90A8801320A808022A277E1
:109718000A88FF258554A27F5208A2773AB90A8899
:1097280001320A808022A2770A88FF258554A27F09
:109738005208A277002A7FF418AF0A8801320A80FB
:109748008022A2770A88FF2585540EE7AC0D0020F9
:109758002DE9F0479C4C802500270F80A577FF2531
:1097680005709846002B00F02C8103F1FF3912FA9E
:1097780089F9561EBA463B460BE0554540F0C08075
:109788000137BFB20A88424580F0B3804E4500F0E9
:10979800078116F8015F002BEFD16B1EDBB2FD2BA2
:1097A80000F2AA803F2B40F2E18005F14103DBB2D1
:1097B8003F2B00F2AC80A37F01355B08EDB2A377A5
:1097C800002B00F0E4805B08A37743B90B880133D2
:1097D8000B808023A3770B88FF22C254A37FAA069D
:1097E80008D4B1F800C010F80C2022EA030300F8EE
:1097F8000C30A37F5B08A37743B90B8801330B8038
:109808008023A3770B88FF22C254A37FEA0608D4DB
:10981800B1F800C010F80C2022EA030300F80C305D
:10982800A37F5B08A37743B90B8801330B808023A0
:10983800A3770B88FF22C254A37F2A0708D4B1F864
:1098480000C010F80C2022EA030300F80C30A37FB4
:109858005B08A37743B90B8801330B808023A37778
:109868000B88FF22C254A37F6A0708D4B1F800C04E
:1098780010F80C2022EA030300F80C30A37F5B08E1
:10988800A37743B90B8801330B808023A3770B8818
:10989800FF22C254A37FAA0708D4B1F800C010F869
:1098A8000C2022EA030300F80C30A37F5B08A3779F
:1098B80043B90B8801330B808023A3770B88FF22E1
:1098C800C254A37FEA0705D40D88425D22EA030348
:1098D8004355A37F5B08A377BBB90A8801320A8086
:1098E8008022A2770A88FF2585540A884245FFF41A
:1098F8004DAF0020BDE8F0870127AA463B4641E767
:10990800FBB25246FFF744FD47E700233AE70A88CF
:1099180094F81EC0835C23EA0C038354A37F3F356D
:109928005B08EDB2A37743B90B8801330B80802322
:10993800A3770B88FF22C254A37F5B08A37743B9A0
:109948000B8801330B808023A3770B88FF22C25436
:10995800A37F6A063FF537AFB1F800C010F80C20B6
:1099680022EA030300F80C30A37F2CE7A37F7F359E
:109978005B08EDB2A377002BEED10B8801330B8087
:109988008023A3770B88FF22C254A37FE4E70B88C8
:1099980001330B808023A3770B88FF22C254E3E7AF
:1099A8005BB9A37F802B1EBF013292B20A8090451B
:1099B80094BF00200120BDE8F087FBB25246FFF7B4
:1099C800E7FC0A88EDE700BFAC0D00202DE9F04F59
:1099D80047F26F730022827003800B78A3F1FE03B5
:1099E800B3FA83F35B0983708A780D4612F001019C
:1099F8001CBF43F080038370D5F8202122F07F42FA
:109A080022F0FF0285B0044612B143F008038370C8
:109A1800AA68C2F31702FF2A1ED9B2F5803F18D3ED
:109A280063F07F03A37041F002014FF0020B09239A
:109A38004FF00A0C0822E1700B20CDF804C01E4636
:109A480017464FF0070E4FF006094FF0050A04219C
:109A580017E043F00203A370180600F1D68008232C
:109A68004FF0090C07220A204FF0000BCDF804C074
:109A78001E4617464FF0060E4FF005094FF0040A30
:109A8800032195F8018004F8018004EB0108297985
:109A980004F80A10697904F80910A97904F80E1075
:109AA800A178090709D595F82111A15495F8221133
:109AB800A1550346674662460646A968A154A2789E
:109AC800900707D5BA1C1F46AB68C3F30F23A355ED
:109AD80096B23346BBF1000F05D05A1C1F46AB7A2D
:109AE800A35596B23346A278D10606D55A1C1F460E
:109AF80095F82331A35596B23346454A127803F1B7
:109B0800010914FA89FA05F10C0B42B16B785A462F
:109B18000DF10E015046FFF71BFE00285AD16A7856
:109B2800504659461FFA82FA0AF006F92278394B4C
:109B38006178D243D2B2072F9A5C82EA0102995C1B
:109B4800A27882EA0102995CE27882EA0102995CD1
:109B5800227982EA0102995C627982EA0102995CBF
:109B6800A27982EA0102995CE27982EA0102995CAF
:109B78001BD0227A5140082F595C16D0627A514086
:109B8800092F595C11D0A27A51400A2F595C0CD088
:109B9800E27A51400B2F595C07D0227B51400C2FA1
:109BA800595C1EBF627B5140595CA1551AFA89F372
:109BB8009BB2B5F80C21E2545A1CB5F80C1192B2BC
:109BC800090AA154AA78981CD20780B20BD405B010
:109BD800BDE8F08FA378BDF80EA043F04003A37052
:109BE80088F800A0A2E7D5F81071D5F81811D5F8B3
:109BF8001461275022180F335660916095F81C1194
:109C0800117398B205B0BDE8F08F4FF0000B0EE766
:109C18007C060020805901082DE9F04F8F4D0C4635
:109C280083B001460746284616460AF085F88C4A4E
:109C3800002380212380138482F82210002E00F054
:109C4800C58028784FF0400B4FEAD01C82F822B02C
:109C58009E464FF0FF0892F8229015F803A04FEAAD
:109C68004C001AEA090F4FEA590C18BF40F00100DE
:109C780082F822C0BCF1000F00F0AB80022800F08F
:109C88004484032800F0E083012840F0B2809E421B
:109C980040F29C8015F8039019EA0C0F14BF0120BC
:109CA80000205FEA5C0A40F0B88301339BB29E4211
:109CB800138482F8221040F2898015F903C0BCF1A0
:109CC800000F4FEA400001DA40F0010082F822B0AC
:109CD8004FF0400C9E4279D915F80390400019EADC
:109CE8000C0FC0B218BF40F001005FEA5C0A40F0F8
:109CF8002C8401339BB29E42138482F8221065D9CA
:109D080015F903C015F803904000BCF1000FC0B26C
:109D180001DA40F00100400019F0400F5FFA80FAC4
:109D280018BF4FF0200C00F0A3854AF0010ABCF1DF
:109D3800000F40F09F8501339BB29E42138482F846
:109D4800221043D915F9039015F803C04FEA4A00C9
:109D5800B9F1000FC0B201DA40F0010040001CF078
:109D6800400FC0B218BF4FF0200C00F0BC8540F087
:109D7800010082F822C0BCF1000F03D10133138423
:109D880082F822107D2821D84130238803F1010C64
:109D9800A4F800C0F854138C9E4217D992F82200F8
:109DA80015F803C010EA0C0F4FEA500014BF4FF02B
:109DB800010C4FF0000C82F8220020B901339BB24D
:109DC800138482F822109E423FF645AF03B0BDE8E7
:109DD800F08F01339BB20228138482F8221000F01E
:109DE800B481032800F03C8201284FF0800C3FF436
:109DF8004EAF9E42EAD9E85C1CEA000F1ED05FEA2B
:109E08005C092FD101339BB29E42138482F8221041
:109E1800DCD9E8560028C0F2F1804FF080094FEAFB
:109E2800590082F8220018B90133138482F82210ED
:109E38002388581C208007F80380ACE74FEA5C00B1
:109E480082F8220018B90133138482F8221023887B
:109E5800581C208007F803E09DE700BF800C002015
:109E6800AC0D002019EA000FD9D05FEA9C0C40F035
:109E7800C78001339BB29E42138482F82210A5D971
:109E8800E8560028C0F26E824FF0800C5FEA5C0052
:109E980040F0478201339BB29E42138482F822101D
:109EA80094D915F803C04FEADC101CF0400F4FEAB4
:109EB800400000F0BF844FF0200C40F0010082F811
:109EC80022C0BCF1000F06D101339BB2138482F883
:109ED80022104FF0800C9E427FF678AF15F8039061
:109EE80040001CEA090FC0B218BF40F001005FEA49
:109EF8005C0C40F0718301339BB29E42138482F85C
:109F080022107FF663AF15F903C04000BCF1000FC3
:109F1800C0B280F231844FF0800C5FEA5C0C40F0F4
:109F2800010040F0658301339BB29E42138482F89E
:109F380022107FF64BAF15F903C04000BCF1000FAB
:109F4800C0B280F225844FF0800C5FEA5C0C40F0D0
:109F5800010040F0598301339BB29E42138482F87A
:109F680022107FF633AF15F903C04000BCF1000F93
:109F7800C0B280F226844FF0800C5FEA5C0C40F09F
:109F8800010040F04D8301339BB29E42138482F856
:109F980022107FF61BAF15F903C04000BCF1000F7B
:109FA800C0B2C0F211844FF0400C15F80390400085
:109FB8001CEA090FC0B200F052834FEA5C0C40F073
:109FC800010082F822C0BCF1000F40F00484013384
:109FD8009BB2138482F822101FFA80FC00283FF4F9
:109FE800DBAE00232088013300F10109A4F80090BA
:109FF80007F800E098B26045F4D3CCE64FF0400C87
:10A00800E85C1CEA000F3FF441AF5FEA5C0C40F0EB
:10A01800AB8101339BB29E42138482F822107FF6F3
:10A02800D5AE15F803904FEAD91019F0400F4FEA52
:10A03800400000F0F4834FF0200C40F00100BCF128
:10A04800000F40F0EE8301339BB29E42138482F8E6
:10A0580022107FF6BBAE15F903C015F80390400037
:10A06800BCF1000FC0B201DA40F00100400019F065
:10A07800400FC0B218BF4FF0200C00F0298440F008
:10A088000100BCF1000F40F0258401339BB29E42D1
:10A09800138482F822107FF699AE15F903C04000A8
:10A0A800BCF1000FC0B201DA40F0010082F822B022
:10A0B8004FF0400A9E427FF689AE15F803C0400073
:10A0C8001AEA0C0FC0B218BF40F001005FEA5A0C40
:10A0D80040F0D48201339BB29E42138482F822104E
:10A0E8007FF674AE15F903C04000BCF1000FC0B292
:10A0F800C0F274834FF0400C15F8039040001CEA3E
:10A10800090FC0B200F0D9824FEA5C0C40F00100A0
:10A1180082F822C0BCF1000F40F0678301339BB284
:10A12800138482F822101FFA80FC00283FF434AE12
:10A1380000232088013300F10109A4F8009007F8F2
:10A14800008098B28445F4D825E69E427FF63EAE5C
:10A15800E85C4FF04009C009B2F820C0430015F888
:10A168000C0019EA000F4FEA590A01D043F0010325
:10A17800BAF1000F40F0B0820CF1010C1FFA8CFC10
:10A188006645A2F820C082F822107FF61FAE15F9A6
:10A198000C905800B9F1000FC0B280F2DB82402366
:10A1A80040F00100002B40F0A4820CF1010C1FFAD2
:10A1B8008CFC6645A2F820C082F822107FF606AE15
:10A1C80015F90C304FEA4009002B5FFA89F980F243
:10A1D800CA82402049F00109002840F099820CF118
:10A1E800010C1FFA8CFC6645A2F820C082F82210E8
:10A1F8007FF6ECAD15F90C004FEA49030028DBB2F5
:10A2080080F2BD824FF0400943F00103B9F1000F1D
:10A2180040F08D820CF1010C1FFA8CFC6645A2F807
:10A2280020C082F822107FF6D1AD15F90C005B0032
:10A238000028DBB280F2C282402043F0010382F89A
:10A24800220028B90CF1010CA2F820C082F82210D3
:10A258002088013300F1010CA4F800C03B549AE5B2
:10A268009E427FF6B3AD15F803A04FF040094FEAC0
:10A27800DA101AEA090F4FEA40004FEA590C01D0E8
:10A2880040F00100BCF1000F40F0338301339BB272
:10A298009E42138482F822107FF698AD15F903C008
:10A2A80015F803A04000BCF1000FC0B201DA40F07D
:10A2B800010040001AF0400FC0B218BF4FF0200C48
:10A2C80000F0EE8240F00100BCF1000F40F0EA829D
:10A2D80001339BB29E42138482F822107FF676AD3A
:10A2E80015F9039015F803C04000B9F1000FC0B28A
:10A2F80001DA40F0010040001CF0400FC0B218BF66
:10A308004FF0200C00F0D78240F0010082F822C004
:10A31800BCF1000F03D10133138482F822104138B5
:10A3280033E515F8039019EA000F14BF0120002047
:10A338005FEA9C0A40F0388201339BB29E42138444
:10A3480082F822107FF642AD15F903C0BCF1000F68
:10A358004FEA400001DA40F0010082F822B04FF0E5
:10A36800400CB8E54FF0400C15F8039019EA0C0FB3
:10A3780014BF012000205FEA5C0A40F00C82013320
:10A388009BB29E42138482F822107FF61FAD15F906
:10A3980003C015F80390BCF1000F4FEA400001DA42
:10A3A80040F00100400019F0400FC0B218BF4FF054
:10A3B800200A00F0478240F00100BAF1000F40F097
:10A3C800438201339BB29E42138482F822107FF6A7
:10A3D800FDAC15F9039015F803C04000B9F1000F62
:10A3E800C0B201DA40F0010040001CF0400FC0B2DA
:10A3F80018BF4FF0200A00F0638240F0010082F895
:10A4080022A0BAF1000F7FF455AE01339BB213843A
:10A4180082F822104FF0800A4CE619EA0A0F4FEA38
:10A428009C0C4FEA400001D040F0010082F822C0A5
:10A43800BCF1000F7FF44EAC01339BB2138482F859
:10A4480022104FF0800C45E415F803A01AEA0C0F0F
:10A4580014BF012000205FEA99097FF40AAF013395
:10A468009BB29E42138482F822107FF6AFAC15F996
:10A4780003C015F803A0BCF1000F4FEA400001DA51
:10A4880040F001001AF0400F4FEA400018BF4FF0AB
:10A49800200900F0B98140F00100B9F1000F40F047
:10A4A800B58101339BB29E42138482F822107FF655
:10A4B8008DAC15F903C015F803A04000BCF1000FDE
:10A4C800C0B201DA40F0010040001AF0400FC0B2FB
:10A4D80018BF4FF0200900F0C08140F00100B9F129
:10A4E800000F40F0BC8101339BB29E42138482F876
:10A4F80022107FF66BACEB564000002BC0B201DA9D
:10A5080040F0010082F822B009E792F8229019EA97
:10A518000A0F14BF012000205FEA59097FF41CAE1E
:10A5280001331FFA83FC6645A2F820C082F8221086
:10A538007FF64CAC15F90C90B9F1000F4FEA4003C7
:10A5480080F200814FF0400A10E64000C0B200904F
:10A5580019EA0A0F4FEA9C00019003D0009840F0D6
:10A56800010000900198002840F0CC8101339BB293
:10A578009E42138482F822107FF628AC009815F9C1
:10A5880003C015F803904000BCF1000FC0B201DA17
:10A5980040F00100400019F0400FC0B218BF4FF062
:10A5A800200A00F0718140F00100BAF1000F40F07C
:10A5B8006D8101339BB29E42138482F822107FF68C
:10A5C80005ACEB564000002BC0B201DA40F00100A8
:10A5D80082F822B0FFF7D6BB15F8039040001CEABA
:10A5E800090FC0B27FF499AC5FEA5C0C3FF49BACF6
:10A5F80015F8039040001CEA090FC0B27FF4A5AC1F
:10A608005FEA5C0C3FF4A7AC15F8039040001CEA25
:10A61800090FC0B27FF4B1AC5FEA5C0C3FF4B3AC95
:10A6280015F8039040001CEA090FC0B201D040F0B1
:10A6380001005FEA5C0C7FF4B8AC01339BB29E4228
:10A64800138482F822107FF6C1AB15F903C04000CD
:10A65800BCF1000FC0B2C0F2BA804FF0800C4FEAD4
:10A668005C0C82F822C0BCF1000F3FF4B0AC1FFABA
:10A6780080FC00287FF4B5ACFFF790BB15F8039079
:10A6880040001CEA090FC0B201D040F001005FEAA7
:10A698005C0C7FF431AD01339BB29E42138482F887
:10A6A80022107FF693AB15F903C04000BCF1000FF0
:10A6B800C0B2C0F296804FF0800C4FEA5C0C82F872
:10A6C80022C0BCF1000F3FF429AD1FFA80FC00281E
:10A6D8007FF42EADFFF762BB15F80C9058001AEA0C
:10A6E800090FC0B24FEA5A037FF45AAD002B3FF46A
:10A6F8005CAD15F80CA04FEA400913EA0A0F5FFA9F
:10A7080089F94FEA53007FF465AD00283FF467AD3F
:10A7180015F80CA04FEA490310EA0A0FDBB24FEA1A
:10A7280050097FF471ADB9F1000F3FF473AD15F81E
:10A738000CA05B0019EA0A0FDBB24FEA59003FF49C
:10A748007EAD7AE515F80C305B064FEA80004FD5F0
:10A75800202325E59B005FFA83F915F80C3058068D
:10A7680048D5202036E58000C3B215F80C00400615
:10A7780042D54FF0200947E54FF0400C38E715F86F
:10A788000C004FEA89034006DBB238D5202054E597
:10A798004FF0400C38E719EA0A0F4FEA9C0C4FEAD1
:10A7A80040003FF44CAC48E419EA0A0F4FEADC0CCD
:10A7B8004FEA40003FF483ABFFF77FBB82F822B03B
:10A7C80046E54FF0400C2BE74FF0800C2FE740F0A8
:10A7D800010082F822B01FFA80FC02E44FF0800CDE
:10A7E80053E740F0010082F822B01FFA80FC9FE492
:10A7F80020237EE720208BE74FF0200997E74FF0D2
:10A80800200082F8220023E54FF02009400019EAD1
:10A818000A0FC0B24FEA590C3FF456AD52E54FF05B
:10A82800200C400019EA0C0FC0B24FEA5C0A3FF452
:10A83800C4ADC0E54FF0200C82F822C04FF0200CC8
:10A84800FFF749BB4FF0200A400019EA0A0FC0B2CF
:10A858004FEA5A0C3FF415AC11E44FF020094000C0
:10A8680019EA0A0FC0B24FEA590C3FF44FAD4BE555
:10A878004FF0200C4FEA4A001CEA090FC0B24FEA19
:10A888005C0A3FF492AE8EE64FF0200A400019EAC7
:10A898000A0FC0B24FEA5A0C3FF46BAAFFF767BA27
:10A8A8004FF0200C40001CEA0A0FC0B24FEA5C09C6
:10A8B8003FF415AE11E64FF0200382F822302EE562
:10A8C8004FF0200C82F822C04FF0200AFFF7F2BBAD
:10A8D8004FF0200C400019EA0C0FC0B24FEA5C0A96
:10A8E8003FF48DAD89E54FF0200382F82230FFF761
:10A8F80049BA40001CEA0A0F4FEA9909C0B23FF46E
:10A90800CCADC8E5009840005FFA80FA019819EAD2
:10A91800000F4FEADC0C3FF40AAAFFF706BA00BFA3
:10A928002DE9F04F5788B7F58F7F8BB01446064650
:10A938000BD90022227000226F2B628000F0658103
:10A94800002333700BB0BDE8F08F12780E2A0D4645
:10A9580024D80E2A00F2118101A151F822F000BF7B
:10A968003FA900088FAB000883AB000883AB000841
:10A978008FAB00088FAB00088FAB00088FAB0008C7
:10A988008FAB00088FAB0008DDAB000883AB000875
:10A9980083AB000883AB000801AC0008692A40F2C9
:10A9A800EA806A2A40F0E9809C4FFA8A02F1FF3C6B
:10A9B8001FFA8CFC002A00F077820CF1030CDFF8F8
:10A9C80064E2BC44FF22B91C11F8010B4240614506
:10A9D8001EF80220F8D1934200F0CF8100222270A5
:10A9E800C4F80220E280FA8A022AA9D939796F29A3
:10A9F80000F02B83032AA3D079796F2900F03583DF
:10AA0800042A9DD0B9796F2900F03283052A97D09E
:10AA1800F9796F2900F03B83062A91D0397A6F299A
:10AA280000F04482072A8BD0797A6F2900F03283AC
:10AA3800082A85D0B97A6F2900F02F83092A3FF4B4
:10AA48007FAFF97A6F2900F02B830A2A3FF478AF99
:10AA5800397B6F2900F027830B2A3FF471AF797B8C
:10AA68006F2900F023830C2A3FF46AAFB97B6F2962
:10AA780000F01F830D2A3FF463AFF97B6F2900F0C4
:10AA88001B830E2A3FF45CAF397C6F2900F01A83D0
:10AA98000F2A3FF455AF797C6F2900F01083102AF4
:10AAA8003FF44EAFB97C6F2900F00F83112A3FF4B1
:10AAB80047AFF97C6F2900F00B83122A3FF440AFAF
:10AAC800397D6F2908BF4FF012087FF439AF02F1C2
:10AAD80001091FFA89F93A44A7F816905FFA89F92B
:10AAE80093704F494A4602A809F026F96F234FF0A0
:10AAF800010CBB704FF0000E6423A7F800E0A7F824
:10AB080016C0237008EB0C0399451FFA89F27FF6EB
:10AB180017AF901E02A9A0EB08005A1E0B440A4466
:10AB280013FA80F04FF06A084FF007094FF0660AF1
:10AB380005E0002B40F0BD8190423FF401AFFB8A55
:10AB480012F8011F07EB030B01338BF80210FB828D
:10AB58002378092BEDD9A3F1640BBBF1050FEBD8D2
:10AB6800653B042B00F2B782DFE813F01E011601E3
:10AB780011010D011A01632A05D800232370C4F8B6
:10AB88000230E380DDE6254FFA8AB91801328B706E
:10AB9800FA822278092A00F2A480002A3FF4D0AE73
:10ABA800013A082A3FF6CCAE01A151F822F000BFC5
:10ABB80077AE000849A9000849A90008D9AD0008DE
:10ABC800D9AD000861AE00082DAE00089BAE0008A4
:10ABD8004BAE00087A1C6280104EEB55A088727F3D
:10ABE800618883189942FFF6ADAE33785F0600F1AD
:10ABF800E1810E232370A5E67A1C6280EB55E2887A
:10AC08006388934210D201239BE604490A800122FB
:10AC1800CA8264228B702270002392E6AC0D002059
:10AC2800AE0D0020805901080023638023700223A1
:10AC3800037042802B78FD2B00F08680EB7803723E
:10AC48002B7943726B7943606A78083272800022EC
:10AC58004FF4BC70DFF8B0C47281F62104460134A9
:10AC680099424FEA54042ED849D38B4240F0898048
:10AC78002B78FD2B7ED04FF0060B2846DFF8888412
:10AC880010F801AF0BEB0A0909F1FF3189B2F7F7A8
:10AC98009FF804EB440708EB8707ADF808003979FB
:10ACA800019102A8F7F76EF805EB090215F80930CB
:10ACB8005278019903EB0223BDF808209BB29A420F
:10ACC8001FD005233DE6601E1418824204F10107D7
:10ACD80080F0698127F0010101EB57015CF8211030
:10ACE800BDE7A2F1640105293FF62AAE653A042AB8
:10ACF80000F2FA81DFE802F0807C78749200224644
:10AD0800E2E7BB79DA0706D5FA79924582BF52198C
:10AD180012F80B20B2729B070BD56300234408EB93
:10AD280083036A781B7A9A4282BF5B1913F80B3047
:10AD3800F3726300234408EB8308317398F80530F5
:10AD480073730BB0BDE8F08F6B790372AB79437204
:10AD58006B7A297AEA791B0403EB012313444360D5
:10AD68006A7802F10C014180A978C9077FF56FAFB5
:10AD780019326BE74FF00A0B7FE70A220123227092
:10AD8800DFE50323DDE5F97684F80090D4E64FF09B
:10AD98006803B9762370CFE6797084F800C0CBE6F3
:10ADA800397784F80080C7E6397001F001036188BB
:10ADB80087F801E0033B01F1010BA4F802B06B54E2
:10ADC80097F90030002BACBF634653462370B3E6B7
:10ADD8006288511C6180AB54237801332370AFE53E
:10ADE8000722FB76227017E76822BB76227013E7EA
:10ADF80001227B7022700FE762883B70002103F00C
:10AE08000103033B7970511C6180AB5497F9003002
:10AE1800002BC0F230810123237091E56A223B7731
:10AE28002270F9E66288511C6180AB543B787A78CD
:10AE3800134313F0020340F0D5806288511C6180EF
:10AE4800AB546288511C6180AB543B78D8064CBF28
:10AE580069236A23237073E56288511C6180AB54AF
:10AE68003B781D074CBF67230723237068E562887A
:10AE78003A83511C6180AB543A787B7712F0010217
:10AE880000F0CE8006220833A280E38004232370DA
:10AE980056E56288511C6180AB547B7813F002033D
:10AEA800CFD0092323704BE5FF2294E54FF0060825
:10AEB8000DE6013B082B3FF63FAE0FF2080B5BF89F
:10AEC80023F000BF05AF000841AB000841AB000804
:10AED800F1AE0008F1AE000879AF000847AF0008EE
:10AEE80093AF00082BAF0008638803F1010BA4F8A7
:10AEF80002B0E9542378013323701DE663883B834D
:10AF080003F1010BA4F802B0E9543B78797713F008
:10AF180001036AD008310623E180A380042323704B
:10AF28000AE6638803F1010BA4F802B0E9543B7800
:10AF3800DB067FF536AF4FF069032370FCE56388C5
:10AF480003F1010BA4F802B0E9543B7879780B437C
:10AF580013F0020343D1618801F1010BA4F802B098
:10AF68006B54618801F1010BA4F802B06B54DEE761
:10AF7800638803F1010BA4F802B0E9543B78190780
:10AF88007FF502AF67232370D6E5638803F1010BD1
:10AF9800A4F802B0E9547B7813F00203E1D04FF033
:10AFA80009032370C8E5584902EB4200144651F8DA
:10AFB80020105AE602A92844FEF72EFE737FBDF83A
:10AFC80008106288CB1A9BB21A446280727F1A44B6
:10AFD8007277E2881344E380338BE95409E6082347
:10AFE8002370A9E508232370AAE40C31E18079785D
:10AFF8004FF00A0B11F00101A4F804B028D06188C1
:10B0080001F1010BA4F802B005F801C0618801F153
:10B01800010BA4F802B06B54E3880D33E3807DE79D
:10B0280079780C33E38011F001014FF00A03A38013
:10B0380024D06388012158186080E954638859181E
:10B048006180EA54E3880D331FE74FF002083EE5BC
:10B05800638803F1010BA4F802B0E954638803F193
:10B06800010BA4F802B0E95458E74FF003082EE5A5
:10B078004FF004082BE56623237061E463885A1CAB
:10B088006280E95463885A1C6280E954FEE64FF0F6
:10B0980005081CE54FF0070819E54FF0080816E504
:10B0A8004FF0090813E54FF00A0810E54FF00B08B8
:10B0B8000DE54FF00C080AE54FF00D0807E54FF0D5
:10B0C8000F0804E54FF00E0801E54FF01008FEE404
:10B0D8004FF01108FBE477290ED084F800E0C4F89B
:10B0E80002E0A4F806E027E5772B09D000232370B7
:10B0F800C4F80230E38023E44FF0650323701BE5B6
:10B10800652323701CE400BF805A010837B500F599
:10B11800EF65044600F5CA612846F6F794FF024633
:10B12800A0680192036829461B699847E06838B10E
:10B138000368019A1B69294603B0BDE830401847E7
:10B1480003B030BD08B583684BB1B0F84C14B0F803
:10B158004A04F7F771FA003818BF012008BD1846ED
:10B16800FCE70346806880B1B3F84C24B3F84A146E
:10B17800914209D09918013291F85004B3F84E144D
:10B188000A40A3F84C24704700207047836810B524
:10B1980004467BB10023A0F84C34A0F84A34C068B8
:10B1A80010B10368DB699847A0680368BDE81040E0
:10B1B800DB69184710BD0000F8B5224F0446384631
:10B1C800F5F778FEF5F7D0FE064697F99200F5F701
:10B1D800CBFE05463846F5F776FE642384F86236DA
:10B1E800FF2384F86436332384F85536442384F8DF
:10B1F8005636D4F8583684F860666D2262F3170321
:10B20800C4F85836C0F10A000023C4F85C3684F844
:10B21800713700B24FF43943A4F8723780F307004E
:10B22800092384F8630684F8615604F5CA6084F833
:10B23800743704F5A471F7F779FA2046BDE8F840A9
:10B24800FFF764BFCC30002010B5332380F85536A3
:10B25800442380F85636D0F85836144AC0F8602689
:10B268006FF31703C0F85836002380F85C3680F86F
:10B278005D3680F85E3680F85F3680F871374FF4B7
:10B288004853A0F8723703220923044680F864263D
:10B2980080F8743700F5A47100F5CA60F7F746FA2C
:10B2A8002046BDE81040FFF731BF00BF000880040A
:10B2B80070B586B004460021102202A8019108F05A
:10B2C800D3FC01AB03CB01ABC4F88006C4F88416E9
:10B2D80003CB01ABC4F88806C4F88C1603CB04F57D
:10B2E800D362C4F89006C4F8941601AB05AE1D46A7
:10B2F80003CDB542106051602B4602F10802F6D129
:10B308002B881380332384F85536442384F8563623
:10B31800D4F85836942262F3170310214222C4F855
:10B32800583684F85C16002384F86C2620212822DD
:10B3380084F85D1684F85E3684F85F3684F86036E3
:10B3480084F8613684F8623684F8633684F86436A3
:10B3580084F8653684F8663684F8673684F8683683
:10B3680084F8693684F86A3684F86B3684F86D2672
:10B3780084F86E3684F86F3684F8703684F871363F
:10B3880084F8723684F8733684F8743684F875361F
:10B3980084F8763684F8773684F8783684F87936FF
:10B3A80084F87A3684F87B3684F871374FF4324360
:10B3B800094AA4F872374E2304F5CA60C4F87C26FB
:10B3C80084F8743704F5A471F7F7B0F9204606B08D
:10B3D800BDE87040FFF79ABED016CB0F10B50446F3
:10B3E8009DF8080084F85E26002284F85F2684F819
:10B3F800602684F8612684F8622684F8632633225E
:10B4080084F85526442284F85626D4F85826A4F8F9
:10B418005C1684F8643684F871374D218F2361F304
:10B42800170284F873370A2384F8650684F87207CC
:10B43800C4F8582604F5CA6084F8743704F5A47172
:10B44800F7F774F92046BDE81040FFF75FBE00002B
:10B45800F0B502298DB004460D461CD1404B414839
:10B468001B7800EB031000F58970F5F755FE3E4B8D
:10B4780018603E4A0C236B43D718D3583A790021F9
:10B488000391511E082908D8DFE801F009095F5F18
:10B498006363070766002D29EBD90DB0F0BD1B7853
:10B4A8008DF80C308DF82C200021102207A8039E5F
:10B4B80008F0DAFBB96801910846F4F7B3FEC2B2A6
:10B4C800102A28BF1022019907A808F035FC2E225F
:10B4D8009DF82C3084F860260022C4F85C66A4F835
:10B4E800625684F8743684F8612607AB04F2646502
:10B4F8000BAE1A4603CAB24228606960134605F1CA
:10B508000805F6D1332384F85536442384F8563693
:10B51800D4F85836162262F31703C4F858360023B5
:10B5280084F871374FF45C43A4F87237192304F593
:10B53800CA6084F8743704F5A471F7F7F7F8204661
:10B548000DB0BDE8F040FFF7E1BD1B88ADF80C3049
:10B55800A8E71B680393A5E71B680393A2E700BF4E
:10B56800CC03002028040020E80600200800002062
:10B578002DE9F041884D894F2A780B46142101FBAB
:10B58800027288B092F85520012A044613D193F824
:10B59800212132B1332A0ED193F822210AB1442A4B
:10B5A80009D19A68C2F31702172A58D006D8142A64
:10B5B80031D0152A47D008B0BDE8F08102F1807279
:10B5C8004B3A22F07F42012AF5D8D3F8202174495A
:10B5D80022F07F4222F0FF028A42ECD1198DDA680C
:10B5E80040F20720814200F0D180B1F5027F00F0DF
:10B5F800BF80B1F5007F0CD107EE902AFCEEE77A08
:10B6080017EE902A942A00F0B380B2F5967F00F0E6
:10B61800BD800222B3E002A81946F6F748FEBDF93C
:10B628000800002804DA03A8F6F7BEFF0028C2DBEA
:10B638002D28C0DCA4F8BA08B4F8B03843F01003D9
:10B64800A4F8B038B7E7012384F8B8380023A4F881
:10B65800BA38544B1B68643BC4F8BC38ABE7D3F822
:10B6680020214F4922F07F4222F0FF028A42A2D1D4
:10B678005E78162E03F10C012DD8324602A808F088
:10B688005BFB02ABC6F117020021981908F0ECFA2F
:10B698000DF10E00F6F788FFB0F100088BDB424A87
:10B6A8009DF81E1008EB4803980002EB83031B79F2
:10B6B800994280D1B8F12D0F1FFA88F622DC0139A2
:10B6C800029B125808291DD8DFE801F01B1B3939E5
:10B6D8003B3B1C1C3D000A4602AE1C3310685168F7
:10B6E800B446ACE8030008329A426646F6D11068C0
:10B6F800CCF80000918893798CF80630ACF80410E7
:10B70800C6E713702878F8F75FF92A78142303FB43
:10B718000273012183F8551097F82D300BB987F87B
:10B728002D10B8F1020F10D1204B07EB0210196849
:10B7380000F58970F5F72AFDA4F8BA687CE713804C
:10B74800E0E71360DEE71360DCE7B8F1000FF3D140
:10B75800174B1A78002AEFD083F8008060232380E3
:10B76800104B1B680BB16360E6E74FF0FF33FAE755
:10B77800B4F8B02842F00202A4F8B0280022987960
:10B7880000905B792046FFF729FE14E7B4F8B0284B
:10B7980042F00402F0E700BFCC0300202804002098
:10B7A80000334400984A002008000020E8060020E2
:10B7B8008A2F002010B52F4B1A782F4B142101FB2C
:10B7C8000233044693F85530012B37D12B4BD0F870
:10B7D800B4281B689A1AB2F57A7F21BFB0F8B0284E
:10B7E800C0F8B43842F00102A0F8B02890F8B828A0
:10B7F80062B1D0F8BC289A1A312A81BFB0F8B028B3
:10B80800C0F8BC3842F01003A0F8B038B4F8B0382B
:10B81800DA0614D523F01003A4F8B038B4F8BA182F
:10B828002046FFF715FEB4F8BA3801339BB22D2B2A
:10B83800A4F8BA3802D9002384F8B83810BD98079C
:10B8480008D523F00203A4F8B0382046BDE810401C
:10B85800FFF72EBD590702D523F00403F3E7DA07F3
:10B86800ECD523F00103A4F8B0382046BDE8104019
:10B87800FFF7EABCCC03002028040020984A0020E7
:10B8880038B5134B134A1B68C0F8B438002380F846
:10B89800B838A0F8BA38C0F8BC38A0F8B038137077
:10B8A8000D4B0E481B780E4D00EB031000F5897008
:10B8B800F5F732FC0B4B02241860E0B2F9F7FAFCFA
:10B8C80001342C2C286305F10C05F6D138BD00BFD6
:10B8D800984A00208A2F0020CC030020280400204A
:10B8E80008000020E806002000230370FF234370AF
:10B8F8008370C37003717047F8B53A4D04462E78CB
:10B908003948142707FB060090F84F60012E0CD029
:10B91800022E0CD076B9A16090F84C30032B18BFDA
:10B928000022A368E26033B9FEE7A360F4E7A260EF
:10B938000022F6E7FEE70023C4E90433C4E95233E2
:10B94800C4E95433A3617F23A4F85831F6F734FCD3
:10B95800A878022844D0431F58425841234940F24E
:10B96800FF12FDF70DFD0220A4F84E24204A0870AE
:10B97800002348708870C8701E4913705370937004
:10B98800D370C4F8DA31C4F8DE31C4F8E231C4F84F
:10B998001233C4F81633C4F81A33A4F84C34A4F894
:10B9A8004A341A4601330C2B0A70CA704A708A70DE
:10B9B80001F10401F6D1104B1B6803F57A7304F604
:10B9C800A800C4F8A438FFF78FFF84F8AD2884F8DE
:10B9D800AE28228062602046BDE8F840FFF750BFDD
:10B9E8000120BBE7CC03002028040020B10600207A
:10B9F8007D06002081060020984A00204378FF2B0E
:10BA080005D0012B03D18278012A08BF02231846EA
:10BA18007047007840B14B79834204D18879431E3E
:10BA28005842584170470020704710B54B79037051
:10BA38009379DB0943705379032B044607D11079B6
:10BA4800FCF738FBE0701368DBB2237110BDFF23ED
:10BA5800C370FAE77FB58B6833F07F4305460C4621
:10BA680000F6A8060ED18B79012B0BD101A8F6F7A9
:10BA780071FB9DF80930082B04D001AA21463046F5
:10BA8800FFF7D3FF21463046FFF7C3FF78B3A3681B
:10BA9800C3F31703F52B16D16678012E29D8324641
:10BAA80004F10C0101A808F047F901ABC6F1020244
:10BAB8000021981908F0D8F89DF805309A1E5342CD
:10BAC800534185F8AA3895F8AD3853B195F8AE3892
:10BAD80021790A480133DBB2CB1A59425941F5F7AB
:10BAE80009FA012385F8AD38237985F8AE3804B012
:10BAF80070BDA389ADF80430DEE700BFCC3000206C
:10BB08007FB52E4E044600F11C05B4F85411B4F864
:10BB18005621881A83B2000444BF80339BB20BB904
:10BB280004B070BD91421FBFB4F85811A318013278
:10BB38000A4096F82D101ABF93F85A31A4F85621E6
:10BB48000023022904F110022946684620D1FEF795
:10BB5800E7FE9DF80030022BD7D1E368DBB9A06877
:10BB68000368BDF802201B692946984704F5CA6690
:10BB78002A4669463046F6F72DFB31461048FDF750
:10BB88001DFA3146204604B0BDE87040FFF762BF99
:10BB9800F6F7BEFBDDE70B4E69460020F6F778FDA9
:10BBA800737833B1A068BDF80220036829461B6981
:10BBB8009847B378002BD9D0E068D1E72804002053
:10BBC800940700207D0600200148FFF717BF00BF3B
:10BBD800C816002070B5594C594E86B0002116225F
:10BBE800684608F041F82046F5F776F994F88C3065
:10BBF8008DF800008DF80130204694F88D308DF8CE
:10BC08000230F5F760F994F8913094F890208DF8A7
:10BC180003005B0002F0010203F00203134394F8EF
:10BC2800A52043EA821394F8A62043EAC2139DF89C
:10BC38000B2002F03C02134320468DF80B30F5F739
:10BC480039F905463046F8F783FC01462846F5F7EA
:10BC5800FDF994F893308DF8073094F8943094F8FF
:10BC680095208DF8083094F8963094F992508DF814
:10BC78000400DB00920002F0040203F008031343FF
:10BC88009DF80B208DF8095022F00C021343304622
:10BC98008DF80B30F8F75CFC01462846F5F7D6F925
:10BCA8008DF80A0004F12800F5F7FDFC8DF80C006A
:10BCB8002046F5F7DDF88DF80D0004F11400F5F7CE
:10BCC800F2FC8DF80E0004F13C00F5F7ECFC8DF861
:10BCD8000F002046F5F7DDF88DF810002046F5F73F
:10BCE8000CF994F8A7308DF81230164B8DF8110026
:10BCF800DB7D8DF81330FFF767FF134B1A78931E1F
:10BD08005A425A4100F0030343EA02230F4A1048FB
:10BD1800127943EA4223BDF8142023F0FC039B0563
:10BD280022F4407222F003029B0D134302216A465B
:10BD3800ADF81430FAF7FFFF06B070BDCC30002024
:10BD480074310020A00B00208D070020C0060020C1
:10BD5800E016002070B54C88B4F5427F4FF0000320
:10BD68000AD80D780B2D73D8DFE805F0060D1A2ACE
:10BD78002D30363952555969A2F1240462424B805C
:10BD880062410A7007E04D2A01D0582A06D1027094
:10BD980002230B70002380F8093333E00023F8E70F
:10BDA80002F0FD033C2B01D0212AF7D10378427021
:10BDB8004D2B0CBF082303230B7000238370E9E786
:10BDC80082700422DDE782800522DAE7838803EBAC
:10BDD800022383800623DCE7C2800722D1E7C388D9
:10BDE80003EB02239BB2002BC3800CBF0B230A2357
:10BDF8000B7000234B80012380F80933C388B3F507
:10BE0800407F01D8002002E000200870488070BD03
:10BE1800C2800922B5E70A2382800B70EBE7B4F5EC
:10BE2800407F3CBF241822724B8801339BB24B8061
:10BE3800C2889A429CBF0B230B700123ABE780F8A2
:10BE480008230B704B80022380F809330120DEE7BA
:10BE58000B704B80D6E7CB88B3F5407F70B531D8EF
:10BE6800242303700B7843704B7883700B784D2B29
:10BE780014D1CB88C3708B88037105230022CD8829
:10BE8800D4189542A6B210FA84F415D891F808236C
:10BE98002270CA880132981880B270BD8B78C3703E
:10BEA8008B8803718B881B0A4371CB888371CB887D
:10BEB8001B0AC3710823E1E78C180132247A8455E0
:10BEC80092B2DCE70020E8E72DE9F74F16464A88EA
:10BED800B2F5427F04460D462ED80B780A2B0FD9AF
:10BEE800A3F16402032A03D90020287068802DE09A
:10BEF800653B8F4F022B33D8DFE803F063A4A7001C
:10BF080000210A2BF0D801A050F823F041BF000807
:10BF18005BBF0008F1BE0008F1BE00089FBF000823
:10BF2800ADBF0008B9BF0008BFBF0008F1BE0008D8
:10BF3800F1BE00082DC00008A6F124077E424FF08C
:10BF480000007E4168802E7084F8090303B0BDE8C4
:10BF5800F08F6F2E0CBF642300232B700020F3E7B3
:10BF680016F0040F14BF4D2358233E7023703A78FF
:10BF7800D1070ED412F0020F14BF21233E236370A1
:10BF8800C2F3C003D20648BF43F00203A3700423E0
:10BF9800E3E73C23F3E7A68005232B7084F8091315
:10BFA8000020D3E7A38803EB0623A3800623D4E766
:10BFB800E6800723F1E7E38803EB0623E3806523A4
:10BFC800CBE70DF106007E70F6F710F83978F6F732
:10BFD80005F8A7882179F6F701F8390AF5F7FEFF81
:10BFE800E788A179F5F7FAFF390AF5F7F7FF9DF821
:10BFF8000630B34206D000232B706B80032384F8ED
:10C008000933CDE7002F0CBF66230A232B700123C9
:10C0180084F8093300236B80E288B2F5407FBFD9EA
:10C028002B70BDE7B2F5407F3CBF121916726B88C2
:10C0380001339BB26B80E2889A4201D866232B7049
:10C048000123DCE77E806723F9E7B7F8028097F8D9
:10C05800009008EB06284FF6FF730DF106001FFA53
:10C0680088F84946ADF80630A7F80280F5F78AFE49
:10C078002679B4F804A03146F5F784FE4FEA1A2170
:10C08800F5F780FE94F806B0B4F806A05946F5F71F
:10C0980079FE4FEA1A21F5F775FE797804F1080759
:10C0A800F5F770FE52463946F5F778FEBDF80630CA
:10C0B80043453AD119F0040015D086EA0B01E21D78
:10C0C800002398B2824584F8081307D80223012078
:10C0D80000222A706A8084F8093337E712F8010FC2
:10C0E80001334140EDE7A178F4F7CAFF217984F8DC
:10C0F8000803F4F7C5FFA18884F80803090AF4F7D0
:10C10800BFFFA17984F80803F4F7BAFFE18884F83F
:10C118000803090AF4F7B4FFE28884F808033946EB
:10C12800F4F7B4FF84F80803D0E703230020CFE72F
:10C13800202F0020CB88B3F5407F2DE9F04104463D
:10C148000D464AD84B783C2B40D0A3F121004342FE
:10C1580043415B002A784D2AAA7808BF43F00403BC
:10C16800D10748BF43F0080392074FF0240222701A
:10C1780048BF43F010036F226270A370AB88E3706E
:10C18800AB881B0A2371EB886371EB88A71C1B0A19
:10C19800A3713846F6F72CFA0822E071E988A2F173
:10C1A80008039BB2561C8B42B6B204EB02080FD3AD
:10C1B800063189B23846F5F70BFE88F80000000A08
:10C1C800A055E8880A3080B2BDE8F0810123C1E7B4
:10C1D8002B441B7AA3543246E0E70020F4E710B55D
:10C1E800044681780020F4F74BFF217984F808038E
:10C1F800F4F746FFA18884F80803090AF4F740FF1A
:10C20800A17984F80803F4F73BFFE18884F8080370
:10C21800090AF4F735FFE28884F8080304F10801F5
:10C22800F4F734FF84F8080310BD00002DE9F74F38
:10C23800C788DFF890800D4604463A4600F10801A9
:10C248000026284607F078FD55FA87F7E6804FF074
:10C258003B09BD4205D1204603B0BDE8F04FFFF7CA
:10C26800BEBF15F8013BFF2B2AD0FE2B28D0FF2E8E
:10C278001ED1362BEDD858F833204FF0000A10465F
:10C288000192F3F7CFFF5FFA8AFB5845E388019ADA
:10C298000AF1010A05D85A1C2344E28083F8089061
:10C2A800D7E7591CE180234412F80B101972E6E70E
:10C2B800FE2ECED1E288511C2244E1801372C8E7D9
:10C2C8001E46C6E7446F010830B50F4B1C780F4B6C
:10C2D800142505FB043393F84F30012B03D0022BB0
:10C2E80010D00BB1FEE7114600234360C0F81233AB
:10C2F800A0F82236A0F8203640F2FF330160A0F8FB
:10C30800243630BD0021EFE7CC03002028040020AC
:10C31800F8B5B0F82026B0F82236D21A93B2120433
:10C3280044BF03F580639BB2E62B044608D800F2AD
:10C33800163500F21236206803685B69984700B921
:10C34800F8BD206803689B6998473146024628462D
:10C35800FFF700FD0028EED004F6262729463846C8
:10C36800FFF7E8FE00239AB29042E4D9B4F8201609
:10C37800B4F824C64A1C02EA0C02B4F822C6944552
:10C388001EBF091917F803C081F826C603F1010377
:10C3980018BFA4F82026E6E7F8B500F1080504461A
:10C3A8000A46011D2846FFF78FFD70B3637A3E2BBE
:10C3B80014D004F6262629463046FFF74CFD0246DF
:10C3C800206801680F693146B847637A3E2B1CD153
:10C3D80029460E48BDE8F840FCF708BEA389742B2F
:10C3E8000AD042F6FF729B1A18BF0123A27A92075D
:10C3F800EBD4002BDDD1E8E70023A37204F6262155
:10C408002846FFF713FF0123F0E7F8BD9407002043
:10C4180003680BB1FFF7C0BF70470346006868B1F7
:10C42800B3F82026B3F82236D31A98B21B0444BFB7
:10C4380000F5806080B2003818BF012070470346BD
:10C44800006880B1B3F82226B3F82016914209D0CB
:10C458009918013291F82606B3F824160A40A3F871
:10C468002226704700207047036843B10022A0F8D5
:10C478002226A0F820261A681846D2691047704765
:10C4880010B504460548FEF781FE0548FFF7ECFFA6
:10C4980060680368BDE81040DB691847200E00207B
:10C4A800E021002070B50A4C25780A4C142606FBBA
:10C4B800054494F84F40012C03D0022C05D00CB150
:10C4C800FEE71946416011B9FEE71146FAE770BD6B
:10C4D800CC0300202804002070B504464068A168F9
:10C4E80003681D4D9B68984760680368DB69984737
:10C4F8004FF0904301229A6202229A616326F7F76D
:10C5080079F910B12B88E3B92E80206803685B693C
:10C51800984738B1206803689B6998470146606866
:10C52800F6F761F9606803685B6998470028E6D008
:10C53800606803689B69984701462068F6F753F9D5
:10C54800DDE7013B9BB22B80002BDED1F6F71CFC0C
:10C55800F6F726FCD9E700BF0E0E0020026808B5E2
:10C568001AB143680BB1FFF7B7FF08BD2DE9F041D9
:10C578001C46064640681C4F1546F6F740F900234E
:10C588002370D7F8008023781F2B27D83B68A3EBAC
:10C598000803632B22D8706803685B6998470028F2
:10C5A800F1D0706803689B69984723780A2803F1DB
:10C5B80001022270E854E6D12378032B11D92A7896
:10C5C8004F2A0ED16A784B2A0BD12B4413F8020C50
:10C5D800A0F10D0358425841BDE8F08100202070B9
:10C5E800FAE70020F8E700BF984A002010B542F2A9
:10C5F8000F73994228BF19460446084692B0B0F511
:10C608007A7F38BF4FF47A7001A905F026FE01A899
:10C61800F4F7D4FD0A4905A807F086FB01A905A887
:10C6280007F02AFB0DF1030309AA05A92046FFF725
:10C638009DFF10B10348F6F72BFC12B010BD00BFE8
:10C648001C48010860E3160010B541229AB00A7030
:10C6580054224A700DF1030311AA0446FFF786FF1E
:10C66800002830D01948F6F713FC01A9A06805F096
:10C6780002FE01A8F4F7A2FD154909A807F054FB2A
:10C6880001A909A807F0F8FA124909A807F0F4FA6D
:10C698000DF1030311AA09A92046FFF767FF90B11E
:10C6A8000A48F6F7F5FB6068A16803689B68984735
:10C6B80060680368DB69984707490DF1030311AA0D
:10C6C8002046FFF753FF1AB010BD00BF60E3160005
:10C6D800244801082D480108B04A01082DE9F04313
:10C6E8004368A1B00446002B6DD04FF416524FF4A6
:10C6F8009643CDE905234FF416414FF46143CDE944
:10C7080007134FF4E1304FF46133CDE90903A3680F
:10C71800049301A8F6F734FA002501AB0B22197827
:10C7280013F8010F013A01EB00210D4412F0FF024A
:10C73800ADB2F4D12849294FDFF8A88014A807F032
:10C74800F3FA284605F0F0FD014614A807F094FA1C
:10C75800234914A807F090FA04AE0725606856F834
:10C76800049B036849469B68984760680368DB69CF
:10C7780098470DF103030BAA39462046FFF7F6FE4A
:10C7880020B39DF8033080336B44002203F8562C05
:10C7980014A90BA8F3F73CFD10B9A368994512D06A
:10C7A800082241460BA807F083FA78B914A9204655
:10C7B800FFF74AFF6068A16803689B68984760684C
:10C7C8000368DB69984721B0BDE8F083013D15F0A7
:10C7D800FF05C3D1EEE700BF30480108484801080B
:10C7E8004448010852480108024B1A790AB9012243
:10C7F8005A717047C0060020024B1A790AB101220B
:10C808009A717047C0060020F8B572B6F6F724FB97
:10C81800F7F71EF8F6F7A2FAF6F78EFAF6F752FED1
:10C82800F6F7D0FFF6F7C8FA284B294C294E002511
:10C8380080225A701D70F7F70BFD02232373C4E999
:10C848000455A560F6F76EFC234B1D70F6F7FAF950
:10C85800224B23484FF400425A614027F6F738FA32
:10C86800F6F716FB41F28830B762F6F711FB4CF287
:10C878005030B761F6F70CFB2046F6F711FA294657
:10C888002046184C05F082FE4FF47A70F6F700FB4C
:10C8980094F8572094F856101348FAF7C3F994F807
:10C8A80057101248FBF77CFD94F858401048214671
:10C8B800F5F7B8F83CB10F4B0F4A1A600F4B104A06
:10C8C8001A60F9F7B7FE62B6F8BD00BF9E0B0020EC
:10C8D80074310020000400483802002000040140A0
:10C8E800E0930400CC030020E01600209407002009
:10C8F800DC0D00203C020020911E000840020020B0
:10C90800ED270008184B4FF4004273B55A611748D9
:10C91800174C4FF6FF7105F089FF208023889B078D
:10C9280012D5144E35798DB1104808236A46002176
:10C9380005F0FDFDD6E90602DDE900139A4208BFBD
:10C94800884201D00023238002B070BD02236A46CA
:10C958000648294605F0EBFD074BDA8BBDF8003099
:10C968009A4218BF2580EFE7000401407431002087
:10C978000A0E0020C0060020CC030020044A002331
:10C988001370044A1380044A1370044A13707047E2
:10C99800160E0020180E0020B8310020940B00203D
:10C9A800024B1878B0FA80F040097047160E002044
:10C9B8000D4A11780346A9B910700C4A012010706D
:10C9C8000B4A032B118009D0042B01D083420AD1D2
:10C9D800084B002283F87220012070474FF4FA7345
:10C9E8001380704700207047160E0020B8310020D1
:10C9F800180E0020E4050020034A00231370034AA0
:10CA08001380034A13707047160E0020180E00207A
:10CA1800B83100200A4A08B5138883B1013B9BB29C
:10CA2800138063B9074B1B78032B02BF064B012207
:10CA38001A70FFF7E1FF054B002283F8FA2A08BDB8
:10CA4800180E0020160E0020940B0020E01600207F
:10CA580010B5C379212B0ED1074CF8F709F8FFF769
:10CA6800CBFF94F8FA1A032902D12046FAF735FBCE
:10CA7800002384F8FA3A10BDE016002010B50D4BDB
:10CA88001B78013B032B14D8DFE803F002090D07DC
:10CA98002023BDE81040F7F7DBBF2423F9E7BDE802
:10CAA8001040F8F72FB82323F7F7D2FF024B0022E4
:10CAB8001A7010BD160E0020B8310020034B012259
:10CAC8001A7000225A711A71704700BF8B2F00200C
:10CAD800054A064B12791B7F1AB105495B22F8F704
:10CAE800A5BA04495B22FAE7C0060020CC0300205F
:10CAF800B93100201432002038B5114B1A79054697
:10CB080032B1014600221846BDE83840F8F7E8BAC5
:10CB18000C4A0D495B23F8F773FA7DB90A48F7F711
:10CB280093FE0128044607D000280849284614BF68
:10CB380001240224F8F79AFA204638BD0148EEE7A6
:10CB4800C00600207030002015300020CC300020B6
:10CB5800024B1878831E5842584170478D070020B1
:10CB6800044B1B78022B06BF034B93F8720000207E
:10CB7800704700BF8D070020E405002038B5184B2A
:10CB88001A78184B0546142000FB023393F85540D9
:10CB9800012C22D12A88930606D522F020022A8069
:10CBA800052301200B7038BD12F0400316D0FFF7A3
:10CBB800D7FF20B1FFF7F4FE08B90023F1E7686852
:10CBC80030B1094B1B681B1A312BF6D900236B6057
:10CBD80022F040022A800623E3E700231846E1E713
:10CBE800CC03002028040020984A002013B50DF13A
:10CBF80007010446FFF7C2FF18B19DF8070002B00D
:10CC080010BD2080FBE700002DE9F04106460C46E8
:10CC18001546FFF7A5FF70B1184B93F82D30581E35
:10CC2800012819D8164BB3F85861B3F85671002289
:10CC380091B28D4201D8BDE8F081B3F85401411C8E
:10CC48003140B9421FBFC01814F802C080F85AC159
:10CC5800A3F854110132EBE7032B09D1094E0D4417
:10CC6800AC42E8D014F8011B3046FFF7D1FBF7E7D8
:10CC780070680368BDE8F0411B6918472804002064
:10CC8800200E0020E0210020F8B5214B214D1F790E
:10CC9800CB78C3F3000385F895304B79C3F3801341
:10CCA80085F896300646C87840080C46F4F756F9D9
:10CCB80085F892002379C3F3060385F893306379E6
:10CCC800227903F03F035B0043EAD21385F89430DE
:10CCD800E6B1DFB1A37803F0F003202B04D120469E
:10CCE800BDE8F840FFF7B4BEA2790B48E11D520831
:10CCF800FFF78AFFA17905F164004908F4F7D5FC2C
:10CD080005F13C00BDE8F840F4F7C9BCF8BD00BF28
:10CD18008B2F0020CC3000209031002070B50546C4
:10CD2800B8B9184B184E1B78184A14794CBB022B0B
:10CD3800174812D1B17801F00701F8F72BFA4379B7
:10CD4800C3B931460120FFF79FFF1248F4F78DF869
:10CD580009E0114B114E1B78E6E70122934202705D
:10CD680044710471EDD80B4880F89050BDE87040CC
:10CD7800F4F779B80A4B1C745C825C61094B1C712E
:10CD8800DFE770BD120E002015300020C00600201D
:10CD98008B2F0020CC300020130E00207030002094
:10CDA800200E0020E021002010B50246FFF7D8FE33
:10CDB800B8B10C4B93F82D30591E012904D8BDE8A1
:10CDC80010400948FEF7BEB9032B04D1BDE8104056
:10CDD8000648FFF722BB50680368BDE810405B694E
:10CDE800184710BD28040020200E0020E021002054
:10CDF80010B50246FFF7B4FEB8B10C4B93F82D30CE
:10CE0800591E012904D8BDE810400948FEF7A9B900
:10CE1800032B04D1BDE810400648FFF710BB50684B
:10CE28000368BDE810409B69184710BD280400201E
:10CE3800200E0020E02100202DE9F04FDFF8E880E7
:10CE480098F8004097B081460E461746002C53D1FB
:10CE58002D4B1B78022B4BD1DFF8C8B00DF1180A07
:10CE680025465846ECB2FFF79FFF40B15846FFF7FA
:10CE7800BFFF0135402D0AF8010BF2D12C4623489B
:10CE88002146F4F712FC2248F4F709FC214D8DF8ED
:10CE9800129095F8A4308DF80C301F4B85F89190BE
:10CEA800DB788DF80D30284695F890308DF81130E4
:10CEB800F4F700F88DF80E00F7F780FE10F0010F78
:10CEC8008DF8130018BF3E4628468DF81460F4F715
:10CED80003F898F800308DF810007BB90F4A104815
:10CEE800009406AB03A9F7F7A3FC17B0BDE8F08FD1
:10CEF8000C48FFF7C5FAC9E70024C7E7074A0848FE
:10CF080003A9FFF7BBFDF0E78D0700201C310020C7
:10CF1800F4300020CC3000208B2F0020922F0020EE
:10CF28001432002090310020B831002030B4084C71
:10CF3800257925B10146204630BCF7F7FFBE054CE0
:10CF480094F8A430013384F8A43030BCFFF774BFE0
:10CF5800C0060020CC30002008B50246FFF700FECE
:10CF680018B9A2F82206A2F82006054B93F82D302E
:10CF7800032B04D1BDE808401046FFF7C9B908BD26
:10CF88002804002070B500239CB2A24200D870BDCE
:10CF9800058886886C1C34404688A6421EBF2D181A
:10CFA800CE5CAE7103F1010318BF0480ECE708B54D
:10CFB8006830FFF7E7FF08BDA0F11400F7E70000AD
:10CFC80038B50A4B93F82D3000F5EF65022B04466F
:10CFD800284608D1FCF7FAFC0246294604F24A40E2
:10CFE800FFF7D0FF38BDF5F72EF8F5E72804002045
:10CFF8002DE9FF410446B0F84C14B0F84A04F5F79F
:10D008001BFBE3684BBBDD2808D804F5F37604F571
:10D01800ED75A06803685B69984710B904B0BDE86E
:10D02800F081A06803689B6998472A460346314601
:10D038006846F5F76DF90028EBD09DF80030022B13
:10D04800ECD104F5CA65324669462846F5F7C2F8B8
:10D0580029462046FFF7B4FF94E0DD28DED84D4D81
:10D068002B780133DBB2012B2B700FD900232B70E7
:10D07800A06803685B69984750B901232B70E06882
:10D0880003685B69984730B9287004E0002BEFD03B
:10D098002B78012BF3D004F5F37604F5ED772B7894
:10D0A800002B36D1A06803685B69984788B3A068ED
:10D0B80003689B6998473A46034631466846F5F740
:10D0C80027F90028EBD0DFF8D08069460120F5F772
:10D0D800DFFA98F8023033B1E068BDF8022003683F
:10D0E80031461B6998479DF80030022B11D104F591
:10D0F800CA67324669463846F5F76CF898F8003042
:10D108001BB139462046FFF75BFF39462046FEF73C
:10D118002FFA04F21E3604F212372B78012B7FF413
:10D128007DAFE06803685B69984700283FF476AFF5
:10D13800E06803689B6998473A4603463146684663
:10D14800F5F7E6F80028E8D0134F69460220F5F70E
:10D158009FFA7B7833B1A068BDF802200368314696
:10D168001B6998479DF80030022B7FF457AF04F5F0
:10D17800CA65324669462846F5F72CF83B78002BF5
:10D188007FF466AF2946204604B0BDE8F041FEF7BB
:10D19800EFB900BFBC0600207D0600201D4B70B50E
:10D1A8001D680446FFF7DCFC58B9C4F8A458A4F875
:10D1B8005601A4F85401A4F84C04A4F84A0484F8CD
:10D1C800AD08154E96F82D30013B012B21D820468D
:10D1D800FEF796FC2046FFF70BFF104B1B78142236
:10D1E80002FB036696F8523063B1D4F8A438EB1A00
:10D1F800B3F57A7F08D3C4F8A4582046BDE8704038
:10D20800FDF7DABFC4F8A4582046BDE87040FEF721
:10D21800D1BA70BD984A002028040020CC03002011
:10D228002DE9F04FDFF8B48198F80030012B85B074
:10D2380000F25B811BB9F5F7F1FC04F04DFC5B4D86
:10D24800FFF7E2FA696C5A48F6F7ACF8696C594886
:10D25800F6F72CFA584B00221A809A704FF0904338
:10D2680001229A6207244CF25030013CF5F798FDF0
:10D27800F5F70EFE14F0FF04F5D1504805F006FB53
:10D28800013880B24FF6FD73984203D94C4901200A
:10D29800F7F74EFF4B4B4C491C804C4B47481C80C2
:10D2A800F7F78CF87D20F5F7F3FD4948F5F738FDD9
:10D2B800F7F79EFC95F820B0BBF1200F00D9FEE7E8
:10D2C80095F82800434EAB8D01930528696A95F8B7
:10D2D800297095F82A30B07100D9FEE73E4A4FEA26
:10D2E800001E02EB001C52F80E2002B9FEE7B260E5
:10D2F8009CF804209CF80C900092F271DCF808204D
:10D30800326186F80C9086F8D900B482A446A24609
:10D31800A646019A42FA0CF2D20707D5012202FA70
:10D328000CFA4EEA0A0A1FFA8AFE92460CF1010C20
:10D33800BCF1060FEDD1DFF89CC0BAF1000F01D0A7
:10D34800ACF814E0BCF814E0BEF1000F00D1FEE721
:10D35800009AA2EB0902D2B25A4528BF5A460528BC
:10D368008CF8172000F0FD80012800F2018107F1F8
:10D37800FF30C0B200F0EB80022831D8581EC0B28E
:10D3880003280CD80C2A02D90C208CF817009CF81A
:10D398001700904201D98CF817203C4623E0122A46
:10D3A80084BF12238CF817300023F0E7CC03002049
:10D3B80030020020340200200E0E002074310020BC
:10D3C8005B480108080E0020D00300200A0E002048
:10D3D800C0060020A00B002000520108B72F002033
:10D3E800052B28BF00236C482246F4F7B5F8002423
:10D3F8006A4B86F8D840FF27B47567481F705F707E
:10D40800F7F7CCF801466648664E05F0E4F8664B37
:10D418001C80664B1C70664B1C70664B1C80664BF0
:10D428001C80664B1C70664B1C80664B1C70664BE0
:10D438001C70664B1C70664B01201C70FFF79EFA2F
:10D44800FFF7B6FAB5F84830B5F84A2095F8401015
:10D458006048F3F7CDFCB5F848105F48F3F7FCFFD8
:10D468005E48F7F76DFE2A785D4B5E48142101FB94
:10D47800023393F84E10F4F7DDFA5B4B5B4A5C48D5
:10D488003146FEF739FA584A5A483146FEF71CFF2A
:10D4980013465948554A3146FFF704F8B5F848206D
:10D4A80056495748F8F77AF956486B6C8360C0E9D3
:10D4B8000016FFF713F93A48F7F761F801465248A2
:10D4C800F7F78EFD5148F4F726F95148F4F7FDF8BF
:10D4D8005048F4F771FA504B1C70504B1C80504B5D
:10D4E8001C80F6F77DF988F80070F6F783F9304D5F
:10D4F800002800F0BF80324A13880BB1013B13802B
:10D50800294A138813B9474BB3F84830013B9BB2FB
:10D51800012B138030D1254A1370FFF77BFA2B7843
:10D52800002B40F0A780254B3F4A19781388022921
:10D538002BD173B3013B9BB213809278002A77D02A
:10D54800002B7FD1F5F720FCF5F72AFC7AE00228BA
:10D5580005D80C2A02D90C238CF817303C46002336
:10D5680041E77B1E022BFAD8082AF7D90823F3E7EC
:10D578000948F3F78BFF3AE7002BCED101232B7034
:10D588002A4B5A6A0B4B1A80C7E7002BD2D1C72304
:10D59800D2E740F2F313CFE7A00B0020B82F00200A
:10D5A8007431002030020020703200200C0E002060
:10D5B800950B0020882F0020140E00208D070020D6
:10D5C800900700208E0700208C070020130E0020F3
:10D5D800120E0020CC300020A43100208B2F002018
:10D5E80028040020DC0D002034020020F41600205E
:10D5F800200E0020E02100209031002000000020B3
:10D60800F4060020D00D00209E0B00208C4A00203C
:10D618009831002084070020B62F0020B431002064
:10D62800B6310020CC0300200E0E0020000400407C
:10D6380002294FF0904040F0D0800BB9F5F7A4FBD9
:10D6480001238362954C2388002B00F0CC80013B9A
:10D658009BB293482380F7F70DFB9248F6F78FFFAC
:10D6680001469148F7F7BCFC23881BB98F499048BD
:10D67800F5F7C5F88F4E904C3388022B00F0B68032
:10D68800042B00F0DB80012B0FD18C4B9A7DD97DC8
:10D698000132D2B2914298BF00229A75884B114646
:10D6A800187AFFF743FC0223338023889BB2EBB13F
:10D6B8003388032B40F0DB802388D80703D5002369
:10D6C80023800423338023889BB27BB1238823885B
:10D6D8009A0748BF238823887A4ADB0748BF2388EC
:10D6E80000231370784A2380338013702B78002B23
:10D6F80000F05681744F6B4800242C70F6F7E4FE56
:10D7080097F80090B9F1000F00F0BF802046FFF7AE
:10D7180005FB6B4B694D1C726C4BAA7D83F8A720E7
:10D728003A7868496A4C012A94BF0022012283F89A
:10D73800A5200A78012A94BF00220122B9F1010F1D
:10D7480083F8A62023780AD96248002B00F0A0802D
:10D75800012B00F0D980604BB0F84C201A80237858
:10D76800022B03D15C4B1B8803B92370227800235A
:10D778000120022A30803B700B7006D057490B708D
:10D788001AB9FFF739F9FFF713F9554A138813B98E
:10D79800504BB3F84A30013B9BB2138013B94B4846
:10D7A800F3F7AEFB4948F3F75DFB2378022B02D071
:10D7B8004648F3F705FB4B4B1F78002F00F0CD8050
:10D7C8004FF09043012402229C619A61F6F724FDF0
:10D7D80088F8004005B0BDE8F08F02228262002B75
:10D7E8007FF430AFB0E640F2E73332E73E4B3F4AD2
:10D7F8005B6A12889B1A9BB240F2ED2293427FF635
:10D8080054AF3B4B3B4800271F70F7F7CDFC2B4824
:10D81800F6F7C4FE0146234804F0DDFE284B187ACB
:10D82800FFF756F903233380334B34481F80344BBA
:10D83800278001221A71F3F772FF36E719484FF66D
:10D84800FF71F5F73DFA04F05CFF1648002104F07B
:10D858008CFF7D20F5F71CFB1A4A05233380002333
:10D868001370194A1370244A138023801DE7052B6F
:10D878007FF429AF238899077FF525AF0020208002
:10D88800FFF73AF9104B18701DE7FFF717F940E753
:10D89800012222701B4A13705DE700BFB4310020DB
:10D8A800C0060020743100209E0B0020AA3D01080C
:10D8B80004000020140E00200A0E0020A00B0020F7
:10D8C800A4310020130E0020120E0020CC300020BE
:10D8D8008D070020CC030020900700208B2F00200C
:10D8E800B6310020940B002000040040882F00204F
:10D8F8000C0E0020B82F0020080E00208C4A0020B3
:10D90800940700208E070020944ADFF8909213783D
:10D918000133DBB2137099F80020C2B990F850C0F7
:10D928009C453FF618AFDFF878A29AF8723043B9F1
:10D938008B4B1B792BB96AB1FFF75EF801238AF884
:10D94800723002232370012389F8003003E74FF077
:10D95800050CE5E783490C209AE48148F7F7B4F908
:10D96800F7F7DEF90128064606D003287FF432AF20
:10D97800012388F800302DE77948F7F755F941F287
:10D988008833A5F8DA304FF09043022285F8D86042
:10D99800A5F8DC709A619E62734B27709E7019E738
:10D9A800724C734D94F85630EBB172497248F9F7DE
:10D9B80073F968B12278714B142101FB02330122FB
:10D9C80093F84C30032B04BF01232B706A4B1A7158
:10D9D80069480DF10B01F9F778F920B19DF80B3082
:10D9E800F3B1012B1FD094F8563023B994F857306F
:10D9F800002B00F00D8160480DF10B01F9F78AF951
:10DA080070B39DF80B30033B0F2B29D8DFE803F0E8
:10DA18001628284528282847284D6371767C787A67
:10DA2800FEF7D8F8DFE7544803A9F9F7A1F9002869
:10DA3800D9D09DF80C00F9F76DFCD4E7F6F7FCFB9C
:10DA48004F4B1B78022B07D10420FEF7B1FF4A4B3E
:10DA5800032283F8FA2A03E003214748F9F73DFB3C
:10DA680094F85730002B00F0D38042494548FAF724
:10DA7800EDFC08B101232B70B4F84820414802A9F5
:10DA8800FAF706FD00284CD09DF80830042B48D83A
:10DA9800DFE803F0415B5F88B8000621DDE73A491B
:10DAA800A1F13300F9F7F0FADAE7334F03A907F1E8
:10DAB8003300F9F711FC0028D2D09DF80C30002B68
:10DAC800CED02F4B18780228CAD1FEF771FF0C234D
:10DAD80087F8FA3AC4E72A4B1B78022B05D10320B2
:10DAE800FEF766FF244B0D22B3E7284B01221A707C
:10DAF800B6E701212648F3F703FEB1E70221F9E76B
:10DB08000321F7E70821F5E71B4B224893F8331068
:10DB1800F3F756FFA4E71B48FBF748FB1E4B002210
:10DB28001A70184F0DF109013846FAF7EBFC002876
:10DB38006ED09DF80930022B68D8002B00F0AE801B
:10DB480013480121F3F7DEFD62E00E48FBF776FB90
:10DB5800E7E70C48FBF7AAFBE3E700BF8E070020C6
:10DB6800C0060020654801080E0E0020CC030020E6
:10DB7800B62F0020922F0020E01600202804002055
:10DB88008D0700209407002013170020940B002015
:10DB98009831002084070020B70600208C07002059
:10DBA800E4050020684F3B784BB968480DF10A013D
:10DBB800F9F7DEF818B19DF80A00F9F7ABFB6348EE
:10DBC8000DF10B0203A9F9F717F868B19DF80B20BE
:10DBD80003995F48FAF7EAFC3B780133DBB2022B82
:10DBE80088BF00233B709CE7FEF7BAFF0028F3D0FC
:10DBF800584B93F82D30013B022BEDD85448FAF7D7
:10DC08009FFEE9E75248FBF77FFB8AE7032B4BD0DF
:10DC180094F8583023B150495048F4F743F808B9FC
:10DC28002B78BBB100232B704A4D23784A494C48C6
:10DC3800142707FB035393F84D20F3F7B7F823781D
:10DC48004549484807FB035595F84A3095F856204A
:10DC5800F7F7CAFA444B1B78002B7FF4BBAD338827
:10DC6800022B3FF4B7AD4148FFF798FA4048FFF759
:10DC780073F94048F3F760FD3F48F3F72BFD10B9FF
:10DC88003A48FEF7B3FF431E0B2B58D8DFE803F0E2
:10DC98003B3E41571520335757434B4F97F8691070
:10DCA8003648F3F78DFEB3E7BA7D2848023AD2B278
:10DCB80007F11801F8F78BFFAAE7314B187802280B
:10DCC8000FD1FEF775FE214BFF2283F8FA2A08E0F0
:10DCD8002B4B1B78022B01D10320F2E7294B0122A1
:10DCE8001A702648F3F780FE00283FF473AD254BE1
:10DCF80001221A706EE5F6F79FFA214B1B78022B6A
:10DD0800EFD10420DDE7FEF76FFDEAE7FEF774FDCB
:10DD1800E7E7F4F73FFF1848F3F7FBFCC1B21748F1
:10DD2800F3F74EFEDDE71848FEF718FCD9E712486E
:10DD3800F3F7EFFC81B21448FEF758FCD1E704284A
:10DD48003FF416AECDE700BFB7060020E01600206E
:10DD58009407002028040020922F0020DC0D0020CA
:10DD6800EC060020B82F00200C0E0020200E00200A
:10DD7800E02100208C4A00209831002084070020F0
:10DD88008D070020940B0020D00D002008B5FFF768
:10DD980047FAFCE738B5244B244A1A60244B254A35
:10DDA8001A605A619A62DA63234A1A655A66234AE4
:10DDB8009A67234A234B244802F108012832002499
:10DDC8005A6140F2FF12C3E91A427F251F4A1960BF
:10DDD800C3F87022C3F86C42C3F8744AC3F8785A7F
:10DDE8001B4B036000F58E70FAF782F9194B1A4A3B
:10DDF8001A601A482146F2F789FF194B194AC3F8E5
:10DE08004C24C3E95545A3F84A44174B40F2FF3266
:10DE1800C3F82426C3F82046144B154A1A60154B3C
:10DE2800154A1A6038BD00BF7431002084480108C3
:10DE3800CC300020043F0108EC3E0108F83E010800
:10DE480050710108E0160020940700200000FF0729
:10DE580048710108DC0D00206C490108EC0600201F
:10DE6800200E00200000FF01E0210020903100205A
:10DE7800047101088C4A00203471010810B594B06F
:10DE88003822002106A805F0EFFE1422002101A87F
:10DE980005F0EAFE002001F0A5F901224FF48033D5
:10DEA800CDE9062303240223552206A8CDE90D3423
:10DEB800CDE91023CDE912330F9301F0F5F908B13C
:10DEC80072B6FEE70421CDE903000F2305900DEBA0
:10DED8000100CDE9013401F02DFC08B172B6FEE76E
:10DEE80014B010BD07B5104A136823F4806313609B
:10DEF80000F0B4F8FFF7C2FF0C4BDA6C42F02002D6
:10DF0800DA64DA6C02F020020192019ADA6C42F0CB
:10DF18000102DA64DB6C03F001030093009B03B099
:10DF28005DF804EBFFF732BF00200240001002400A
:10DF380072B6FEE70B4B1A6E42F001021A661A6EB1
:10DF480082B002F001020092009A9A6D42F080526B
:10DF58009A659B6D03F080530193019B02B001F019
:10DF68009BB900BF00100240FEE7FEE7FEE7FEE7B0
:10DF7800FEE7704770477047F5F74CBC034AD2F884
:10DF8800883043F47003C2F88830704700ED00E031
:10DF98000D488546FFF7F2FF0C480D490D4A00234E
:10DFA80002E0D458C4500433C4188C42F9D30A4A46
:10DFB8000A4C002301E013600432A242FBD305F0AF
:10DFC8008FFEFFF78FFFFEE7008000200000002093
:10DFD800AC03002068770108B0030020806B0020A4
:10DFE800FEE7704710B5094B4FF0FF3200249A63E3
:10DFF8009C631A641C649A629C62DA62DC621A632B
:10E008001C63FFF7EEFF204610BD00BF0010024062
:10E0180038B50F4B1A6805460AB9012038BD4FF4C8
:10E028007A73B3FBF2F30B4A1068B0FBF3F000F01D
:10E038008FF804460028F0D10F2DEED80246294665
:10E048004FF0FF3000F032F8034B20461D60E5E743
:10E0580048020020440200204C02002010B5032092
:10E0680000F012F80F20FFF7D3FF044618B9FFF7A6
:10E0780061FF204610BD0124FBE70000014B186832
:10E08800704700BF984A00200749CA6822F4E06236
:10E098000302120403F4E063120C134343F0BF635A
:10E0A80043F40033CB60704700ED00E0164B30B509
:10E0B800DC68C4F30224C4F10703251D042B28BF20
:10E0C8000423062D4FF0FF358CBF033C002405FACE
:10E0D80003F321EA0303A54022EA0502A34000282E
:10E0E80043EA0203ACBF00F16040084A4FEA031359
:10E0F800B8BF00F00F00DBB2AABF00F561401354AF
:10E1080080F8003330BD00BF00ED00E014ED00E002
:10E11800002807DB044A4109012300F01F0083405F
:10E1280042F82130704700BF00E100E000280CDB16
:10E138004309064900F01F0020330122824041F8BC
:10E148002320BFF34F8FBFF36F8F704700E100E0CC
:10E158000138B0F1807F0BD24FF0E023054A5861B7
:10E16800F02182F823100020072298611A61704775
:10E178000120704700ED00E0094A536943F4802309
:10E1880010B55361EFF3108272B60023CC58C45017
:10E198000433B3F5807FF9D182F3108810BD00BF36
:10E1A80000200240064B5A69002ABFBF054A9A6000
:10E1B80002F188329A60BABF5869C00F00207047D0
:10E1C8000020024023016745044B5A6942F000428F
:10E1D8005A615869C043C00F704700BF0020024011
:10E1E80070B50646FFF74AFF0F4C05462369DB0367
:10E1F8000BD423694CF2FA3213400DD00B494A680C
:10E208001A434A600120236170BDFFF737FF401BA6
:10E21800B042EBD90320F7E7206910F00100F3D0F2
:10E22800012222611846EFE7002002405002002038
:10E238002DE9F0471D4E99463378012B05460F46C8
:10E24800904631D04FF0010A4FF47A7086F800A05A
:10E25800FFF7C6FF0446B8B97060CDB9144A5369D0
:10E2680043EA0A035361C7F80080BFF36F8FC7F80A
:10E27800049054464FF47A70FFF7B2FF24B10C4A69
:10E28800536923EA0403536100233370BDE8F08720
:10E298006B1E012BEED841463846FFF76DFFAB1ECB
:10E2A8005D425D41AC04E5E70220EFE75002002043
:10E2B80000200240064B10F0010F1EBF5A6942F0C1
:10E2C80004025A615A6942F480325A61704700BFA9
:10E2D80000200240084B5A69C00022F4FC7200F486
:10E2E800FF60104358615A6942F002025A615A6944
:10E2F80042F480325A617047002002401548037F7B
:10E30800DAB203F0FD03012B10D1134B196821F485
:10E3180000711960196841F400611960196821F4E5
:10E3280000611960196841F400711960931E012B8E
:10E338000CD8094B1A6842F480521A601A6822F401
:10E3480080521A601A6842F480621A6000230377C8
:10E35800704700BF50020020002002402DE9F8431A
:10E36800314D2B78012B064688465AD001274FF4A9
:10E378007A702F70FFF734FF044610BB2B4B686090
:10E388001A6812F4007F1A6820D0510506D51A6859
:10E3980022F480621A6003232B7700E02F7733681A
:10E3A800012B1DD17068FFF785FF4FF47A70FFF7D6
:10E3B80017FF1E4A536923F0040304465361FFF70D
:10E3C8009DFF00232B702046BDE8F883520505D534
:10E3D8001A6822F480621A600223DDE72877DEE7F4
:10E3E8004FF0FF33C8F80030B768DFF84090D6E93F
:10E3F80002321344BB42E2D971683846FFF76AFF1C
:10E408004FF47A70FFF7ECFED9F8143023F4FD735B
:10E41800C9F8143018B1C8F800700446CFE70137BE
:10E42800E5E70224CFE700BF5002002000200240A9
:10E43800F0B5044687B0002858D090F8AD3203F004
:10E44800FF021BB980F8AC2203F080FC03230025EF
:10E4580084F8AD326562206801F095FF2B46666846
:10E46800282501271846D9B28E4203F1010323D883
:10E47800002328251946D8B2864203F1010328D87B
:10E4880004F110060FCE6D460FC596E8030085E827
:10E498000300231D0ECB206801F07FFF0025012318
:10E4A80084F8285084F8AD32E369012B02D1204664
:10E4B80000F080FE28461AE005FB0142C2E90F0081
:10E4C80082F82D7082F82C10518782F82F00506442
:10E4D800C9E705FB0042C2E95F1182F86D1182F8B5
:10E4E8006C0182F86F11C2F88411C4E7012007B0EB
:10E4F800F0BD38B5044610B90125284638BD0323B8
:10E5080080F8AD32006802F0EFF905460028F3D133
:10E51800204603F039FC84F8AD52EEE710B590F8C8
:10E52800AC32012B04460CD0012380F8AC320068D1
:10E5380001F020FF206802F0E8F9002084F8AC021E
:10E5480010BD0220FCE710B590F8AC32012B044650
:10E558000CD0012380F8AC32006801F014FF206869
:10E5680002F0DEF9002084F8AC0210BD0220FCE7BE
:10E5780010B590F8AC22012A04460BD0012280F88D
:10E58800AC2280F82810006802F0B9F9002084F85D
:10E59800AC0210BD0220FCE72DE9F74F04460068E5
:10E5A80002F0C6F910F4004100F02F84DFF8088368
:10E5B800C04F2068B0F844301A0402D403B0BDE854
:10E5C800F08FB0F84450A9B215F00F0540F0B780AD
:10E5D80011F010012AD103889BB203EA080343F41F
:10E5E80000430380B0F8503094F82C2000F2024029
:10E5F80010FA83F3204633F83230226CC3F3090350
:10E608001A44A364226403F0E0FB94F82830002B3A
:10E61800CFD0626C2168002ACBD194F8283043F01F
:10E628008003A1F84C3084F82820C2E70588ABB2F3
:10E6380015F4006520D0B0F8503094F86C2100F241
:10E64800064111FA83F304F52D7133F83230B4F82A
:10E658007221C3F30903C4F8883102F0B9FB2268B8
:10E66800138823F070031B051B0D43F080031380F0
:10E67800204603F09BFB9CE71A049AD5038823F0F5
:10E6880070031B051B0D43F080030380B0F8503066
:10E6980094F86C2100F2064111FA83F333F8323012
:10E6A800C3F30903C4F888318BB1D4F8801171B170
:10E6B800B4F8722102F08CFBD4F88031D4F88821A8
:10E6C8001344C4F880312946204603F075FB2168BD
:10E6D8000B881B053FF56DAFD4F87C51B1F850306D
:10E6E8003E2D9BB201F2064008D96A09EE0608BF22
:10E6F80002F1FF3247EA822292B20AE0CDB9C25A49
:10E7080022F4F8421204120CC252C25A92B242F4D3
:10E718000042C2520B8823F4804323F070031B0489
:10E728001B0C83F4405343F4004343F080030B80F5
:10E738003FE76A08ED0748BF01329202DCE70FFAAB
:10E7480085F930F8293019049EB240F1F58030F887
:10E75800293023F070031B051B0D43F0800328218B
:10E7680020F8293001FB054191F87831BBB9B0F8A0
:10E77800503091F86C2100F2064C1CFA83F333F800
:10E7880032A0CAF3090ABAF1000F00F0B980B1F853
:10E7980072215346D1F8801102F01AFBB0E091F8CB
:10E7A8006F31022B91F86C3140F08880B0F850C07E
:10E7B800D1F884214FEAC30A10FA8CFC16F4804B76
:10E7C800D44406F0400E3AD0BCF802A4CAF3090AB1
:10E7D800924513D90022C1F8842130F8232022F46D
:10E7E800804222F070021204120C82F4005242F4A9
:10E7F800004242F0800220F8232005E0A2EB0A0242
:10E80800C1F88421002AE8D0BEF1000F0DD030F8FD
:10E81800232022F4E04222F070021204120C42F487
:10E82800004242F0C00220F82320BAF1000F67D05E
:10E83800282101FB0541B1F874215346AAE7BCF829
:10E8480006A4CAF3090A924512D9C1F884B130F86E
:10E85800232022F4804222F070021204120C82F467
:10E86800005242F4004242F0800220F8232005E0E2
:10E87800A2EB0A02C1F88421002AE8D0BEF1000FF9
:10E888000DD130F8232022F4E04222F07002120465
:10E89800120C42F4004242F0C00220F82320BAF1E0
:10E8A800000F2DD0282101FB0541B1F876215346F0
:10E8B80070E700BF0080FFFF0F8FFFFF30F82320B5
:10E8C80022F4E04222F070021204120C42F40042D8
:10E8D80042F0C00220F8232091F86C2130F8223051
:10E8E80013F4804FB0F8503062D000F2024C1CFA9A
:10E8F80083F333F832A0CAF3090ABAF1000F9AD1A8
:10E90800282101FB0543D3F888215244C3F8882104
:10E91800D3F880215244C3F88021D3F884211AB156
:10E92800D3F87C319A454FD2282303FB0543204670
:10E9380093F86C1103F040FA320620687FF539AE7F
:10E9480030F829309BB203EA080343F4004320F867
:10E95800293009EB890904EBC9094FF0280C99F80B
:10E968002F30022B5BD00CFB054C00259CF838306F
:10E97800CCF84450002B3AD016F0400699F82D30C8
:10E9880099F82C2039D03BBBB0F8503000F2024047
:10E9980010FA83F303EBC2031A8822F4F842120434
:10E9A800120C1A801A8892B242F400421A801EE0B1
:10E9B80000F2064C1CFA83F333F832A0CAF3090AB2
:10E9C800BAF1000F9CD070E701FB0541206801F502
:10E9D800B67101F0C1FFAFE7012B08D1B0F8503094
:10E9E80000F2024010FA83F303EBC2031D8099F88A
:10E9F8002C10204603F0E9F9DBE523B9B0F85030D4
:10EA080000F20640C4E7012BF1D1B0F8503000F213
:10EA1800064010FA83F303EBC2031E80E7E799F878
:10EA28002C100CFB054E16F4807ADEF844300A46AA
:10EA38004FEAC10B22D1B0F850201BFA82F20244EF
:10EA4800B2F80264C6F309069E4202D3CEF844A087
:10EA5800CFE79B1BDEF84020CEF84430DEF8483084
:10EA680005FB0CCC324433440CF10401CEF84020B1
:10EA7800CEF84830214401F06FFF9AE516F0400ABD
:10EA8800B0F850C006F4804600F0E18000F2024E73
:10EA98001EFA8CFC4FF0280A3CF831C0CCF3090C64
:10EAA8009C450AFB054A34BFA3EB0C030023CAF8B4
:10EAB8004430B6B2002B54D199F82D50002D3FD1D7
:10EAC800B0F850501EFA85F535F8313023F4F84384
:10EAD8001B041B0C25F8313035F831309BB243F458
:10EAE800004325F83130B0F8503000F2064010FAF3
:10EAF80083F030F8313023F4F8431B041B0C20F862
:10EB0800313030F831309BB243F4004320F83130D3
:10EB1800204603F05AF9002E00F0E28099F82C10F4
:10EB2800226832F8213023F4E04323F070031B04F9
:10EB38001B0C43F4404343F0800322F82130CFE01C
:10EB4800012DE5D1B0F850501EFA85F525F8313081
:10EB5800B0F8505000F2064010FA85F525F831302B
:10EB6800D6E76EB130F8213023F4E04323F0700388
:10EB78001B041B0C43F4404343F0800320F821306E
:10EB8800282606FB054696F85030012B40F0A88051
:10EB9800B36C316CD6F84CA06344B364F36B614436
:10EBA8009A4531641CD3AAEB030AC6F84CA099F81D
:10EBB8002D601FFA83FA002E40D1B0F850603E2B2A
:10EBC8001EFA86F619D94FEA531CDB0608BF0CF16A
:10EBD800FF3C47EA8C2C1FFA8CFC26F832C01CE05C
:10EBE800BAF1000F03D186F850A06346DFE700238F
:10EBF80086F85030F3645346D9E7B3B936F8323063
:10EC080023F4F8431B041B0C26F8323036F8323054
:10EC18009BB243F4004326F83230282202FB054217
:10EC28005346928E01F088FE5AE04FEA530CDB07F8
:10EC380048BF0CF1010C4FEA8C2CCCE7012E02BF27
:10EC4800B0F850301EFA83F323F832A0E5E700F25B
:10EC5800064E1EFA8CFCB6B23CF831C0CCF3090C57
:10EC68009C4588BF53464FF0280A0AFB054A98BFBF
:10EC7800A3EB0C03CAF84430002B53D199F82D505C
:10EC8800002D40D1B0F8505000F2024313FA85F538
:10EC980035F8313023F4F8431B041B0C25F83130C8
:10ECA80035F831309BB243F4004325F83130B0F8E1
:10ECB80050001EFA80F030F8313023F4F8431B047A
:10ECC8001B0C20F8313030F831309BB243F400434C
:10ECD80020F83230204603F078F8002E3FF41EAFBB
:10ECE80099F82C10226832F821309BB223F4E043C3
:10ECF80023F0400383F0300343F4004343F08003E0
:10ED080022F8213055E4012DE4D1B0F8505000F23A
:10ED1800024C1CFA85F525F83130B0F850001EFA7F
:10ED280080F0D5E76EB930F8213023F4E04323F0C2
:10ED380070031B041B0C43F4404343F0800320F88A
:10ED48002130282606FB054696F85030012BC7D1FE
:10ED5800B36C316CD6F84CA06344B364F36B614474
:10ED68009A4531641CD3AAEB030AC6F84CA099F85B
:10ED78002D601FFA83FC002E3ED1B0F850603E2B68
:10ED88001EFA86F619D94FEA531EDB0608BF0EF1A4
:10ED9800FF3E47EA8E2E1FFA8EFE26F832E01CE070
:10EDA800BAF1000F03D186F850A06346DFE70023CD
:10EDB800F36486F850305346D9E7A3B936F83230B1
:10EDC80023F4F8431B041B0C26F8323036F8323093
:10EDD8009BB243F4004326F83230282303FB054551
:10EDE8006346EA8E1EE74FEA530EDB0748BF0EF173
:10EDF800010E4FEA8E2ECEE7012E02BFB0F850303A
:10EE08001EFA83F323F832C0E7E7430513D52268D7
:10EE18000191B2F8443023F480631B041B0C204694
:10EE2800A2F8443002F0DDFF0199204603B0BDE8A6
:10EE3800F04FFFF79DBB47040AD52268B2F844306B
:10EE480023F480431B041B0CA2F84430FFF7B6BB25
:10EE580010F4005105D02268B2F8443023F400536E
:10EE6800F0E7C60422D52268B2F8403023F0040344
:10EE78001B041B0CA2F84030B2F8403023F0080302
:10EE88001B041B0CA2F8403094F8E432012B04D187
:10EE980084F8E412204600F0A4F9204602F0C4FFEA
:10EEA8002268B2F8443023F48053CBE705051BD51C
:10EEB8002268B2F840309BB243F00803A2F8403011
:10EEC800B2F8443023F400631B041B0CA2F844304E
:10EED800B2F840309BB243F00403A2F84030204619
:10EEE80002F092FFFFF76ABB01062BD52368B3F83F
:10EEF800442022F080021204120CA3F8442094F853
:10EF0800E422002AEBD1B3F8402092B242F0040286
:10EF1800A3F84020B3F8402092B242F00802012141
:10EF2800A3F8402084F8E412B3F85430C3F38D03F7
:10EF380003F03C032046C4F8E83203B0BDE8F04FC4
:10EF480000F04FB982050DD52268B2F8443023F499
:10EF580000731B041B0CA2F84430204602F03DFF4E
:10EF6800FFF72CBBC3057FF529AB2268B2F8443004
:10EF780023F4807366E700BF11F0800F70B5054673
:10EF88004FF0280401F007001ED000FB0444211DA7
:10EF98002C440126294466710A614A780870CB70AE
:10EFA80002B1C881022B04BF00230B7195F8AC3263
:10EFB800012B13D00123286885F8AC3201F002FA3E
:10EFC800002085F8AC0270BD04FB005104FB00541E
:10EFD800002601F5B67184F86D61DDE70220F2E7DD
:10EFE80011F0800F10B501F0070204464FF0280316
:10EFF80015D002FB0333191D034401440120587145
:10F008000A7094F8AC32012B13D00123206884F8DD
:10F01800AC3201F02DFB002084F8AC0210BD03FBDC
:10F02800020103FB0203002001F5B67183F86D01AC
:10F03800E6E70220F2E770B501F00701282606FB93
:10F048000104002584F86C11C4E96023C4F88851D0
:10F0580084F86D5104F5B671006801F07DFC28460E
:10F0680070BD01F00701282303FB0100D0F88801D7
:10F07800704770B501F00701282404FB0105C5E9B4
:10F088001023EB6401EB810300EBC303012200268C
:10F0980001FB044485F85020AE6483F82C10211D30
:10F0A800014483F82D20006801F056FC304670BDFD
:10F0B80010B5044601F007006368984226D811F09D
:10F0C800800F4FF0280317D000FB03331A1D234489
:10F0D80001212244597101239370107094F8AC12E5
:10F0E800994215D0206884F8AC32114601F093FBA0
:10F0F800002084F8AC0210BD03FB014203FB014170
:10F10800002302F5B67281F86D31E4E70120F2E7D9
:10F118000220F0E738B5436801F00F029A4204462E
:10F1280028D811F0800F01F007024FF0280317D0FC
:10F1380002FB0333191D03440144012058710025C3
:10F148008D700A7094F8AC32012B15D00123206819
:10F1580084F8AC3201F07FFB84F8AC52284638BD05
:10F1680003FB020103FB0203002001F5B67183F8DB
:10F178006D01E4E70120F2E70220F0E711F0800FCB
:10F1880018BF01F0070110B54FF0280417BF01FBA5
:10F19800044404FB01000434001908BF00F5B670EC
:10F1A80099B21AB90273C180002010BD01220273FE
:10F1B8008360F9E70268002180F8E4120123C0F8AF
:10F1C800EC32B2F854309BB243F00103A2F8543049
:10F1D800B2F854309BB243F00203A2F85430084608
:10F1E80070477047294B1A6830BB02F4C062B2F509
:10F1F800806FD3F8802022F48072C3F880201AD15F
:10F208001A6822F4C06242F400721A60204A126836
:10F2180032214A431F49B2FBF1F2013259694905CB
:10F2280000D522B95B69580503D400207047013A1C
:10F23800F4E7032070477047B0F5007F1FD102F450
:10F24800C062B2F5806FD3F8802042F48072C3F8B0
:10F258008020EAD11A6822F4C06242F400721A606F
:10F268000B4A126832214A430A49B2FBF1F20132D1
:10F2780059694905D6D5002AD4D0013AF8E722F4CD
:10F28800C06242F480621A60CFE700BF007000409D
:10F298004402002040420F00024A936843F480432E
:10F2A80093607047007000402DE9F341044640B375
:10F2B8000368DF0714D423689E075BD423681E07FE
:10F2C80000F1A48023685D0700F1CB8023689B06CA
:10F2D80000F13281E069002840F06081002028E0D8
:10F2E800A14DAB68EA6803F00C030C2B0BD102F0BC
:10F2F8000303032B09D12B689D03DCD56368002B1E
:10F30800D9D1012015E0082BF4E76368B3F5803FF5
:10F3180012D12B6843F480332B60FEF7AFFE06460C
:10F328002B689803C7D4FEF7A9FE801B6428F7D979
:10F33800032002B0BDE8F081B3F5A02F04D12B68FB
:10F3480043F480232B60E4E72A6822F480322A60A1
:10F358002A6822F480222A60002BDED1FEF78EFE76
:10F3680006462B689903A6D5FEF788FE801B6428FD
:10F37800F7D9DDE77C4DAB68EA6803F00C030C2B8A
:10F3880017D102F00303022B15D12B685A0502D5B9
:10F39800E368002BB5D06B68226923F0FE4343EA8B
:10F3A80002636B60714B1868FEF732FE002885D047
:10F3B800A7E7042BE8E7E368BBB12B6843F4807345
:10F3C8002B60FEF75BFE06462B685B0507D56B686E
:10F3D800226923F0FE4343EA02636B606EE7FEF79F
:10F3E8004DFE801B0228EFD9A2E72B6823F4807317
:10F3F8002B60FEF743FE06462B685F057FF55EAF80
:10F40800FEF73CFE801B0228F6D991E76369564D4A
:10F418009BB1D5F8943043F00103C5F89430FEF75A
:10F428002DFE0646D5F8943098073FF54BAFFEF70A
:10F4380025FE801B0228F5D97AE7D5F8943023F009
:10F448000103C5F89430FEF719FE0646D5F8943046
:10F4580099077FF537AFFEF711FE801B0228F5D913
:10F4680066E7414DAB6DDA0027D4AB6D43F08053AE
:10F47800AB65AB6D03F080530193019B01273C4EB4
:10F488003368DB051BD5A368012B29D1D5F890304B
:10F4980043F00103C5F89030FEF7F0FD41F28838DB
:10F4A8000646D5F89030990740D5002F3FF40EAFA7
:10F4B800AB6D23F08053AB6508E70027DFE73368BF
:10F4C80043F480733360FEF7D9FD80463368D8056E
:10F4D800D9D4FEF7D3FDA0EB08000228F6D927E718
:10F4E800052B06D1D5F8903043F00403C5F89030C9
:10F4F800CCE7D5F8902022F00102C5F89020D5F885
:10F50800902022F00402C5F89020002BC4D1FEF709
:10F51800B5FD41F288380646D5F890309A07C4D52B
:10F52800FEF7ACFD801B4045F6D901E7FEF7A6FDC6
:10F53800801B4045B5D9FBE6A3690B4DD3B1D5F87F
:10F54800983043F00103C5F89830FEF797FD06465A
:10F55800D5F898309F073FF5BDAEFEF78FFD801BAD
:10F568000228F5D9E4E600BF001002404C02002052
:10F5780000700040D5F8983023F00103C5F89830A2
:10F58800FEF77CFD0646D5F8983098077FF5A2AEC1
:10F59800FEF774FD801B0228F5D9C9E6484DAB6813
:10F5A80003F00C030C2B57D02B68022823F0807330
:10F5B8002B603AD1FEF762FD06462B6899012ED4DE
:10F5C800EA68404B1340226A1343A26A43EA0223C3
:10F5D800E26A43EAC263626A013A43EA0213226BAF
:10F5E8005208013A43EA4253626B5208013A43EA2D
:10F5F8004263EB602B6843F080732B60EB6843F049
:10F608008073EB60FEF73AFD04462B689A013FF5DC
:10F6180065AEFEF733FD001B0228F6D988E6FEF733
:10F628002DFD801B0228C8D982E6EB6823F003036E
:10F63800EB60EB6823F0887323F48033EB60FEF70C
:10F648001DFD04462B689B017FF548AEFEF716FDAD
:10F65800001B0228F6D96BE601283FF46AAEEB6876
:10F66800226A03F0030191427FF44BAE616A03F012
:10F67800F0020139B2EB011F7FF443AEA16A03F433
:10F68800FE42B2EB012F7FF43CAEE16A03F0784210
:10F69800B2EBC16F7FF435AE226B520803F4C001A0
:10F6A800013AB1EB425F7FF42CAE626B520803F073
:10F6B800C063013AB3EB426F3FF410AE21E600BFDE
:10F6C800001002400C809F01174B9A6802F00C0250
:10F6D800042A23D09A6802F00C02082A20D09A68DB
:10F6E80002F00C020C2A1DD1D968DA68D868DB68E8
:10F6F80001F00301C3F341630329C2F30312C0F30A
:10F70800062003F101030CBF084909495B000132D7
:10F71800B1FBF2F25043B0FBF3F070470448704776
:10F7280002487047002070470010024000127A001B
:10F738000024F4002DE9F8430E46054610B90120CF
:10F74800BDE8F8836D4A136803F00F038B4245D375
:10F75800296811F001084CD12A68910740F1A78067
:10F76800674B12F0040F1EBF996841F4E06199607D
:10F77800120741BF9A6822F47C5242F4E0629A6010
:10F788009A68A96822F0F0020A439A605B4C2368E1
:10F7980003F00F03B34200F293802A68584C12F02A
:10F7A800040F40F0A380130706D5A3682A6923F441
:10F7B800605343EAC203A360FFF786FFA368514A78
:10F7C800C3F30313D35C03F01F03D8404E4B1860F8
:10F7D8004E4B1868BDE8F843FEF71ABC136823F0CF
:10F7E8000F030B431360136803F00F038B42A6D17A
:10F7F800AEE76F68424C032F236849D19B019ED521
:10F80800E368E26803F00303032BE3680CBF404896
:10F818004048C2F30312C3F306230132B0FBF2F2ED
:10F828005343E268C2F3416201325200B3FBF2F380
:10F83800394A93421AD84FF00008A36823F003030B
:10F848003B43A360FEF71AFC41F288390746A368D8
:10F858006A6803F00C03B3EB820F3FF47DAFFEF749
:10F868000DFCC01B4845F2D9032069E7A36813F0D3
:10F87800F00F04D08807DED5AB68002BDBD1A36876
:10F8880023F0F00343F08003A3604FF08008D4E72F
:10F89800022F09D113F4003F3FF451AFFFF714FFD3
:10F8A8001D4B9842C7D9EAE713F4806FF4E7B8F123
:10F8B800800F01BF124A936823F0F003936065E755
:10F8C800236823F00F0333432360FEF7D7FB41F28D
:10F8D80088380746236803F00F03B3423FF45DAF4F
:10F8E800FEF7CCFBC01B4045F4D9BDE7A368E96827
:10F8F80023F4E0630B43A36055E700BF00200240F8
:10F9080000100240A0710108440200204C020020AF
:10F9180000127A000024F40000B4C4042DE9F34175
:10F928000446006810F4002039D0994DAB6DD8001A
:10F9380027D4AB6D43F08053AB65AB6D03F08053B8
:10F948000193019B0126934F3B6843F480733B600E
:10F95800FEF794FB80463B68D90514D5D5F890305E
:10F96800226C13F4407302D0934240F0EB80D5F838
:10F978009030226C23F440731343C5F89030002074
:10F9880008E00026DFE7FEF779FBA0EB0800022875
:10F99800E1D903201EB1AB6D23F08053AB6523681A
:10F9A800DE0708D57A496568D1F8882022F0030275
:10F9B8002A43C1F888209D0708D57549A568D1F85C
:10F9C800882022F00C022A43C1F88820590708D55C
:10F9D8006F49E568D1F8882022F030022A43C1F83F
:10F9E80088201A0708D56A492569D1F8882022F0A5
:10F9F800C0022A43C1F888209F0608D56449656972
:10FA0800D1F8882022F440622A43C1F888205E0693
:10FA180008D55F49A569D1F8882022F440522A43C5
:10FA2800C1F888201D0608D55949E569D1F888200C
:10FA380022F440422A43C1F88820D90508D5544900
:10FA4800256AD1F8882022F440322A43C1F8882058
:10FA58009A0508D54E49656AD1F8882022F44022D3
:10FA68002A43C1F888205F050FD54949A56AD1F80E
:10FA7800882022F440122A43C1F88820B5F5801F57
:10FA880002BFCA6842F48012CA601E050FD54049F9
:10FA9800E56AD1F8882022F440022A43C1F8882078
:10FAA800B5F5800F02BFCA6842F48012CA60DD044F
:10FAB8000FD53749256BD1F8882022F040722A43A8
:10FAC800C1F88820B5F1807F02BFCA6842F480126D
:10FAD800CA6099040FD52E49656BD1F8882022F0A9
:10FAE80040622A43C1F88820B5F1006F02BFCA6896
:10FAF80042F48012CA605A040FD52549A56BD1F883
:10FB0800882022F040622A43C1F88820B5F1006FAE
:10FB180002BFCA6842F48012CA601B040FD51C4A8F
:10FB2800E16BD2F8883023F040530B43B1F1805F8A
:10FB3800C2F8883003D1D36843F48033D36002B06D
:10FB4800BDE8F081D5F89020D5F8903043F48033A3
:10FB5800C5F89030D5F8903022F4407123F4803302
:10FB6800D207C5F89030C5F890107FF500AFFEF7C2
:10FB780085FA41F288380746D5F890309B073FF55B
:10FB8800F6AEFEF77BFAC01B4045F5D901E700BF8A
:10FB98000010024000700040024AD36A1843D06245
:10FBA800704700BF00100240B0F1904F08B509D16E
:10FBB8000120FFF7F1FF254AD36A23F00103D3623E
:10FBC800002008BD224B984207D10220FFF7E4FF2E
:10FBD8001E4AD36A23F00203F1E71E4B984207D16D
:10FBE8000420FFF7D9FF194AD36A23F00403E6E794
:10FBF800194B984207D10820FFF7CEFF134AD36A62
:10FC080023F00803DBE7154B984207D11020FFF7D4
:10FC1800C3FF0E4AD36A23F01003D0E7104B984273
:10FC280007D12020FFF7B8FF084AD36A23F0200342
:10FC3800C5E70C4B984207D14020FFF7ADFF034AB8
:10FC4800D36A23F04003BAE70120BAE70010024064
:10FC58000004004800080048000C00480010004854
:10FC680000140048001800482DE9F04F02460D68BE
:10FC780095FAA5F44FF0010EB4FA84F403274FF077
:10FC88000F0C6FEA050835FA04F001D1BDE8F08FD2
:10FC98000EFA04F32B4067D04868461E012E1ED882
:10FCA800966893FAA3F9B9FA89F94FEA490907FA64
:10FCB80009F926EA090993FAA3FA8E68BAFA8AFAC0
:10FCC8004FEA4A0A06FA0AF646EA090696605668AC
:10FCD80008EA0609CE686E4349EA06065660D66801
:10FCE80093FAA3F9B9FA89F94FEA490907FA09F920
:10FCF80026EA090993FAA3FA0E69BAFA8AFA4FEAC8
:10FD08004A0A06FA0AF646EA09060228D66018D10F
:10FD1800FF2BD1F814A029D8D2F8209093FAA3F693
:10FD2800B6FA86F6B6000CFA06F629EA060993FA38
:10FD3800A3F6B6FA86F6B6000AFA06F646EA090601
:10FD48001662166893FAA3F9B9FA89F94FEA4909CC
:10FD580007FA09F926EA090693FAA3F3B3FA83F333
:10FD68005B0098403043106001348CE7D2F824904F
:10FD78001E0A96FAA6FBBBFA8BFB4FEA8B0B0CFA12
:10FD88000BFB29EA0B0996FAA6F6B6FA86F6B60030
:10FD98000AFA06FA4AEA09065662D2E7F8B504688A
:10FDA80014F0010405460F463ED13A69BB68016864
:10FDB80013437A6913431D4A0A4013430360436897
:10FDC800FA6823F44053134343608368BA6923F401
:10FDD8004073134383604FF4406000F059F93E6864
:10FDE80000B37F68F7B1B3B2114A214632F8132045
:10FDF8002346F0F70DFE7A080302090241EA106172
:10FE0800981841F100013A462346F0F701FEC0F385
:10FE18001300E8602046EB6AB6B223F00F031E43D6
:10FE2800EE62F8BD0120F6E70120FAE7F3E9FFEFFB
:10FE3800B8710108024B1868C0F38020704700BFF2
:10FE480000100240024BD3F89000C0F34000704706
:10FE580000100240024B1868C0F34060704700BFB2
:10FE680000100240044B054A9B68C3F30313D35C9C
:10FE780003F01F03D840704700100240A07101082A
:10FE8800044B054A9B68C3F30223D35C03F01F03AA
:10FE9800D840704700100240B0710108124B9A68B0
:10FEA80002F00C02082A1BD00C2A1BD1DA680F4872
:10FEB8000F4902F00302032A08BF0146D868DA682E
:10FEC800DB68C3F34163C0F30620C2F303120133B6
:10FED800484301325B00B0FBF2F0B0FBF3F070472F
:10FEE80002487047024870470010024000127A002A
:10FEF8000024F400164A08B5136843F480731360AD
:10FF0800FFF798FF0028FBD0536823F0FE4343F027
:10FF18008043536001239360936803F00C03042B20
:10FF2800FAD14FF4807313601360FFF793FF002832
:10FF3800FBD14FF4805140F23B73D1609061136262
:10FF4800D2F8943043F40003C2F8943008BD00BFDF
:10FF580000100240032810B52DD12D4C2D4AD4F89D
:10FF6800883003F0030343F44033934209D0B3F1DC
:10FF7800031F0CD0013A934210D1BDE81040FFF79F
:10FF88008DBFFFF757FF002840D1002010BDFFF7B5
:10FF980059FF003818BF0120C003F7E7FFF77EFFBD
:10FFA800FFF760FFA3681C4AC3F3C223D35C03F0C6
:10FFB8001F03D840EAE70C2817D1154B174AD3F886
:10FFC800883003F00C0343F440239342D9D0B3F1B3
:10FFD8000C1FDCD0043A9342CFD0FFF75FFFFFF746
:10FFE80041FFBDE81040FFF74BBF3028CDD1084B8B
:08FFF8000B4AD3F8883003F036
:020000040801F1
:10000000300343F440139342BFD0B3F1301FC2D04A
:10001000103AE4E70548BDE7001002400200030083
:10002000B071010808000C00200030000024F4002A
:10003000C02808B501D0002008BD144B144AD3F8DD
:10004000883003F0C00343F44003934209D0B3F176
:10005000C01F0CD0403A934210D1BDE80840FFF7D2
:1000600021BFFFF7EBFE0028E5D00A48E4E7FFF7E1
:10007000EDFE003818BF0120C003DDE7FFF712FFD7
:10008000FFF7F4FEBDE80840FFF7FEBE0010024097
:100090008000C0000024F40008B5134BD3F888306A
:1000A0001840B0F5006F09D0B0F5406F0DD0B0F535
:1000B000806F11D1BDE80840FFF7F4BEFFF7BEFE28
:1000C0000A4B002818BF184608BDFFF7BFFE0038CE
:1000D00018BF0120C003F7E7FFF7E4FEFFF7C6FEF5
:1000E000BDE80840FFF7D0BE001002400024F40035
:1000F00003685B0670B502462DD4D1E90036334360
:10010000CE68056848690C6A33430E6933438E69CB
:1001100003433343CE6925F47F45334325F0BF05C0
:1001200023432B43136053688D6823F4706323F0DB
:10013000040345EA10401843B5F5006F50603EBF18
:10014000536843F480535360B4F5005F01D18B8C46
:100150001361002000E00120D36923F40063D36120
:1001600070BD00002B4A036890420ED0B0F1804F62
:100170000BD0A2F59432904207D002F580629042F3
:1001800003D002F59632904215D14A6823F07003ED
:100190001343204A904219D0B0F1804F16D0A2F5F7
:1001A0009432904212D002F5806290420ED002F555
:1001B000963290420AD0184A904207D002F58062E7
:1001C000904203D002F58062904203D1CA6823F4C2
:1001D0004073134303608B68C3620B8883620D4BCB
:1001E00098420FD003F5006398420BD003F54063AB
:1001F000984207D003F58063984203D003F58063EB
:10020000984201D10B690363436943F001034361E1
:1002100000207047002C0140004001401C4B9842D8
:100220000BD103F558431A6C42F480421A641A6CDD
:1002300022F480421A6400207047164B98420AD17B
:1002400003F5E6339A6B42F400329A639A6B22F418
:1002500000329A63EFE7104B984209D103F5E4337B
:100260009A6B42F480229A639A6B22F48022F0E720
:100270000A4B984209D103F5E2339A6B42F400220B
:100280009A639A6B22F40022E3E70120704700BFD3
:10029000003801400044004000480040004C00404D
:1002A00038B50368DB0704460D4659D42A69AB68A4
:1002B000016813436A691343EA691343294A0A40F0
:1002C000134303604368EA6823F4405313434360D5
:1002D0008368AA6923F4407313438360224B9842D6
:1002E00020D10320FFF73AFE2B6840B36A6832B38F
:1002F0000B2B15D81D4951F82330E969B0FBF3F0F9
:10030000B1F5004F4FEA520325D103EB4003B3FB95
:10031000F2F34FF6F0721A40C3F342031343E36063
:1003200000200DE0124B984201D10C20DAE7114B6E
:10033000984201D13020D5E70F4B984207D00120D9
:10034000E26A2B8822F00F021343E36238BDC0201B
:10035000FFF76EFEC8E70344B3FBF2F39BB2DEE7A0
:100360000120F3E7F369FFEF00380140D071010885
:100370000044004000480040004C004000234BF681
:100380008072A0F84430A0F8402018467047B0F8BA
:10039000403023F47E535B045B0CA0F84030002017
:1003A000704784B010B503AC84E80E00BDE810407F
:1003B0000123A0F840300023A0F8403004B0A0F89A
:1003C0004430A0F85030184670470000F0B591F85E
:1003D00000C0CD7830F82C4024F4EC4424F07004B4
:1003E000240403466246240C032D4BD8DFE805F0B5
:1003F0000247454344F40074284648F280063443DB
:1004000023F8224033F82240984FA4B23C4044EAFB
:100410000C04344323F822400C7B03EBCC0C002C5F
:100420007DD1CC884E78640864006EB3B3F8501068
:100430001CFA81F1A1F8004433F82210490609D5CD
:1004400033F8221089B2394041F4004141F0C00133
:1004500023F8221033F82210854C89B2012D01EACD
:10046000040101D081F0200141F4004141F08001FC
:1004700023F82210B2E044F4C0640020BDE744F445
:100480008064FAE70120B8E7B3F850501CFA85F50C
:10049000A5F80444B3F850401CFA84FC0C693E2CC7
:1004A00027D965097349E60608BF05F1FF3541EA1A
:1004B000852189B2ACF8061433F822104F040DD50B
:1004C00033F8221021F4E04121F070010904090CF5
:1004D00041F4404141F0800123F8221033F822100A
:1004E00021F4804121F070010904090C81F440518C
:1004F000BAE774B9BCF8061421F4F8410904090CF0
:10050000ACF80614BCF806146FEA41416FEA514199
:10051000CFE76108E40748BF01318902C9E7022D2E
:1005200033F822405BD1A4B23C4044F4014444F08F
:10053000800423F82240B3F850600C891CFA86F638
:1005400064086400A6F800444C89B3F8506064085D
:100550001CFA86F66400A6F804444978002948D1BC
:1005600033F822104E040DD533F8221021F4E04167
:1005700021F070010904090C41F4404141F080016F
:1005800023F8221033F822104D060DD533F822102F
:1005900021F4E04121F070010904090C41F400410B
:1005A00041F0C00123F8221033F8221021F48041D9
:1005B00021F070010904090C48F2800481F44051D3
:1005C000214323F8221033F8221021F4E04121F0D6
:1005D00040010904090C0C4323F82240F0BD24F427
:1005E000E24424F070042404240C264323F82260FF
:1005F000A1E733F822104C040DD533F8221021F472
:10060000E04121F070010904090C41F4404141F03E
:10061000800123F8221033F8221049060DD533F853
:10062000221021F4E04121F070010904090C41F489
:10063000004141F0C00123F8221033F822100C4C85
:1006400089B22140012D18BF81F0200141F4004101
:1006500041F0800123F8221033F8221021F4804168
:1006600021F070010904090CFEE600BF8F8FFFFF27
:10067000BF8FFFFF0080FFFF4A780B78097BD9BB53
:100680000AB330F8232051060DD530F8232022F488
:10069000E04222F070021204120C42F4004242F0D6
:1006A000C00220F8232030F8232022F4E04222F078
:1006B00040021204120C42F4004242F0800220F880
:1006C00023200020704730F8232052040DD530F845
:1006D000232022F4E04222F070021204120C42F4B1
:1006E000404242F0800220F8232030F8232022F4F8
:1006F000804222F07002DCE7002A4AD130F8232041
:1007000051040DD530F8232022F4E04222F070028B
:100710001204120C42F4404242F0800220F82320DE
:1007200030F8232052060DD530F8232022F4E04281
:1007300022F070021204120C42F4004242F0C00295
:1007400020F8232030F8232022F4E04222F0700227
:100750001204120C42F4004242F0C00220F823209E
:1007600030F8232022F4804222F070021204120C8E
:1007700048F280010A4320F8232030F8232022F495
:10078000E04222F040021204120C114320F8231020
:1007900097E730F8232051040DD530F8232022F4B8
:1007A000E04222F070021204120C42F4404242F085
:1007B000800220F8232030F8232052060DD530F88F
:1007C000232022F4E04222F070021204120C42F4C0
:1007D000004242F0C00220F8232030F8232022F407
:1007E000E04222F070021204120C42F4404242F045
:1007F000800220F8232030F8232022F4E04222F067
:1008000040021204120C48F280010A4320F823200F
:1008100030F8232022F4804222F07002B3E74B78B4
:100820000A788BB130F8223023F4E04323F0400300
:100830001B041B0C83F0100343F4004343F08003BC
:1008400020F822300020704730F8223023F4804313
:1008500023F070031B041B0C83F48053ECE70B7B29
:100860003BBB4B780A7833B330F822305B060DD5AA
:1008700030F8223023F4E04323F070031B041B0CF8
:1008800043F4004343F0C00320F82230CB78012B1F
:100890000FD030F8223023F4E04323F040031B0450
:1008A0001B0C83F0200343F4004343F0800320F843
:1008B00022300020704730F822305B040DD530F82C
:1008C000223023F4E04323F070031B041B0C43F499
:1008D000404343F0800320F8223030F8223023F4E4
:1008E000804323F070031B041B0C83F44053DAE7AE
:1008F0000123A0F8403003220023A0F84430A0F8E0
:1009000040201846704711B98023A0F84C300020D1
:100910007047B0F858306FEA43436FEA53439BB2D5
:10092000A0F8583000207047B0F85830C3F30E03D9
:10093000A0F8583000207047B0F8440080B27047EB
:1009400002F58062013310445B0801EB4303401A57
:10095000994200D170470A880A520231F8E7000034
:100960002DE9F0474A780E7B012A05460C4640F0F7
:100970001781D1F810A08F694969574528BF57469C
:1009800016BBBFB2E2883B46FFF7DAFFB5F850204E
:10099000237805F2024111FA82F202EBC3021780BA
:1009A000227835F8223023F4E04323F040031B047F
:1009B0001B0C83F0300343F4004343F0800325F81D
:1009C00022300020BDE8F087E378266A94F800C062
:1009D000022B40F0CE80B24530F82C2080F0B2805F
:1009E00022F4E04222F070021204120C42F401429E
:1009F00042F0800220F82C2030F82C80B0F85020F3
:100A0000F61B18F04008266201EB0709BBB24ED076
:100A100000F2064E1EFA82F222F83C306289FFF79D
:100A20008FFFB2456278C4F8149036BFF31B0023E1
:100A30003E462362B3B26ABBB5F85020217805F276
:100A4000024010FA82F23E2E02EBC1020FD9700969
:100A5000AE49F60608BF00F1FF3041EA802189B2B5
:100A60001180228949462846FFF76AFF98E75EB958
:100A7000118821F4F8410904090C118011886FEAEA
:100A800041416FEA5141EAE77108F00748BF01317F
:100A90008902E4E7012AE4D1B5F85020217805F273
:100AA000024010FA82F202EBC1021380D9E700F291
:100AB000024E1EFA82F222F83C302289FFF740FFF4
:100AC000B2456278C4F8149036BFF31B43463E46E5
:100AD0002362B3B24ABBB5F85020217805F2064034
:100AE00010FA82F23E2E02EBC1020BD9700987493F
:100AF000F70608BF00F1FF3041EA802189B211807A
:100B00006289AFE75EB9118821F4F8410904090C44
:100B1000118011886FEA41416FEA5141EEE7710897
:100B2000F60748BF01318902E8E7012AE8D1B5F8A4
:100B30005020217805F2064010FA82F202EBC10241
:100B40001380DDE722F4E24222F070021204120C5C
:100B500042F4004242F0800220F82C20B0F85020ED
:100B600000F2024313FA82F2B3B222F83C30228937
:100B70007AE730F82C20F61B12F0400F2662B0F80E
:100B80005020BBB207D000F2064616FA82F222F8D5
:100B90003C30628968E700F2024616FA82F2E4E726
:100BA000002E3CD18A690B699A4284BFD61A1A4634
:100BB000B0F850308E6100F20640097810FA83F3E5
:100BC0003E2A03EBC10315D95109D0064F4A08BF8D
:100BD00001F1FF3142EA812292B21A80227835F87F
:100BE000223023F4804323F070031B041B0C83F496
:100BF0004053E0E65AB91A8822F4F8421204120C63
:100C00001A801A886FEA42426FEA5242E4E75108BA
:100C1000D20748BF0131890289B21980DEE7CB785B
:100C2000022B75D1002A4BD1B0F850200B7800F27E
:100C3000024111FA82F202EBC30223693E2B22D950
:100C400058093249DF0608BF00F1FF3041EA802130
:100C500089B21180B5F85020217805F2064010FACB
:100C600082F23E2B02EBC10220D8002B46D1138822
:100C700023F4F8431B041B0C138013886FEA4343CF
:100C80006FEA53431AE05BB9118821F4F841090473
:100C9000090C118011886FEA41416FEA5141D7E791
:100CA0005908DE0748BF01318902D1E75909D80642
:100CB000164B08BF01F1FF3143EA81239BB2138039
:100CC000E369002B8AD0227835F8221044F24003E1
:100CD00003EA01008B4302D000287FF47FAF35F890
:100CE000223023F4E04323F070031B041B0C43F475
:100CF000004343F0C00325F822306FE75908DB07B3
:100D000048BF0131890289B21180D9E70080FFFF15
:100D1000012B5DD18B6909698B428ABF581A00206B
:100D20000B46A061002A7FF459AFB5F85020217816
:100D300005F2024010FA82F23E2B02EBC10221D9E9
:100D400058092449DF0608BF00F1FF3041EA80213D
:100D500089B21180B5F85020217805F2064010FACA
:100D600082F23E2B02EBC1021FD84BBB138823F447
:100D7000F8431B041B0C138013886FEA43436FEA8C
:100D800053431AE05BB9118821F4F8410904090CB6
:100D9000118011886FEA41416FEA5141D8E7590843
:100DA000DE0748BF01318902D2E75909D806094B4D
:100DB00008BF01F1FF3143EA81239BB213800DE7A5
:100DC0005908DB0748BF0131890289B2118005E764
:100DD0000120F7E50080FFFF02F58062F0B51044C6
:100DE0005D080C462E46471A3A19023436B9DB071D
:100DF00044BF30F8153001F81530F0BD128892B2BA
:100E000004F8022C120A04F8012C013EECE7D0F899
:100E1000D43200EB830010B5D0F8C04284B1D0F8D2
:100E2000C4325BB194F84000FF2807D09B6894F867
:100E3000412021469847FF2384F84030002000E0FD
:100E4000032010BD0A23038000487047EC020020F5
:100E500070B5822106460F4800F028FB01210546A7
:100E60000C4800F023FB812104460A4800F01EFBD9
:100E70000DB11022AA711CB14022227100226271B0
:100E800018B140220271002242714323014833808D
:100E900070BD00BFA8020020FFF7DABFFFF7D8BF80
:100EA00038B5D0F8D432B033044650F823507DB171
:100EB00001F078F8D4F8D43204EB83042946D4F84E
:100EC000C43241F84C0FDB68686C9847002038BD8D
:100ED0000320FCE7F8B5D0F8D462D0F8C87200EB74
:100EE00086060A46D6F8C05225B3142401F00F0C2A
:100EF00004FB0C039C6984B14FF0280E0EFB0C77A9
:100F0000FF6BB4FBF7FC07FB1C4434B99C61224621
:100F1000234601F035F820460BE0D6F8C4321C69B0
:100F200000276F65002CF6D0A86C05F15001A04792
:100F30003846F8BD0320FCE7D0F8D4322DE9F34160
:100F400000EB83034FF00008D3F8C0728DF80580E2
:100F500005460E46ADF80680002F6ED00A7812F0D6
:100F600060042ED0202C64D1CC8891F801C00CB341
:100F7000120613D5D3F8C432224639469B68604620
:100F80009847F288072A28BF07223946284600F0EA
:100F9000FCFC4446204602B0BDE8F081402C28BF4E
:100FA000402487F840C087F841402246394600F087
:100FB00001FDEEE7D3F8C43222469B6860469847AD
:100FC000E8E74F780B2F34D801A353F827F000BF80
:100FD00001100108950F01083310010833100108B2
:100FE00033100108331001083310010833100108D1
:100FF0003310010833100108171001082B100108E5
:1010000090F89C32032B14D102220DF1060100F05E
:10101000BCFC3C46BEE790F89C32032B09D1012270
:101020000DF1050100F0B1FCB4E790F89C32032B00
:10103000B0D03146284600F081FC0324AAE700BF67
:1010400038B504460025812100F063FF0121258782
:10105000204600F05EFFA4F878518221204600F07F
:1010600058FFD4F8D432E56404EB8303D3F8C022EC
:101070008AB1D3F8C4325B689847D4F8D432B0331D
:1010800054F8230000F096FFD4F8D432B03344F87B
:101090002350C4F8BC52002038BDF8B504465C208B
:1010A00000F084FF054630B9D4F8D432B03344F8A8
:1010B000230002253BE05C22002102F0D9FDD4F898
:1010C000D432B033012644F8235002224023812138
:1010D000C4F8BC52204600F010FF402302223146E3
:1010E0002687204600F009FF10230322A4F84E3083
:1010F00082210823A4F87861204600F0FEFED4F88F
:10110000D432A4F84C6004EB83030027D3F8C43234
:101110006F641B6898476A6C6F65AF65002AC8D01A
:10112000257C4023314620461DB900F032FF284679
:10113000F8BD00F02EFF3D46F9E739B1D0F8D432C2
:1011400000EB8300C0F8C4120020704703207047F2
:10115000D0F8D432B03350F823301BB199641A65FB
:101160000020704703207047D0F8D432B03350F8D5
:10117000233013B159640020704703207047D0F822
:10118000D432B03310B550F823205AB1546D012336
:1011900054B95365136DC362926C812100F0F0FE67
:1011A000204610BD0320FCE71846FAE7D0F8D42209
:1011B000B03208B550F8222032B1526C40230121E0
:1011C00000F0E7FE002008BD0320FCE778B1002313
:1011D000C0F8B832C0F8C432C0F8D03209B1C0F893
:1011E000B412012380F89C32027000F029BE032063
:1011F000704710B5044600F077FE012384F89C3256
:10120000D4F8B8321BB15B68217920469847002397
:10121000C4F8C432C4F8B432C4F8D0322046BDE8B1
:10122000104000F04FBE13B500230446ADF8063061
:1012300081B1CB6AC0F8B81223B10DF1060098470E
:10124000C4F8D002D4F8D8320133C4F8D832002020
:1012500002B010BD0320FBE700F03DBED0F8B8326D
:101260000BB11B6818471846704708B5D0F8B8325C
:101270005B689847002818BF032008BD38B50446AE
:1012800000F2AA25284600F04EFB012394F8AA128A
:10129000C4F89432B4F8B032C4F8983201F01F03A5
:1012A000012B08D0022B0CD08BB929462046BDE873
:1012B000384000F019B929462046BDE8384000F012
:1012C00067BA29462046BDE8384000F090BA20466B
:1012D00001F08001BDE8384000F024BE70B504463E
:1012E000164609BBD0F89432032B0CD1D0E9573203
:1012F00093420AD99B1A9A42C0F85C3128BF1A4619
:10130000314600F064FB002070BD90F89C32032B46
:1013100006D1D0F8B8321B6913B1C0F8D41298477F
:10132000204600F05CFBEEE790F89C32032BEAD1FC
:10133000D0F8B8329B69002BE5D00022BDE87040A0
:10134000C0F8D422184773B504461646002941D187
:10135000D0F89422022A0FD1D0E90752954214D92D
:10136000AA1A0191C261314600F01CFB019B1A468A
:101370001946204600F00DFE94F8A03213B1002368
:1013800084F8A032002002B070BD0ED1826995426F
:101390000BD8D0F89852AA4207D20A46019100F021
:1013A00001FB019BC4F89832E1E794F89C32032BCF
:1013B00008D1D4F8B832DB6823B10022C4F8D422B3
:1013C000204698478021204600F0ACFD204600F0E2
:1013D00011FBD1E790F89C32032BD3D1D0F8B8326F
:1013E0005B69002BCED00022C0F8D42202B0BDE849
:1013F00070401847F8B5012380F89C32D0F8B83215
:1014000000210446C0F894124160C0F8A41280F88C
:10141000A012B3B90026002240251146012740231F
:10142000204600F06AFDA4F86471C4F860512B46B0
:1014300000228021204600F060FDA784256230460E
:10144000F8BD5B68002BE5D098470028E2D0032662
:10145000E1E701740020704790F89C32042B1EBF16
:1014600090F89C32DBB280F89D32042380F89C32E5
:101470000020704790F89C32042B02BF90F89D32F8
:10148000DBB280F89C320020704708B590F89C22AF
:10149000032A05D1D0F8B83213B1DB6903B19847FC
:1014A000002008BD002070470020704710B542881A
:1014B00003789A420AD90478204423444478052CBE
:1014C0009BB2F6D184788C42F3D110BD0020FCE7AA
:1014D00010B58021044600F025FD20460021BDE81E
:1014E000104000F01FBD00002DE9F3410D7805F01C
:1014F0006005202D04460E4614D0402D12D0002D3C
:1015000040F00A814F78092F00F20681DFE817F0DA
:101510000B013201040121010401860016000401BF
:10152000F300A200D4F8D432AE33314654F823305D
:101530009B68204602B0BDE8F04118470023ADF893
:1015400006304B881A0A013A062A37D8DFE802F03B
:10155000041C293636515B00D0F8B4321B68207C5D
:101560000DF106019847F288002A00F0FF80BDF8CF
:1015700006301BB39A4228BF1A46ADF80620014632
:10158000204600F002FA1CE0027CD0F8B83232B9F2
:101590009B6A0DF10600984702234370E3E7DB6A7C
:1015A000F7E7DBB2052B09D8DFE803F0030F1317C9
:1015B0001B1FD0F8B4325B68002BD0D12046FFF758
:1015C00087FF284602B0BDE8F081D0F8B4329B68AE
:1015D000F2E7D0F8B432DB68EEE7D0F8B4321B693A
:1015E000EAE7D0F8B4325B69E6E7D0F8B4329B6939
:1015F000E2E7037C002BE1D1D0F8B8320DF1060010
:101600005B6B9847AFE7037C002BD7D1D0F8B8329B
:101610000DF106001B6B98470723BEE78B88002B54
:10162000CCD1CB88002BC9D14E887F2EC6D890F85C
:101630009C32032BC2D0F1B280F89E1200F097FCCE
:10164000204600F0CCF91EB1022384F89C32B8E7A2
:101650000123FAE78E784D4F012E3E7003D9FFF734
:1016600037FF0325ADE790F89C32022B5FFA83F831
:1016700009D0B8F1030F18D0FFF72AFF39782046B8
:10168000FFF7F3FDEDE7002E70D001214160FFF779
:10169000E5FD0546204625B1FFF71AFF84F89C8238
:1016A0008FE700F09CF90323CFE75EB9022380F8AF
:1016B0009C3246603146FFF7D8FD204600F08FF996
:1016C00035467EE74168012950D0C9B2FFF7CDFD0C
:1016D000397861602046FFF7C1FD0646002845D0F5
:1016E0002046FFF7F5FE21792046FFF7BEFD0223D5
:1016F00084F89C32E4E7CA88012A7FF45FAF90F84F
:101700009C120229CBB205D833B10146002341F81F
:10171000083F35E7032B04D02046FFF7D9FE00250C
:101720004FE7011D2CE790F89C32013B022BF3D8C8
:10173000CA88022A7FF442AFD0F8A4320146002BB7
:1017400014BF0323012341F80C3F00F01EF93D466E
:1017500037E74B88012B02D1C4F8A43206E0022BF4
:101760007FF42CAF8B881B0A80F8A032204600F053
:1017700036F926E790F89C32013B022BCCD84B88F7
:10178000012B7FF41EAF0023E6E700BF9C4A002038
:1017900070B50B7803F06002402A04460E4601D073
:1017A0005B061FD494F89C32013B022B1AD8317986
:1017B0000129204617D8FFF775FE88B9D4F8B8324A
:1017C0009B686BB1C4F8D402314620469847054661
:1017D000F3881BB915B9204600F001F9284670BD01
:1017E0000325F5E72046FFF773FE0025F6E770B501
:1017F0000B788A880D7903F06003202B04460E468F
:101800005AD0402B58D09BBB4B78012B42D0032B96
:1018100027D06BBB90F89C32022BD9B268D0032939
:1018200026D105F00F0312F0800F4FF0140202FBD7
:1018300003036CD09B8CDBB105F07F06013606EB11
:10184000860600EB860615F07F0006D02946204666
:1018500000F07AFB003818BF0120306002223146C8
:1018600051E090F89C32022BDAB237D0032A03D031
:101870002046FFF72DFE0BE04B8833B9690604D0F4
:10188000F38813B9294600F04DFB204600F0A7F875
:10189000002070BD90F89C32022BDAB21ED0032AD1
:1018A000E6D14B88002BF3D16B0602D0294600F01D
:1018B00042FB204600F093F829462046FFF7F4FD4E
:1018C0000028E5D1D4F8B832C4F8D4029B68002BC4
:1018D000DED031462046BDE8704018476A06C7D0C2
:1018E000294600F01FFB8021204600F01BFBCFE7BC
:1018F0006906BDD113064CBF00F1140100F5AA71B1
:1019000000230B600222204600F03FF8C0E7B3F846
:101910006431002BACD005F07F06142303FB0606D0
:1019200006F5AA768FE70B7803704B7843704B88E7
:1019300043808B888380CB88C380704710B580211B
:10194000044600F0EFFA20460021BDE8104000F008
:10195000E9BA30B588B10024013823460134055D69
:10196000002DFAD1DBB201335B0013800B7003232F
:101970004B70022310F8012F02B930BDCA545A1C13
:10198000D2B202338D54DBB2F4E710B51346022213
:10199000C0E90633C0F894220A46002100F0F0FAAC
:1019A000002010BD08B513460A46002100F0E8FAF1
:1019B000002008BD10B513460322C0E95633C0F815
:1019C00094220A46002100F0E4FA002010BD08B578
:1019D00013460A46002100F0DCFA002008BD08B5D5
:1019E00004220023C0F8942219461A4600F0C8FACF
:1019F000002008BD08B505220023C0F8942219462E
:101A00001A4600F0C6FA002008BD0020704700000A
:101A100021280ED022281DD0202808D1164B0A6874
:101A20001A600A791A714A795A718A799A71002072
:101A30007047114B1A680A701A68120A4A705A885D
:101A40008A70DA78CA701A790A715A794A719B7960
:101A50008B71ECE7094B498800221A70C80742BF16
:101A60001A7842F001021A708A0742BF1A7842F0CF
:101A700002021A70DBE700BFA04A0020CC650020FC
:101A8000F8B50C461148FFF791FB2368B3F5006FDA
:101A900015D90020F8BD2B8831880133C3F30A0320
:101AA00089B28B421CBF395C0CF8031002F10102B1
:101AB00018BF2B802368D0B29842ECD3E9E7044DDD
:101AC000044E054FDFF814C00022F3E7A84A0020B7
:101AD000865D0020845D0020844D00208455002018
:101AE00030B5A1B03422002102A802F0C1F80125CE
:101AF000202301A801930795FDF7DAFB4022194C3A
:101B00000DEB0200002102F0B3F84FF400530FA8D0
:101B10000F93FDF707FF002213492046FFF756FBFE
:101B200012492046FFF77FFB11492046FFF705FBCE
:101B30002046FFF791FB0F4A4FF4E1331360082171
:101B40000023938091710C4A13800C4A13800C4A35
:101B500013800C4A13800C4A13700C4B1D7021B07B
:101B600030BD00BFA84A00200C03002070020020F6
:101B7000F8020020A04A0020C8650020CA650020A5
:101B8000845D0020865D0020CC650020CD650020AE
:101B900000B50A4B1B788FB063B10948FFF729FBEA
:101BA0003422002101A802F063F820236846009344
:101BB000FDF77EFB0FB05DF804FB00BFCD65002094
:101BC000A84A0020044B1888044B1B8880B29BB2A3
:101BD000C01A18BF01207047865D0020845D002078
:101BE000054A13880133C3F30A0313801388034A99
:101BF0009BB2D05C704700BF845D002084550020FC
